:020000040000FA
:10000000182700207D2300002F830000DD2300003F
:10001000DD230000DD230000DD230000DD230000E0
:100020000000000000000000000000005D21000052
:10003000DD23000000000000052100004118000041
:100040003D2300003D2300003D2300003D23000030
:100050003D2300003D2300003D2300003D23000020
:100060003D2300003D2300003D2300003D23000010
:100070003D2300003D2300003D2300003D23000000
:100080003D2300003D2300003D2300003D230000F0
:100090003D2300003D2300003D2300003D230000E0
:1000A0003D2300003D2300003D2300003D230000D0
:1000B0003D2300003D2300003D2300003D230000C0
:1000C0003D2300003D2300003D2300003D230000B0
:1000D0003D2300003D2300003D2300003D230000A0
:1000E0003D2300003D2300003D2300003D23000090
:1000F0003D2300003D2300003D2300003D23000080
:100100003D2300003D2300003D2300003D2300006F
:100110003D2300003D2300003D2300003D2300005F
:100120003D2300003D2300003D2300003D2300004F
:100130003D2300003D2300003D2300003D2300003F
:100140003D2300000000000000000000000000004F
:10015000000000000000000000000000000000009F
:10016000000000000000000000000000000000008F
:10017000000000000000000000000000000000007F
:10018000000000000000000000000000000000006F
:10019000000000000000000000000000000000005F
:1001A000000000000000000000000000000000004F
:1001B000000000000000000000000000000000003F
:1001C000000000000000000000000000000000002F
:1001D000000000000000000000000000000000001F
:1001E000000000000000000000000000000000000F
:1001F00000000000000000000000000000000000FF
:10020000DEE61E284CBBCE8F025B00003C000000E7
:1002100000000100010000000000000000000000DC
:10022000FFFF02910000000000000000000000003D
:1002300000000000000000000000000053B94AB9AF
:10024000002908BF00281CBF4FF0FF314FF0FF30DE
:1002500000F070B9ADF1080C6DE904CE00F006F8BD
:10026000DDF804E0DDE9022304B070472DE9F04732
:10027000089E0D4604468A46002B7FD18A421746C7
:1002800041D9B2FA82F24AB1C2F1200105FA02F371
:100290009740944020FA01F141EA030A4FEA1748D7
:1002A0004FEA144C1FFA87F9BAFBF8FE08FB1EA3AD
:1002B0000EFB09F14CEA0343994206D9FB1802D21E
:1002C000994200F224810EF1FF3E591AA3B2B1FB0C
:1002D000F8F008FB101100FB09F943EA0144A145BD
:1002E00005D93C1902D2A14500F20E810138A4EBD8
:1002F000090440EA0E4000211EB1D4400023C6E9A3
:100300000043BDE8F08702B9FFDEB2FA82F2002AAC
:100310004FD1CB1B4FEA174E1FFA87F80121250C4E
:10032000B3FBFEFC0EFB1C302B4608FB0CF945EA28
:100330000045A9450AD97D192CBF01230023A945F1
:1003400002D9002B00F0D9800CF1FF3CA5EB090588
:10035000A3B2B5FBFEF00EFB105508FB00F843EA14
:100360000544A04505D93C1902D2A04500F2C98038
:100370000138A4EB080440EA0C40BDE78B4208D9E1
:10038000002E00F0B1800021C6E900050846BDE856
:10039000F087B3FA83F1002946D1AB42C0F0A780C1
:1003A000824240F2A4800846002EAAD0C6E9004A44
:1003B000A7E7C2F12000974001FA02F34FEA174E77
:1003C000C14024FA00F51FFA87F894401D43B1FBA1
:1003D000FEF02B0C0EFB101100FB08FC43EA01435E
:1003E0009C4509D9FB182CBF012100219C4502D94D
:1003F000002900F095800138A3EB0C03ADB2B3FBEC
:10040000FEF10EFB113301FB08FC45EA0345AC4548
:1004100005D97D1902D2AC4500F289800139A5EBDE
:100420000C0341EA00417AE7C1F120048B4002FA53
:1004300001F705FA01FCE24020FA04F8E54000FA71
:1004400001FE134348EA0C024FEA13484FEA124CEC
:100450001FFA83F9B5FBF8FA08FB1A550AFB09F0F5
:100460004CEA054C60450AD913EB0C0C2CBF012556
:100470000025604501D9002D55D00AF1FF3AACEBBB
:10048000000C92B2BCFBF8F008FB10CC00FB09F9A1
:1004900042EA0C4CE14505D913EB0C0C01D2E145C5
:1004A0003BD8013840EA0A40ACEB090CA0FB0789B5
:1004B000CC4545464A4602D306D1C64504D201384A
:1004C000B8EB070569EB03022EB3BEEB05036CEB3B
:1004D000020C23FA01F20CFA04F42CFA01F30021C5
:1004E0001443C6E900430CE73146304609E7841A55
:1004F00065EB030301209A4656E7ACF1020C3D443C
:1005000024E702383C4434E702383C44EFE6AEF1DD
:10051000020E3B44D9E63146F3E602389C44C1E77B
:1005200002383B4468E7AAF1020A9C44A7E7023973
:100530003D4474E7704700BF2DE9E04F2746A046D1
:10054000A146A246A346A446A2B02DEC000A84F31D
:10055000008825462646A4473DEC000A22B0BDE8A7
:10056000E08F000038B54468054604F00304032C0E
:10057000816002D02CB1002000E0006800236B6095
:1005800038BD45220449054807F01EFD45210248B3
:1005900007F0E6FDEFE700BFF38D0000168E0000C8
:1005A0000B6801330B60014B1B68184700000020EB
:1005B000014B1860704700BF0000002007B50B46D4
:1005C000002102460191034801A900F06DFA03B031
:1005D0005DF804FBA10500002DE9F74FB0F81CA061
:1005E00004461AF0080F93461CD001290CBF4AF0AC
:1005F000100A4AF0200AA0F81CA004F1140003F02D
:100600007FFB40B9BA49BB48AC2207F0DDFCAC2106
:10061000B74807F0A5FD8BF31188BFF36F8F03B0C8
:10062000BDE8F08FB44FDFF8CC820AF0070A022948
:1006300006D1204607F0D5FC0028DED0012865D180
:10064000D4F81890A38BB9F1000F19DA00262568A9
:1006500023F00703C4E9006643F00103A383A38BDF
:1006600003F007025245009203D0A268002A40F02E
:10067000F18015B9002E00F02B814FF0000AEBE05D
:1006800003F00702511F012922D8002123F007039C
:10069000062A25689BB2C4E900110CD18D422A4676
:1006A00038BF0A462AB1E18B12680131E183002A82
:1006B000F8D143F002032046A38307F092FC0646DC
:1006C0000028CCD0A38B43F02003A3830026C6E7E9
:1006D000042A0DD123F007039AB22046A28307F023
:1006E00080FC054680B142F020020025A283EDE7A0
:1006F00040F21B123946404607F066FC40F21B11DF
:10070000384607F02DFD00252E46A8E7032831D1F5
:10071000BAF1000F0AD0394640464FF4AB7207F0E9
:1007200053FC4FF4AB71384607F01AFD236853B9F8
:100730003946404640F2571207F046FC40F2571146
:10074000384607F00DFD23691E6856B93946404604
:100750004FF4AD7207F038FC4FF4AD71384607F036
:10076000FFFCA38B23F0070343F006030025A383BC
:10077000A94674E704282ED1BAF1020F0AD03946EF
:10078000404640F25D1207F01FFC40F25D11384612
:1007900007F0E6FCE38B53B1394640464FF4AF72A5
:1007A00007F012FC4FF4AF71384607F0D9FC23690B
:1007B0005E6856B93946404640F2611207F004FCC3
:1007C00040F26111384607F0CBFCA38B23F00703FE
:1007D00043F00403CAE705282ED1BAF1010F0AD06D
:1007E000394640464FF4B27207F0EEFB4FF4B27157
:1007F000384607F0B5FC236853B93946404640F205
:10080000651207F0E1FB40F26511384607F0A8FCDD
:1008100023699E6856B9394640464FF4B47207F0D2
:10082000D3FB4FF4B471384607F09AFCA38B23F046
:10083000070343F0050399E7002540F26B123946A0
:10084000404607F0C1FB40F26B11384607F088FCC8
:100850002E468DE74FF0010A43F00803A38304F10D
:1008600014031846019303F04BFA40B9404620495F
:10087000AC2207F0A9FBAC211D4807F071FC8BF3FB
:100880001188BFF36F8FBAF1000F39D1002D4CD111
:1008900016B120461949B0474FF02003EFF3118BF2
:1008A00083F31188BFF36F8F019803F01BFA40B9EF
:1008B00040460F49812207F087FB81210C4807F051
:1008C0004FFC019803F02AFAA38B23F00803A383BB
:1008D000A38BDA0631D5012123F01003A383B4F8EA
:1008E0001CA00AF0070A00297FF4A1AE85E600BF2C
:1008F000508E0000168E00002E8E00004D09000064
:10090000A1680029C2D00B68002B38BF00239A468B
:1009100020464B46D1F804B0009AD847BAF1000FF0
:10092000B4D05146DAF80030EEE729464B4620466F
:10093000009A2D6807F071FBA8E713F020011EBF95
:1009400023F020030221A383C9E700BFF8B50446C2
:100950000D4600F114064FF02003EFF3118783F3E7
:100960001188BFF36F8F304603F0BCF940B90A49D4
:100970000A48812207F028FB8121074807F0F0FB95
:10098000304603F0CBF93A462046A5610121BDE887
:10099000F840FFF721BE00BF508E0000168E000009
:1009A0002DE9F04704460F4607F04DFB051E54DBCA
:1009B00004F114094FF02003EFF3118A83F3118837
:1009C000BFF36F8F484603F08DF940B9334934487F
:1009D000812207F0F9FA8121304807F0C1FB48462F
:1009E00003F09CF94FF6FF71E38BA28B8B4202F070
:1009F00007064AD0022E1FD135464FF001080133B9
:100A0000E383484603F07CF940B924492448AC22EA
:100A100007F0DAFAAC21214807F0A2FB8AF311882B
:100A2000BFF36F8FB8F1000F17D00023324639465D
:100A3000204607F0F2FA10E0930701D0062E0FD1FE
:100A400000233B606368EBB9C4E900773546F6B92B
:100A5000524602212046FFF7BFFD2846BDE8F08739
:100A6000052E17D0012E0AD00E490D4840F2C912AA
:100A700007F0AAFA40F2C9110A4807F071FB6FF0BB
:100A8000040504E01F606760E0E76FF00A054FF0BF
:100A90000008B6E76FF08505F9E700BF508E00004B
:100AA000168E00002E8E00002DE9F04F8B469246E8
:100AB0001C46002591B002909AF8000008B928461B
:100AC0005EE325280AF1010707D05946029B9847A3
:100AD0000028C0F25583013510E2182200210AA82F
:100AE00007F0A8FC9AF80130252B78D00022944614
:100AF000164696461046394617F8013B2B2B00F058
:100B00009D8000F29480202B00F09B80232B00F02E
:100B10009A8028B19DF8300040F004008DF8300034
:100B2000BEF1000F05D09DF8300040F008008DF8B0
:100B300030002EB19DF8300040F010008DF83000EC
:100B4000BCF1000F05D09DF8300040F020008DF87A
:100B500030002AB19DF8302042F040028DF830205C
:100B60009DF8302002F04400442803D16FF3861230
:100B70008DF830209DF830202A2B42F080028DF82D
:100B800030207BD19DF831204B1C42F001028DF8C2
:100B900031201A782E2A0CBF012100219DF8312026
:100BA00061F341028DF8312074D15A782A2A6AD033
:100BB00000210A260133184610F8012BA2F1300754
:100BC000092F40F28E809DF830200E91C2F3400034
:100BD00040EAD17161F341028DF830205AE00AF108
:100BE00002078DF833309DF83130D90740F1498143
:100BF00054F8049BB9F1000F07DA9DF83020C9F1D1
:100C0000000942F004028DF830205A0740F1428179
:100C100054F8048BB8F1000F80F241819DF8313017
:100C20006FF341038DF831304FF0FF3837E12D2B52
:100C30000CD0302B7FF46DAF01225CE74FF0010E3A
:100C400059E7012657E74FF0010C54E7012052E71E
:100C500033460CFB0202303A1E4616F8010BA0F197
:100C60003007092FF4D9994293D09DF830100D9296
:100C7000D20F62F341018DF830108AE70B46002253
:100C80004FF00A0CE8E79DF83120023342F00402ED
:100C90008DF831201F4617F8012B6C2A41D025D83A
:100CA000682A2BD06A2A46D04C2A4CD01F4617F807
:100CB000012B9DF83130782A8DF8332000F2D9804D
:100CC000572A4DD8412A03D0453A022A00F2D18052
:100CD00004229DF8323062F302038DF83230012392
:100CE0009EE006FB01210346303964E7742A26D0D2
:100CF0007A2ADBD106229DF831300DE05A78682A35
:100D00009DF8312006D1012161F3C6028DF8312012
:100D10009F1CCCE71346022262F3C6038DF83130E4
:100D2000C5E75A786C2A9DF8312001D10421EBE700
:100D300013460322F0E705229DF83130ECE7072245
:100D40009DF83130E8E7BDF8303023F4F04323F06C
:100D5000020343F4804343F00203ADF83030A6E7CA
:100D6000A2F15801202900F2848001A050F821F05E
:100D7000350E0000730E0000730E0000730E0000AD
:100D8000730E0000730E0000730E0000730E00005F
:100D9000730E0000D10C0000730E0000350E000031
:100DA000F50D0000D10C0000D10C0000D10C0000AA
:100DB000730E0000F50D0000730E0000730E0000AE
:100DC000730E0000730E00003D0E0000350E000093
:100DD000590E0000730E0000730E0000590E000043
:100DE000730E0000350E0000730E0000730E00003D
:100DF000350E000001209DF8321003F0780360F3F7
:100E00000201402B8DF8321002BF9DF8301041F0E6
:100E100001018DF83010632A31D1003B18BF012346
:100E20009DF83020C2F340010B4363F341028DF87B
:100E30003020D8E602209DF83210DEE703219DF82D
:100E4000322003F07803A3F1400061F30202434231
:100E50008DF832204341E3E703219DF8322013F05F
:100E6000780F61F3020214BF012300238DF83220B2
:100E7000D6E79DF8303043F001038DF83030002381
:100E8000CEE79DF93020002AACBF4FF0FF39DDF8E6
:100E90003490BAE69B077FF5C7AEDDF838800023B3
:100EA000CDE90D339DF832309DF8312003F0070372
:100EB000012BC2F3C30236D1D31E042B20D8DFE8A6
:100EC00003F00307071F1F0054F8040BC11704E0C9
:100ED000073424F00704F4E80201CDE90A019DF883
:100EE000303013F0030654D03B4652465946029820
:100EF00007F020F90028C0F243810544BA46DBE53B
:100F000054F8040B012A4FEAE071CDE90A0105D13A
:100F10009DF828300A9300230B93E0E7022ADED1E4
:100F2000BDF92800D2E7022B23D1D31E042B13D8FE
:100F3000DFE803F0030A0A12120000212068231DD3
:100F40000A900B911C46CAE7073424F00703F3E824
:100F50000201CDE90A01F5E754F8043B012A0A939E
:100F60004FF000030B93D3D0022AB8D1BDF828303C
:100F7000D0E7042B07D1073424F00704F4E802017A
:100F8000CDE90A01ABE7032B04BF54F8043B0A93F5
:100F9000A5E79DF833007828B0D8622822D8252804
:100FA0003FF493AD5828A9D1DDE90A010DF12603DC
:100FB00000930CAA04AB07F072F88246B8F1000F58
:100FC0000DF126000CDB9DF83020A0EB0A036FF337
:100FD000861298458DF8302002D9A8EB03030D93B3
:100FE00080463DE06338152888D801A151F820F0EB
:100FF00071100000D5100000FD0E0000FD0E000075
:10100000FD0E0000FD0E0000D5100000FD0E0000DA
:10101000FD0E0000FD0E0000FD0E0000331100006B
:101020000111000005110000FD0E0000FD0E000082
:1010300049100000FD0E000001110000FD0E00002F
:10104000FD0E000001110000B8F1000FDDF828A02E
:101050000ADB4146504607F086F900260AEB0008F5
:10106000BAF1000F0CD149E7504607F075F9F4E7E3
:1010700000260A9B0DF111088DF810300DF1100AB1
:10108000A8EB0A0306B101339DF83220D0066BD5D8
:10109000023352060D9948BF0E9A0B4448BF9B1865
:1010A000B9F1000F79DD9DF83020A9EB0309C2F3F7
:1010B00080030393530770D4500664D546B1594654
:1010C0003046029B984700285ADB039B01351E4699
:1010D000302359E01E0711D413F0100618BF202644
:1010E000DDE90A23002A73F10001BFF65DAF524229
:1010F00063EB43032D26CDE90A2355E72B26EFE7C3
:10110000002651E70A9848B30DF126030093002109
:1011100004AB0CAA06F0C3FFBDF83230824603F0E0
:10112000EF0343F4F04343F010030026ADF83230F0
:1011300044E70A9B072A3FF6E1AEDFE802F00D0420
:10114000060D08080D0D1D70D8E61D80D6E6284650
:10115000E917C3E90001D1E61D60CFE6DFF8C480DE
:101160000646A8F1050A8BE7110748BF013390E74F
:10117000184603935946029B98470028039B04DABC
:1011800011B0BDE8F08F20234D444A46002AA5EB5C
:10119000090109F1FF39EBDC0D4636B159463046FD
:1011A000029B98470028EBDB01359DF83230D906C9
:1011B00001D41A0706D559463020029B98470028CB
:1011C000DEDB01359DF83230DB0607D559469DF848
:1011D0003300029B98470028D2DB01350D9E2E4438
:1011E000731B002B16DC434652465946029806F004
:1011F000A1FF0028C4DB0544A944A9EB0503002B8B
:101200007FF77CAE59462020029B98470028B7DB29
:101210000135F2E759463020029B98470028AFDBA2
:101220000135DDE77B8E00004FF02002EFF31183E4
:1012300082F31188BFF36F8F0121044AC2F8401571
:1012400083F31188BFF36F8F002070470090035025
:1012500020B1034B800143F001031847704700BFE2
:10126000808A000084B004AB03E907009DF80430D5
:10127000062B07D10122044BC3F80025BFF34F8F83
:1012800020BFFDE704B0704700400050F8B50546A8
:101290004FF02003EFF3118683F31188BFF36F8FB4
:1012A000194802F01FFD40B918491948812206F07B
:1012B0008BFE8121154806F053FF134802F02EFDE6
:1012C000144B1C68002C38BF00245CB1124FD4E9C9
:1012D0000132002D08BF13460BB1387898472468B7
:1012E000002CF4D1084802F00BFD40B9074908482A
:1012F000AC2206F069FEAC21044806F031FF86F30B
:101300001188BFF36F8FF8BDA0020020508E00003F
:10131000168E0000A4020020AC020020084B10B57D
:101320001C685CB901221A60064B93E8070006F0BE
:1013300021FF2046BDE81040FFF7A8BF10BD00BF49
:1013400004000020AC020020F0B585B06E461D4CB4
:1013500001460546304606F025FF96E8070084E87A
:101360000700207860B30020174B18606B1C19D061
:10137000914208D215491648BD2206F025FEBD212E
:10138000124806F0EDFE4FF400460021A768114810
:101390000023E6FB0701104AFEF750FF0121281A3F
:1013A00003F0E0FF02F086FF0120FFF76FFF94E8F3
:1013B0000700FFF757FFFFF7B1FF03F063F920784D
:1013C00005B0F0BDAC02002004000020808E0000BB
:1013D000168E00003F420F0040420F0010B5074834
:1013E00002F07EF9064C074B1860204601F024FD00
:1013F0002046FFF7DDF8002010BD00BFAB8E0000D7
:1014000009140000B80200200A2838B50446074D28
:1014100004D1286883680D215B6898472868836831
:10142000E1B25B689847204638BD00BFB802002093
:101430002DE9F0410E4C0746051BC5F347130C255B
:101440005D4305F148000E462044402106F0AFFE02
:10145000011E08DB074B2C44C4E91036064B5B59D0
:10146000BDE8F041184738463346BDE8F04118471B
:10147000D0020020118200009C8A000038B5CCB256
:10148000012C054608D9084908487E2206F09CFD33
:101490007E21054806F064FE0C212B6904FB013413
:1014A000A06C00F0070038BDB28E0000168E000060
:1014B000F8B5CCB2012C0546164607690AD9184979
:1014C000184840F2531206F07FFD40F253111448C1
:1014D00006F046FE4FF02003EFF3118283F31188EC
:1014E000BFF36F8F0C2303FB0471896C11F0C001F3
:1014F00001D08E4211D10121002003FB04739964B5
:1015000082F31188BFF36F8F30B90C23696803FB36
:101510000414636898470020F8BD4FF0FF30EFE7F0
:10152000B28E0000168E000070B50D4606490446C6
:10153000411A491140220548FFF7BAFF2B460146E0
:101540002046BDE870401847D0020020D00000209F
:1015500070B5002201210446052000F02DFE052073
:1015600000F00CFE0F4801F073FF0F4B984215D1AD
:1015700001F08EFF26690D49304606F073FD002804
:101580000BDB0125B5642469084904F1200006F04D
:1015900069FD002801DB0020656570BD6FF0040067
:1015A000FBE700BFE51500000000AD0BB48A0000AA
:1015B00001460C2300224B43084870B5C418483339
:1015C000D4E910561844226406F00FFE2DB13246BD
:1015D0002B46BDE870400248184770BDD00200207D
:1015E000D0000020012808B506D0032808D0A0B9F3
:1015F0000F4B9B6C5B0719D1BDE80840FFF7D8BFC4
:101600000C4940F266220C4806F0DEFC40F26621EE
:10161000BDE80840074806F0A3BD064940F26A222B
:10162000054806F0D1FC40F26A21F1E708BD00BF91
:10163000D0020020B28E0000168E000008B54FF0D8
:101640002003EFF3118183F31188BFF36F8F124AE8
:10165000136843F0020013F0010310600CD04FF048
:101660005022D2F80C34D2F80C2413F0010303D02A
:101670000A4806F0BAFD012381F31188BFF36F8F8A
:1016800023B1BDE808400020FFF792BF0120BDE86C
:10169000084001F01BBF00BF2803002018030020F2
:1016A000074BD3E8EF2F22F00201C3E8E01F002828
:1016B000F7D1D30702D4012001F058BF704700BF13
:1016C000280300201FB500220123CDE902236B4629
:1016D000084ACDF800D0CDF804D006F0ABFD0028C4
:1016E00005DB4FF480420023684602F0D9FC05B0C8
:1016F0005DF804FB2F8200002DE9F8430122054626
:101700004649D1E8EF3FC1E8E02F0028F9D19BB965
:10171000434944484B60CB608A60FFF741F9002899
:101720000ADA4149414840F2262206F04DFC40F2D7
:1017300026213D4806F014FDADB36B1E012B59D890
:10174000012D07D14FF05023D3F81C3403F00303CD
:10175000022B28D006F0C4FF044618B9344B1B787E
:10176000002B54D14FF02003EFF3118683F311883F
:10177000BFF36F8F01242F4FDFF8BC80DFF8BC90E0
:101780004FF05022D2F81834D2F81824D2030CD5D6
:1017900003F00303022B01D0012D06D124B386F3FD
:1017A0001188BFF36F8FBDE8F883C4B1304600F0F5
:1017B0006DFD4FF05022D2F81835DBB2012BDFD18E
:1017C00039680029DCD00021396039680221C2F86B
:1017D00018152022C8F88021C9F80030D0E7002170
:1017E000212003F05FFBE4E74FF050230222C3F80F
:1017F0000423D8E70C490D484FF40E7206F0E4FBC1
:10180000BDE8F8434FF40E71074806F0A9BC4FF04D
:10181000502302220646C3F80823ACE72C0300201D
:10182000C0020020F0020020B28E0000168E0000E0
:10183000111700200451005000E100E00850005052
:1018400010B5064C06482146172206F0BDFB20467F
:10185000BDE81040172106F083BC00BF098F0000CF
:10186000168E0000044A1368C81A20F07F40034413
:10187000136003F0B5BD00BF400300202DE9F04721
:101880004FF480374FF00009860000F1500406F154
:101890005026A40006F58036A4B204F15024D6F8F0
:1018A0004035DFF86C8021F07F4504F580348740B7
:1018B000D8F804A5A3EB0A0323F07F432AF07F4264
:1018C000012BC6F8402502D1132006F043FF0AF190
:1018D0000202AB1A23F07F43B3F5000F88BF154611
:1018E000C4F80090236825F07F43C8F84473C6F815
:1018F0004035D8F804359A4506D0EB1A023B23F060
:101900007F43B3F5000F01D8BDE8F0872B46CFE742
:1019100000500150F8B5002427460F4E0F4B104AD7
:1019200018461D6804B1F8BDD2F80413C903FAD5EE
:1019300031680029F7D0346031684FF48031C2F843
:1019400048130124D2F8401525B100205A681F60C1
:10195000A847E3E70560E6E7405101503403002063
:101960000050015038B500244FF480334FF400127A
:101970000D4D0121C5F80845C5F804330B4B152062
:10198000C3F88021224600F017FC152000F0F6FB7A
:101990000123074A02201360064A2B601360FFF7F9
:1019A000ABFE204638BD00BF0050015000E100E012
:1019B000085001503C030020134BB0F1FF3F08BF1B
:1019C0001846013800281CDD9842A8BF18460F4B66
:1019D000D3F804250E4B1968521A12F4000F18BFE1
:1019E000002022F07F4301330A4A03440A48106072
:1019F00000205060044A934294BFC9188918FFF729
:101A00003DBF0020E3E700BFFFFF7F000050015013
:101A1000400300203403002065180000044BD3F875
:101A20000405044B1B68C01A20F07F40704700BFBC
:101A3000005001504003002000280DDB0122430923
:101A400000F01F0002FA00F0044A203342F823009D
:101A5000BFF34F8FBFF36F8F704700BF00E100E00F
:101A6000F7B500281C4614BF4FF400534FF4004351
:101A70008A420BD294222749274806F0A5FA9421DE
:101A8000244803B0BDE8F04006F06ABB40D00D46E4
:101A9000224E002839D005F5E0770135AA4246F8F4
:101AA0002740F6D802FB03F0013A4B4300901C4854
:101AB00006F08AFA1B4B14F0100F1B491B4808BF95
:101AC000194606F081FA14F0040F14BF72212D217B
:101AD000174806F079FA14F0020F14BF77212D2170
:101AE000134806F071FA14F0010F0CBF2D21782174
:101AF0000F4806F069FA6C210D4806F065FA0D48AA
:101B000003B0BDE8F04006F05FBA05F5C077C4E762
:101B100003B0F0BD5A8F0000168E00000030005058
:101B20007B8F00004E8F0000458F00002C9100003D
:101B3000958F0000089B000030B54FF4803485B0CD
:101B40004FF480312548264D06F03EFA216825489D
:101B500006F03AFA2968244806F036FA10220021E5
:101B6000684606F067FC236868460093029400F01C
:101B700003FF012000F030FF002000F019FF0020DB
:101B800000F03EFF0121002000F058FF00F04CFF64
:101B900016482C6806F018FA0820FFF74DFF144A83
:101BA00024F00104D2F82038002B07DA03F00303F5
:101BB000023B012B9CBF0F4BC2F8203801210820AB
:101BC00006F07EFBBFF34F8FBFF36F8F6408640096
:101BD0002046214622462346FEF7AEFC988F0000A1
:101BE00004000100AF8F0000C48F0000E28F0000EE
:101BF00000300050000100802DE9F8435E4806F0F7
:101C0000E3F9002140F2171308460222FFF728FFEC
:101C10005A4D40F20713202202210020FFF720FF37
:101C2000574806F0D1F9C5F30E04564BC4F50044ED
:101C30009C4208D254495548822206F0C5F98221B7
:101C4000514806F08DFA524EC4F34314D6F80025DD
:101C5000C5F3C435D2050AD54E494C484FF4BD7280
:101C600006F0B2F94FF4BD714A4806F079FAD6F899
:101C70000435DB050AD54749444840F27B1206F09B
:101C8000A3F940F27B11434806F06AFA404B424800
:101C9000C3F80055C3F80445D3F80015D3F804255C
:101CA000520106F091F9364806F08EF900F0AEF8D0
:101CB000014610B1394806F087F90024384806F08B
:101CC00083F940F21713082200210120FFF7C8FE14
:101CD0002F4D40F20713202208210120FFF7C0FEFC
:101CE000274806F071F9C5F880442E4806F06CF9D3
:101CF0002D4EC5F8C0442D4F2D4DDFF8C48095F80A
:101D000005902146B9F1000F14BF33463B464046CB
:101D10002A6806F059F9B9F1000F0CD125480134B1
:101D200006F052F91C2C05F10805E8D11448BDE86D
:101D3000F84306F049B995F8049095F90400FFF7C7
:101D40007BFE4FEA890303F1A04303F54053B9F149
:101D5000310FD3F8002806D0002A07DA02F0030278
:101D6000023A012A02D8144AC3F800280121484641
:101D700006F0A6FA1148D2E718900000E0FF000034
:101D8000089B0000200000005A8F0000168E000003
:101D9000003000503C9000006E900000B4900000B5
:101DA000E4900000069100000D900000528F0000AA
:101DB000C08A00002F9100000001008036910000D1
:101DC000229100002DE9F0430746002685B0DFF898
:101DD0003490DFF8348001AD59F8044B98E80700DF
:101DE0003C4485E807000C222946204606F0D0FA3C
:101DF00000B91CB90136052EEED10024204605B0ED
:101E0000BDE8F083A08B0000308A00000022024869
:101E1000114603F03BBC00BF4403002070B50C46E4
:101E20001546064650B96FF01500BDE87040714682
:101E300072467346F4468EF3008C7447002AF2D043
:101E400006F085FA0128EED00C4B9C420BD92A19DA
:101E500003F61D239A4209D82A462146304606F049
:101E6000BEFA0020E1E7064B9C4203D9054B2A1934
:101E70009A42F1D94FF0FF30D7E700BF0302FF00CD
:101E80002F01FF003801FF0070B506460D461446CD
:101E900006F05DFA01280DD0204606F058FA012818
:101EA00008D023462A463146084803F023FC23681D
:101EB000AB4201D06FF01500BDE87040714672462C
:101EC0007346F4468EF3008C744700BF4403002031
:101ED00070B5054610460E46144606F038FA01283D
:101EE0000AD16FF01500BDE8704071467246734626
:101EF000F4468EF3008C74472846FFF763FF0546CF
:101F00003046FFF75FFF0346CDB1296A0E4A914282
:101F100015D148B10120196A0B4A914202D138B952
:101F20002070E0E70028DCD0012300202370DAE7EE
:101F30005B696A699A4234BF00230123F5E7002BED
:101F4000CFD00020E7E700BFFFFF0291014803F078
:101F500095BB00BFB48B000008B5B0B14368042B3B
:101F60000DD100220368D3E8EF1F012903D1C3E894
:101F7000E02F0028F7D1074808BF104608BD3BB145
:101F8000006801F0BBFF0020F8E76FF4E040F5E7E0
:101F90000148F3E7E98FFFFFEA8FFFFF10B5044622
:101FA00018B90D4B0D485B689847616808290DD03A
:101FB00031F004030AD011F0020108D0214608488C
:101FC00001F06AFD002323600023636010BD14222A
:101FD000206806F02FFAF7E7600000204792000023
:101FE0000005002010B5044618B9164B16485B686A
:101FF00098476368042B23D0082B21D0CBB92368E2
:10200000BBB94FF0FF324FF0FF3321460F4801F0CC
:10201000E9FC08B923681BB90A4B0D485B6898476F
:1020200014220021206806F005FA636843F00203D9
:102030006360206806F063FB636843F0010363603C
:1020400010BD00BF60000020479200000005002086
:102050006D92000008B5E8B14368042B0CD1012251
:102060000368D3E8EF1F002903D1C3E8E02F00285D
:10207000F7D10BD1002008BD53B100684FF0FF32FB
:102080004FF0FF3301F068FE0028F3D00348F2E779
:102090000348F0E76FF4E040EDE700BFE98FFFFF92
:1020A000EA8FFFFF08B5064940231422054806F0D1
:1020B000FBFABDE808400449044803F087BB00BFB1
:1020C0002005002000050020CC8B0000BC8B000008
:1020D000094A0A49936809685867996708494B682B
:1020E00043F080534B60002383F31188BFF36F8F5D
:1020F0009368986F704700BF040C0020548C000058
:1021000000ED00E013498A684FF030001044EFF30F
:10211000098C80E8F01F202080F31188BFF36F8FB7
:102120000D4F4FF000664A6A8A603E60506F002390
:10213000536780F3118802F1300090E8F01F8CF3B0
:10214000098802F1000004B506F0E9F8BDE8044092
:1021500070470000040C002004ED00E01EF0040FA6
:102160000CBFEFF30880EFF30980816911F8021CBE
:102170000229FFD001B506F0D6F801BD43B2002B0D
:1021800008DB012200F01F0002FA00F0024A5B099E
:1021900042F82300704700BF00E100E0054B420910
:1021A00053F82220012300F01F0003FA00F0104032
:1021B000704700BF00E100E038B54C1C072C054615
:1021C00008D90D490D48582205F0FEFE58210A484D
:1021D00005F0C6FF6BB2002BACBF03F16043084BA8
:1021E0004FEA4414E4B2ABBF03F5614305F00F05B9
:1021F00083F800435C5538BD9A920000168E0000AB
:1022000014ED00E042F8203C009B0B4942F81C3CD6
:10221000019B21F0010142F8183C029B42F8081C86
:1022200042F8143C4FF0807342F8043C0023203AFB
:1022300002654367704700BF8B800000084B9860C1
:10224000436E83F30B88104681F30988002163B63F
:1022500081F31188BFF36F8F0022002305F015FF73
:10226000040C0020014910220A60704710ED00E0C4
:1022700072B6404080F31188BFF36F8FBFF34F8F6A
:1022800030BF62B6BFF36F8F704700BF72B6494070
:1022900081F3118820BF80F3118862B6704700BFB8
:1022A00037B505460C46C9B18B6810480093D1E993
:1022B0000023452105F069FF636945210093D4E9B6
:1022C00003230B4805F061FF4521E269094805F049
:1022D0005CFF4521A269084805F057FF21462846C2
:1022E00003B0BDE8304001F033BA00BFD092000027
:1022F00004930000389300004C93000030BFFFF7B8
:10230000FDBF00BF0B4A08B50B4B22F07F029A605D
:10231000BFF34F8FBFF36F8FD3F8882022F4700282
:10232000C3F8882001F070FA02F086FE00F006FB88
:1023300001F08EFA0000000000ED00E001B572B679
:102340000B4A106A00281EBF0021116206F0D0F966
:1023500062B6EFF30580A0F110004FEAC000054916
:10236000014409C99847BDE80140034908470000F6
:10237000040C0020C0870000B5280000002080F376
:102380001488BFF36F8F002080F30A8880F30B88D6
:1023900005F0EEFE00200E490860BFF34F8F0D4898
:1023A00080F3088800F0A4FA202080F311880A48FE
:1023B0004FF40061401880F30988EFF31480022184
:1023C000084380F31488BFF36F8FFFF79BFF000073
:1023D00094ED00E01827002058280020EFF3088033
:1023E000EFF3098101B5724600F070F901BD00BF3D
:1023F00070B52B4C06460D462A48452105F0C5FE12
:10240000A26AD00603D54521274805F0BEFEA36A7F
:10241000190703D54521254805F0B7FE204CA36ACE
:102420009A0710D54521224805F0AFFE626BA36ADA
:102430001B0608D545211F4805F0A7FE1EB1A36A5B
:1024400023F08003A362164CA26AD60703D5452168
:10245000194805F09AFEA36A980603D54521174846
:1024600005F093FE0E4B9A6AD10602D49A6A92073F
:102470000DD59B6ADB060AD51149124840F24F126E
:1024800005F0A2FD40F24F110D4805F069FE002055
:10249000034A936A43F0FF039362287070BD00BF44
:1024A00000ED00E07F9300009A930000D2930000BB
:1024B000EA93000007940000229400004694000074
:1024C0007A940000168E000070B5234C06460D4627
:1024D0002248452105F059FEA26AD10403D54521C1
:1024E0001F4805F052FEA36A1A0503D545211D4871
:1024F00005F04BFE184CA36A9B0510D51A484521E0
:1025000005F043FEA26BA36A180408D545211748BD
:1025100005F03BFE1EB1A36A23F40043A3620E4CF8
:10252000A36A590503D54521114805F02EFEA36A7B
:10253000DA050BD545210F4805F027FE0020064A95
:10254000936A43F47F439362287070BDA36A9B042F
:10255000F4D545210848EFE700ED00E0B494000011
:10256000CF940000D2930000E59400000395000092
:102570001D9500003D9500004694000038B5214CA3
:102580004521214805F001FEA26A950103D54521A8
:102590001E4805F0FAFDA36ADC0103D545211C485D
:1025A00005F0F3FD174DAC6A14F4801404D04521F6
:1025B000184805F0EAFD0224AB6A180303D545214B
:1025C000154805F0E2FD0F4DAA6A510303D54521D8
:1025D000124805F0DAFDAB6A9A0303D5452110488D
:1025E00005F0D3FD074DAB6ADB0303D545210D484C
:1025F00005F0CBFDAB6A20466FEA03436FEA134355
:10260000AB6238BD00ED00E05A9500007795000000
:102610008F950000AE950000DD950000009600004B
:102620002A9600004996000010B51E4C1E48452110
:1026300005F0ABFDA2696369580603D545211B4827
:1026400005F0A3FD6369D90708D54521184805F0B1
:102650009CFD636943F0FF03636110BD63699A07E2
:1026600002D545211348F2E763695B0702D545218E
:102670001148ECE76369180702D545210F48E6E7E2
:102680006369D90602D545210D48E0E763699A06DA
:1026900002D545210B48DAE763691B06D9D54521E8
:1026A0000948D4E7D0ED00E0799600009796000045
:1026B000AC960000C7960000EA9600000A9700005A
:1026C0002C97000046970000659700002DE9F04127
:1026D000624B0D465C6800268AB0C4F3080786F397
:1026E0001188BFF36F8F02F07F43B3F17F4F1ED18C
:1026F00012F0010339D012F0400302F0080840F054
:10270000A680520754BF05461E462A68544B58BF40
:1027100001261344012B98BF2A6C4521514805F02E
:1027200034FDB8F1000F1DD0EFF389855DB940F29B
:10273000E1324D494D4805F047FC40F2E1314A484D
:1027400005F00EFD00250023FA1E98468DF807308F
:102750001346092B69D8DFE803F00A595D38616830
:1027600068686865EFF38885E0E71E46DFE7452186
:102770003F4805F00AFD394B8DF80780DC6A14F0FC
:10278000020404D045213B4805F0FFFC48E0DB6A29
:102790005B0022D54521384805F0F7FC374B1B7804
:1027A00033B101200DF10701FFF722FE044614E0CA
:1027B000334B1B782BB101200DF10701FFF784FE8D
:1027C000F4E7304B1B889BB213B1FFF7D7FEEDE760
:1027D0002D4B5B690BB1FFF727FF9DF8073093B9CD
:1027E0002022294602A805F0FAFD099B56B3C3F33F
:1027F000080222B96FEA53236FEA43230993204664
:1028000002A9FFF74DFD0AB0BDE8F08100200DF1EF
:102810000701C9E700200DF10701CFE7FFF704FF2B
:102820000024DAE745211948AEE7194914F4F87F86
:10283000184A194808BF0A46A7F11003452105F0B8
:10284000A4FCEDE723F4FF7323F00103D6E7B8F10E
:10285000000F7FF46BAF0546012667E700ED00E04F
:10286000A6ED0501AB9700007A940000168E0000DB
:10287000CF970000EB9700001198000028ED00E0D2
:1028800029ED00E02AED00E0D0ED00E035980000F1
:102890007D970000929700005E980000044B5A69F3
:1028A00042F010025A615A6942F480625A617047DC
:1028B00000ED00E0044B9968586A884203D0034950
:1028C0004FF080520A607047040C002004ED00E0D5
:1028D00000231846054A1168C1F307218B4200D135
:1028E0007047936010610133F8E700BF90ED00E09E
:1028F00010B572B6002484F31388FFF7E9FF0E4A7F
:10290000234611464FF0FF3403F120000133102B12
:1029100042F82040F8D100234FF0FF3003F160026D
:102920000133102B41F82200F8D162B6BFF34F8F6C
:10293000BFF36F8F10BD00BF00E100E00023202136
:102940000348C2180133412B82F80013F9D17047B4
:1029500000E100E0064B9B68834207D1EFF305835B
:1029600023B1044A536843F08053536002F0D0BA55
:10297000040C002000ED00E082680C4B9A600368B4
:1029800083F38888436883F38988027B02F001011E
:10299000EFF3948323F00303920748BF43F002034D
:1029A00009B143F0010383F39488704700ED02E01E
:1029B000084AD36848B123F400531B041B0C43F0AE
:1029C000BF6343F40033D36070479BB243F40053BA
:1029D000F5E700BF00ED00E0084AD36840B19BB2C4
:1029E00043F4804343F0BF6343F40033D360704744
:1029F00023F480431B041B0CF4E700BF00ED00E050
:102A0000084AD36840B19BB243F0080343F0BF6368
:102A100043F40033D360704723F008031B041B0CFE
:102A2000F4E700BF00ED00E0034AD2F88C3043F435
:102A30004063C2F88C30704700ED00E0084B1A6824
:102A400018B142F001021A60704722F001021A60C8
:102A50001A6811B142F00202F5E722F00202F2E731
:102A6000D0ED00E01FB5094C094A23460121094871
:102A700000F01AF900230393074B0121E41A01A87F
:102A80000193029400F02CF904B010BD0000012065
:102A900000000020E08B00009801002010B50B68BA
:102AA0000C7A23F01F0204F01F031A43CB68640959
:102AB00023F01F03044943EA440343F00103886001
:102AC000CA600B6110BD00BF90ED00E030B54B68EF
:102AD0000C6885B00A898D7A0094013B24F01F04AC
:102AE000234402F01F0242EA451223F01F030F287D
:102AF00004468DF80820039309D90246452106486B
:102B000005F043FB6FF01504204605B030BD694663
:102B1000FFF7C4FFF8E700BF7A9800002DE9F04FF7
:102B20008946144606464FF00008524D85B0C84508
:102B300023DA7768002F42D01F2F17D9FB0615D153
:102B4000D6F800A01AF01F0F10D1504605F0F6FB82
:102B5000834607EB0A00013805F0F0FB834510D0EF
:102B60006FF0150B5A464521434802E04246452185
:102B7000424805F00AFB6FF01504204605B0BDE899
:102B8000F08F1BF1160FEDD0631E5B45EADBC5F835
:102B900008B0E968C5F808B02F6921F01F01D6E92F
:102BA00000321A44994247F01F0702F1FF3A1CD144
:102BB000574508D131465FFA8BF0FFF787FF08F1E0
:102BC00001080C36B3E73146C5F808B0EB6822F0CF
:102BD0001F0203F01F031A43EA60E0B2FFF776FF1B
:102BE00010F1160FC7D0441CE9E7013B5745E0B28E
:102BF00023F01F03C5F808B006D12A69314602F058
:102C00001F0213432B61E9E7296901F01F010B4300
:102C10002B613146FFF75AFF10F1160FABD0C5F804
:102C200008B0EA689DF80830013F62F304038DF8AC
:102C300008302B699DF808205B0863F347128DF874
:102C40000820D6E900321344009323F01F033B44CD
:102C5000441CA3EB0A0AE0B22AF01F030F280393D7
:102C600003D902464521064883E76946FFF716FF68
:102C7000B9E700BF90ED00E0CD980000A5980000F6
:102C80007A9800000522034B5A60BFF34F8FBFF3C1
:102C90006F8F704790ED00E0BFF35F8F0022014B14
:102CA0005A60704790ED00E010B50A4C2278FFF7AB
:102CB00035FF207016300CD10749084840F2051244
:102CC00005F082F9BDE8104040F20511024805F018
:102CD00047BA10BD10170020F5980000168E0000AE
:102CE0002DE9F74F2D4D8A4606464FF00008AB46BA
:102CF0002B4FD04502DB03B0BDE8F08FD6F804902F
:102D0000B9F1000F44D031680846019105F016FB77
:102D10000199044609EB0100013805F00FFB8442DC
:102D20004FF014021F4B13D06FF0150302FB08F88D
:102D30004BF8083040F215121B491C4805F044F9C5
:102D400040F21511184803B0BDE8F04F05F008BA7D
:102D500014F1160F2C60EDD01978A142EADD02FBC8
:102D600008B0BC60BC60FC6800F10801007B64F343
:102D70000400087138690C79400860F347140C713D
:102D8000F96821F01F016960396921F01F0129618B
:102D900008F1010814350C36ABE700BF200A00200B
:102DA00090ED00E010170020F5980000168E00004E
:102DB00070B51B4D2E68102E0DD94FF49E72194917
:102DC000194805F001F917484FF49E7105F0C8F94C
:102DD0004FF0FF3070BDFFF75FFF0020134C144A27
:102DE0002263864215D1134B1E70FFF74BFF2368F9
:102DF000C3F30723102B0AD00A490B484FF4CF72B4
:102E000005F0E2F84FF4CF71064805F0A9F900206B
:102E1000E0E7696801EB0011FFF740FE0130E0E7F1
:102E2000EC8B0000F5980000168E000090ED00E09D
:102E3000AAFF440010170020014B1860704700BF24
:102E400028000020F0B54B79012B2AD0032B25D187
:102E500010268B79032B21D1CC792CB1012C1DD1DB
:102E600043685B689B0719D00A7912B1022A15D111
:102E70000E220B684568B3F5164F2D6865D02DD826
:102E8000B3F5165F64D016D8B3F5966F62D00AD842
:102E9000B3F5967F61D0B3F5167F61D06FF08500F2
:102EA00052E00026D5E7B3F5166F5CD0B3F5965F18
:102EB000F4D1374B3CE0B3F5E14F57D007D8B3F529
:102EC000615F55D0B3F5964FE8D1324B30E047F60D
:102ED0001227BB42E2D14FF4000329E0B3F5613F72
:102EE00048D013D8B3F5963F47D009D84DF6C02740
:102EF000BB4244D0B3F5614FD0D14FF46B0317E020
:102F0000B3F5E13FCAD14FF0EB7311E0B3F5612F98
:102F100038D008D8204FBB4237D0B3F5E12FBDD110
:102F20004FF0E86304E01D4FBB42B7D14FF0805330
:102F3000C5F82435036934432243043303C9C5F873
:102F40006C2583E803000020F0BD4FF41D03EFE77C
:102F5000134BEDE74FF49E23EAE74FF4A033E7E786
:102F60004FF41C33E4E74FF41D23E1E70D4BDFE79B
:102F70000D4BDDE74FF06C73DAE70C4BD8E74FF4FD
:102F80006503D5E74FF07063D2E74FF08063CFE77A
:102F900000B0130000A04E0090D0030040420F008C
:102FA0000050270000C0750000F03A0000903A0180
:102FB000036810B55A090CBF4FF0FF32002203F02E
:102FC0001F0322FA03F3DB0704460AD40E490F4815
:102FD0004FF4057204F0F8FF4FF405710A4805F04C
:102FE000BFF8236803F01F025B0922600AD006497C
:102FF000064840F2192204F0E7FF40F21921024886
:1030000005F0AEF8024810BD3B990000168E000096
:1030100000258450F8B505460F46066905F060FBAB
:1030200010B92C4B1B7883B94FF02003EFF31184B8
:1030300083F31188BFF36F8F284605F06AFA28BB27
:1030400084F31188BFF36F8FEEE76424284605F000
:1030500060FA70B9012005F012FB013CF6D10021A5
:10306000212001F01FFFF0E784F31188BFF36F8F79
:10307000F5E74FF02003EFF3118483F31188BFF3DA
:103080006F8F284605F045FA0028EDD0012206F89A
:10309000107F69680B68C3F84465C3F848250022AF
:1030A000C3F82021D3F82001C3F85821D3F85821C0
:1030B0004A68D20641BF0822C3F800254FF48002B7
:1030C000C3F8042301229A6084F31188BFF36F8F41
:1030D000F8BD00BF1117002030B585B06C4605461D
:1030E000084B0FCB84E80F00002201210820FFF7D6
:1030F00063F80820FFF742F82146284605F02CFA2D
:1031000005B030BD3C8A000030B585B06C46054640
:10311000084B0FCB84E80F00002201210920FFF7A4
:103120004BF80920FFF72AF82146284605F014FA43
:1031300005B030BD4C8A00002DE9F3410F4616461C
:1031400040B91A491A48262204F03EFF26211748A2
:1031500005F006F847B915491548272204F034FF51
:103160002721124804F0FCFF4FF4806500246FF023
:103170001500DFF84080A64202D802B0BDE8F08119
:10318000331BB3F5806F38BF1D46404601AB2A465E
:10319000391902F0AFFA019BAB4203D10028ECD100
:1031A0002C44E8E76FF01500E7E700BF85990000C1
:1031B000168E0000400A0020002208B5114604487F
:1031C00002F064FA002818BF6FF0150008BD00BFB8
:1031D000400A00202DE9F0430025214C214E54F8EF
:1031E000048CDFF8889085B0A84503D8002005B08E
:1031F000BDE8F083636A96E807001F6801AB83E8C7
:1032000007000C221946384605F0C2F890B98FB174
:10321000636A21691B681A6991420BD19A69A16995
:10322000914207D8E169914204D962695B6932EA47
:1032300003030AD0276A67B10B4804F0C5FE40407B
:1032400080F311884FF0040002DFE36801351C446D
:10325000CAE7484604F0B8FE636A1F60F5E700BF9E
:103260003C0200005C8A0000C0990000E99900005F
:10327000054B1868043B1B68092B03D1431E5842B9
:1032800058417047002070473401FF004A4A08B592
:10329000136843F002031360484B1B68092B01BFFE
:1032A0004FF050230022C3F81421C3F81821FFF770
:1032B000DFFF30B10123424A1360A2F63822C2F880
:1032C00078353E4B1B68092B07D13E4B1B68012B01
:1032D0001EBF01223C4BC3F87825FFF7C9FF10B190
:1032E0000E223A4B1A60354B1B68092B04D1002281
:1032F000374B1A6001225A600022D30003F57F0386
:10330000D3F80013013108D0D3F800130132D3F8F9
:103310000433B2F5807F0B60EFD12E4BDA69D10711
:103320003BD52D4B1946D3F80024012AFBD1C3F815
:103330000425D1F80034012BFBD1264BDA69D207E2
:1033400008D5DA69244922F00102DA61D1F80024B3
:10335000012AFBD11A6A01320AD11A6A22F0FF024D
:1033600042F020021A621C4AD2F80034012BFBD131
:103370000022194BC3F80425D3F80024012AFBD1FD
:10338000BFF34F8F1549164BCA6802F4E06213432E
:10339000CB60BFF34F8F00BFFDE71B6A0133C0D086
:1033A0000E4AD2F88C3043F44063C2F88C300D4B97
:1033B0000D4A1A6008BD00BFD0ED00E03001FF00EB
:1033C000384A00503401FF0000400050E4AE035082
:1033D0000C4700500080FF000090035000ED00E01B
:1033E0000400FA05540000200090D00308B570B125
:1033F00001281BD04FF44F721349144804F0E4FD28
:1034000011484FF44F7104F0ABFE00200DE031B1D4
:103410004FF05023D3F8183403F003030B704FF030
:103420005023D3F81804C0F3004008BD31B14FF069
:103430005023D3F80C3403F001030B704FF05023EA
:10344000D3F80C04EFE700BF1C9A0000168E0000B2
:1034500010B5044640B909490948B52204F0B4FD45
:10346000B521064804F07CFE064B1A7922B90122E8
:1034700005481C601A7110BD0448FCE7509A000012
:10348000168E0000FC0B00200000AD0B0C00AD0BF5
:1034900008B50B4B1B7943B90A490B48CE2204F0FF
:1034A00093FDCE21074804F05BFE0520FEF776FE73
:1034B00020B9BDE808400520FEF760BE08BD00BF8A
:1034C000FC0B0020509A0000168E0000224B13B512
:1034D0001B79044653B9214921484FF4857204F001
:1034E00073FD4FF485711D4804F03AFE6CB1012C58
:1034F00028D04FF49E721949194804F065FD4FF425
:103500009E71164804F02CFE18E020460DF10701CC
:10351000FFF76CFF4FF0502390B19DF80720022A6F
:103520000ED1C3F8182500220E4B1A601B68022228
:103530004FF05023C3F8042301229A6002B010BD5B
:103540000122EEE70022084B1A601B684FF050235F
:10355000C3F804431C60F1E7FC0B0020509A000004
:10356000168E000004510050005100502D4B13B531
:103570001B79044653B92C492C4840F2431204F0FD
:1035800023FD40F24311284804F0EAFD74B1012CF8
:1035900027D02549254840F25F1204F015FD40F27E
:1035A0005F11214804F0DCFD02B010BD4FF0502344
:1035B0000222C3F808230122C3F8044142F2107426
:1035C00003F582731B681A4B1A6000210846FFF747
:1035D0000DFF0028E8D0012005F051F8013CF4D19E
:1035E000E2E74FF050230022C3F80843C3F800215C
:1035F00003F580731B680F4B1C608DF8074042F287
:10360000107401200DF10701FFF7F0FE0028CBD068
:103610009DF807000128C7D105F031F8013CF0D131
:10362000C2E700BFFC0B0020509A0000168E00007D
:103630000C50005004500050164B07B51A6852B198
:10364000002018601B6801224FF05023C3F80823A4
:10365000114B1B689847114B1A688AB100200DF175
:10366000070118601B68FFF7C1FE9DF807104FF0B7
:10367000502301294FF0020205D1C3F818259960A3
:1036800003B05DF804FBC3F80823034B01201B685B
:103690009847F5E700510050FC0B00200451005002
:1036A0000E4B70B553F82040013053F82060A6420D
:1036B00000D870BDD4E900352846984765B1EB685D
:1036C00030B10028B8BF4042FF28A8BFFF201870C3
:1036D0005A7842F001025A700834E8E7408C000042
:1036E00070B5054610B90024204670BD0378002B44
:1036F000F9D00F4A0F4C1646944208D10D4CB442F3
:10370000F1D0204604F0BEFF50B91834F7E7204648
:1037100004F0B8FF10B12368AB42E5D01834EBE7F2
:103720002846216804F028FE0028EED1DCE700BF1F
:1037300048010020D000002010B504464521034870
:1037400004F023FD204604F0A6FF00BF8D9A000080
:10375000F7B504460E464FF02003EFF3118783F3CD
:103760001188BFF36F8F01F0CDFB0022042C98BFAE
:103770001D4B054694BF53F824301C4B0092452145
:1037800022461B4804F001FD3EB1F369C3F3080370
:103790001BB14521174804F0F8FC35B1284604F068
:1037A000A5FF034608B1027802B9134B2A4645210A
:1037B000124804F0EAFC31462046FFF7BDFF042C16
:1037C00008D10F490F488F2204F0FEFB8F210C48CF
:1037D00004F0C6FC87F31188BFF36F8F284603B04F
:1037E000BDE8F040FFF7B6B8588C0000A19A000081
:1037F000B79A0000E49A0000AF9A00000A9B00000C
:10380000279B0000168E00000248034A0021121A6E
:1038100004F010BE9801002014170020012208B502
:10382000094B02201A70FFF73BFF01F0CBFE03208B
:10383000FFF736FF00F0D6F904F0ACFB034A137B28
:1038400023F00103137308BD111700201802002094
:103850002DE980483F4BA7B003F5006787F3088840
:1038600083F30A880024E0233B4D4FF0010B85F8D9
:103870002230EC772C766C76AC76EC766B6A374E31
:1038800043F4E0236B626B6ADFF8E8A043F40023A3
:103890006B62AC63EB68DFF8E0809BB243F0BF6320
:1038A00043F40833EB60FEF7F9FFFEF7DBFC4FF063
:1038B000FF33AB62EB62FFF77BFAFFF7D3F840F21E
:1038C0000113274DADF8243006ABAB60CDE91F44A2
:1038D00004F0D7FE2046FFF7E3FE0120FFF7E0FEED
:1038E00001F0C0F91F4B6E624FF480521E490593E0
:1038F00030465346CDE9034BCDE90144009400F036
:103900001DF9737B814623F004033046737301F085
:1039100021F80F234FF4A072CDE902431349144B51
:103920004046CDE904B4CDE9005400F007F998F819
:103930000D30524623F0040388F80D3005F11803CA
:1039400049463046C5E90633C5F80C802C756F60D2
:10395000FEF774FC5828002000ED00E0180200205B
:10396000040C0020939B000018170020182700204B
:103970002D3D00001D380000980100202DE9F04188
:10398000144D154CA846154EAC4208D93146144882
:103990003C2204F019FB3C21304604F0E1FB444595
:1039A00002D30020BDE8F081D4E9041242EA010309
:1039B00013F003030BD1E068A361834201D12034EB
:1039C000E2E7A76901331760A2610A44F5E76FF0E7
:1039D0001500E7E748010020480100209B9B0000FC
:1039E000168E00002DE9F74304460D469046994691
:1039F00000F108064FF02003EFF3118783F31188DD
:103A0000BFF36F8F304600F06DF940B91F49204871
:103A1000812204F0D9FA81211C4804F0A1FB304630
:103A200000F07CF9A369C3B12B601B68A361E36953
:103A30000133E3610024304600F062F940B91349D4
:103A40001348AC2204F0C0FAAC21104804F088FB03
:103A500087F31188BFF36F8F13E058EA090203D18F
:103A60006FF00B042B60E6E7224639463046CDE97D
:103A7000008900F089FD044618B9064B9B685B6914
:103A80002B60204603B0BDE8F08300BF508E0000DD
:103A9000168E0000040C00202DE9F04104460D466E
:103AA00000F108064FF02003EFF3118783F311882C
:103AB000BFF36F8F304600F015F940B91D491E481D
:103AC000812204F081FA81211A4804F049FB304632
:103AD00000F024F9D4F81880B8F1000F0FD1204677
:103AE00001F082F858B12A68C0F87880426100F08D
:103AF00031FF39463046BDE8F04100F0A5BB2B68E8
:103B0000A26930461A602B68A361E369013BE36157
:103B100000F0F6F840B907490748AC2204F054FA1F
:103B2000AC21044804F01CFB87F31188BFF36F8FAE
:103B3000BDE8F081508E0000168E00002DE9F043A4
:103B400085B0DDF83C900446B9F10F0F0F461546DD
:103B500098462ED11F4B98452FD104F15803C4E944
:103B60001633109B00262373042363730E9BE81DFA
:103B700002930D9B20F0070001930C9B3D18C4E9B4
:103B8000197000932A46434639462046C4E9066622
:103B9000A66084F80E90E673E666FEF733FB0E4BE4
:103BA00066659B6803B11B6F2846236705B0BDE8B7
:103BB000F08309F110031E2BCFD94FF4027207498D
:103BC000074804F001FA4FF40271044804F0C8FAFF
:103BD000C3E700BF2D3D0000040C0020C09B000087
:103BE000168E00002DE9F047394F3A4D3E46DFF87A
:103BF000EC8086B0BD420AD9414637484FF4367250
:103C000004F0E2F94FF43671404604F0A9FAB542E7
:103C100005F130041DD300F04DFB40F2E7384FF0C2
:103C200000092C4C2D4DDFF8B0A0B4420AD929462A
:103C3000504640F2F72204F0C7F940F2F721284637
:103C400004F08EFAB44221D306B0BDE8F04700F08C
:103C500019BD54F8043C059354F8103C049354F8EF
:103C6000143C039354F8183C029354F81C3C019301
:103C700054F8203C009354E90A2354E90C01FFF75F
:103C80005DFF54F8303C5D652546B3E7636A5A1C16
:103C90000FD04FF400424046494623EAE373C2FB8B
:103CA0000301494508BF4045276804D1384600F064
:103CB00087FE3034B9E74FF47A720023FCF7BEFA7E
:103CC00002460B4607F11800054901F01FFAF0E71C
:103CD0004801002048010020168E0000C09B000013
:103CE000454A0000006838B1044B00F003001B7D1A
:103CF000C01A18BF0120704701207047040C002033
:103D0000054903468A68087D1968024300209142EC
:103D100004BF186001207047040C0020024A117D86
:103D200093680B4303607047040C002008B5094CEE
:103D30004FF02002EFF3118382F31188BFF36F8FEE
:103D400001F0DAFA2062FDF7FFFA0028F0D1FEF761
:103D50008FFAEDE7040C00202DE9F34104461646E6
:103D60001F46EFF3058343B15F496048652204F0C5
:103D70002BF965215C4804F0F3F94FF02003EFF3D1
:103D8000118883F31188BFF36F8F5948FFF7AAFF9B
:103D900040B958495548812204F016F98121554807
:103DA00004F0DEF95248FFF7B9FFE368524AD3B195
:103DB000A0689168884233D056EA070332D14C4854
:103DC000FFF79EFF40B94B494848AC2204F0FCF88D
:103DD000AC21484804F0C4F988F31188BFF36F8F11
:103DE0006FF00F0019E0916891F90E100133E36054
:103DF00093683F482161A360FFF782FF40B93D49C6
:103E00003A48AC2204F0E0F8AC213A4804F0A8F9B2
:103E100088F31188BFF36F8F002002B0BDE8F081F6
:103E20002169E3E790F90E3091F90E109942A8BF8D
:103E3000194621EAE1718B423CDD00F04BFE05465C
:103E400022464146CDE90067294800F09DFB002845
:103E5000E3D04FF02003EFF3118683F31188BFF313
:103E60006F8F2348FFF73EFF40B922491F48812248
:103E700004F0AAF881211F4804F072F91C48FFF7EA
:103E80004DFF236821699C4207D033B193F90E306E
:103E90009942A8BF194621EAE171A06890F90E3055
:103EA000994209D16DB13146114800F0CDF96FF05A
:103EB0000A00B2E70025C3E700F00CFE0028F2D1AB
:103EC000F0E70B48FFF71CFF40B90A490748AC224E
:103ED00004F07AF8AC21074804F042F986F311881F
:103EE000BFF36F8FE3E700BFE39B0000168E000077
:103EF000340C0020508E0000040C002038B504461D
:103F0000EFF3058343B145494548C72204F05CF807
:103F1000C721424804F024F9A368002B78D0414D12
:103F2000AA68934277D1E36843B93C493C48DF2211
:103F300004F04AF8DF21394804F012F9EFF3058361
:103F400043B139493648FE2204F03EF8FE21364896
:103F500004F006F9AB68DB7B012B08D1324930480D
:103F6000FF2204F031F8FF212F4804F0F9F8AA6885
:103F7000D37B013BD373E368012B05D0013BE360A6
:103F800000F080FB002038BD4FF02003EFF31185D7
:103F900083F31188BFF36F8F2448FFF7A3FE40B966
:103FA00023491F48812204F00FF88121204804F0A2
:103FB000D7F81E48FFF7B2FEA068216990F90E30CD
:103FC000994201D000F086FD204600F00DFEA06071
:103FD00058B190F90E2022610022826700F0BAFCED
:103FE0002946124800F030F9CAE7E0600F48FFF7B1
:103FF00087FE40B90E490A48AC2203F0E5FFAC2128
:104000000B4804F0ADF885F31188BFF36F8FB7E765
:104010006FF01500B7E74FF0FF30B4E7E39B000007
:10402000168E0000040C0020059C0000340C0020BB
:10403000508E000038B504464FF02003EFF3118591
:1040400083F31188BFF36F8F1248FFF74BFE40B91F
:1040500011491248812203F0B7FF81210E4804F074
:104060007FF80C48FFF75AFE204600F0BDFD48B12E
:104070000022826700F06EFC2946BDE83840054802
:1040800000F0E2B8D4E902329A4218BF0133A360CB
:10409000F2E700BF380C0020508E0000168E0000A2
:1040A000F7B5044616461F46EFF305835BB156EAA3
:1040B000070308D02B492C48792203F085FF79218A
:1040C000284804F04DF84FF02003EFF3118583F3F7
:1040D0001188BFF36F8F2548FFF704FE40B92449CC
:1040E0002148812203F070FF8121214804F038F833
:1040F0001E48FFF713FEA368ABB1013B1B48A3604A
:10410000FFF7FEFD40B91A491748AC2203F05CFFE7
:10411000AC21174804F024F885F31188BFF36F8FA2
:10412000002003B0F0BD56EA070313D10F48FFF794
:10413000E7FD40B90E490C48AC2203F045FFAC2125
:104140000B4804F00DF885F31188BFF36F8F6FF003
:104150000F00E6E722462946CDE90067034800F054
:1041600013FADEE7309C0000168E0000380C0020A9
:10417000508E000010B5084C23685BB1FDF74EFC73
:1041800003462068054A03440021BDE8104013613E
:1041900001F0E8B810BD00BF480C0020040C00205E
:1041A000F8B504460D464FF02003EFF3118683F374
:1041B0001188BFF36F8F1E48FFF794FD40B91D496A
:1041C0001D48812203F000FF81211A4803F0C8FF37
:1041D0001748FFF7A3FD4FF40047002240F2E730F5
:1041E0000021164BE7FB04011A6100234FF47A7299
:1041F000FCF724F8002C124B16DC1860114B1D60E4
:10420000FFF7B8FF0A48FFF77BFD40B909490A48A4
:10421000AC2203F0D9FEAC21064803F0A1FF86F3DF
:104220001188BFF36F8FF8BD0228B8BF0220E4E702
:10423000400C0020508E0000168E0000040C002060
:10424000480C0020440C002010B503460C46C1B9B0
:10425000EFF30582AAB9144A516A9268914210D0CC
:10426000FFF74EFD40B911491148C32203F0ACFEDF
:10427000C3210E4803F074FFBDE810400020FDF795
:1042800027BF1846FFF73CFD40B908490848AC2253
:1042900003F09AFEAC21054803F062FF84F3118815
:1042A000BFF36F8F10BD00BF040C0020508E0000C4
:1042B000168E000038B54FF02003EFF3118583F31D
:1042C0001188BFF36F8F2048FFF70CFD40B91F49DD
:1042D0001F48812203F078FE81211C4803F040FF33
:1042E0001948FFF71BFDEFF3058343B1194918483F
:1042F000FE2203F069FEFE21164803F031FF164C42
:10430000A268D27B012A08D112491148FF2203F08A
:104310005BFEFF210F4803F023FFA268D37B013B24
:10432000D3730948FFF7ECFC40B908490848AC22B0
:1043300003F04AFEAC21054803F012FF85F3118813
:10434000BFF36F8F38BD00BF400C0020508E0000BF
:10435000168E0000059C0000040C00200B4B10B5CD
:1043600099420C460AD10A490A484FF4717203F087
:104370002BFE4FF47171064803F0F2FED4E90032CF
:1043800013605A600023C4E9003310BD9801002077
:10439000509C0000168E0000836810B5044653B987
:1043A0000A490B4840F24F2203F00EFE40F24F2123
:1043B000064803F0D5FE2146A068FFF7CFFF637BD8
:1043C00023F0020363730023A36010BD509C000020
:1043D000168E000038B50246124804F0ADF9124DB1
:1043E000044600B9EC68AAB9AB6843B90F49104854
:1043F000852203F0E9FD85210C4803F0B1FEAB688E
:104400005A7BD20606D1A26922B9DA897F2A01D95C
:104410006B6238BDAB68A34201D0FFF7ABFE6C62A4
:10442000F7E700BF2C0C0020040C0020509C00007B
:10443000168E000010B590F90D200446002A437B2B
:1044400006DA03F07F03014643730648FFF786FF51
:10445000054B9868031B58425841BDE81040FFF7D0
:10446000B9BF00BF2C0C0020040C002038B5044656
:104470000D46FFF7DFFF637B43F00203637325B351
:10448000184BA5609C420AD11749184840F2B53232
:1044900003F09AFD40F2B531134803F061FE2B683A
:1044A0009D4208BF0023002B38BF00239BB194F925
:1044B0000E1093F90E20914208D0521A002A05DD01
:1044C0005A68C4E9003214605C6038BD6A6893427F
:1044D00001D01B68EAE76B68C4E900531C606C609C
:1044E000F3E700BF98010020509C0000168E0000EA
:1044F0002DE9F04104460D4616461F464FF02003B5
:10450000EFF3118883F31188BFF36F8F1A48FFF719
:10451000E9FB40B919491A48812203F055FD812170
:10452000164803F01DFE1448FFF7F8FB2046294605
:10453000FFF79CFF1048FFF7E3FB40B90F49104815
:10454000AC2203F041FDAC210C4803F009FE88F3D6
:104550001188BFF36F8F7B1C08BFB6F1FF3F08D0F7
:1045600032463B4604F118000649BDE8F04100F030
:10457000CDBDBDE8F08100BF400C0020508E000092
:10458000168E0000454A000038B505460D4B0C4616
:1045900098680D4B11461860DDE90423FFF7A8FF6A
:1045A0002846FFF7ADFB40B908490948C32203F08C
:1045B0000BFDC321054803F0D3FD2046BDE838407C
:1045C000FDF786BD040C00203C0C0020508E00003E
:1045D000168E000070B50446183000F051FE4FF002
:1045E0002003EFF3118683F31188BFF36F8F204808
:1045F000FFF778FB40B91F491F48812203F0E4FC14
:1046000081211C4803F0ACFD1948FFF787FB94F9A2
:104610000D20637B002A06DA03F07F03214617484A
:104620006373FFF79BFE164D637BA86843F010038E
:104630006373031B58425841FFF7CCFE0C48FFF749
:104640005FFB40B90B490C48AC2203F0BDFCAC2128
:10465000084803F085FD86F31188BFF36F8FAB68C0
:10466000A34203D1BDE8704004F05CB870BD00BF48
:10467000400C0020508E0000168E00002C0C0020F4
:10468000040C002038B54FF02003EFF3118583F3BD
:104690001188BFF36F8F2448FFF724FB40B92349EB
:1046A0002348812203F090FC8121204803F058FD2B
:1046B000204C1D48FFF732FBA268D27B52B91E493D
:1046C0001B4840F2523203F07FFC40F252311A484C
:1046D00003F046FDEFF3058353B11749144840F248
:1046E000533203F071FC40F25331134803F038FDAC
:1046F000A2680020D37B0133D373FFF76BFE0A4817
:10470000FFF7FEFA40B909490948AC2203F05CFC06
:10471000AC21064803F024FD85F31188BFF36F8FA9
:10472000BDE8384003F0FEBF400C0020508E000072
:10473000168E0000040C0020509C000070B590F90B
:104740000D200446002A437B06DA03F07F0301466E
:1047500043732048FFF702FE637B63F07F036373BC
:104760001D4B9C420AD11D491D4840F2B53203F051
:104770002BFC40F2B531194803F0F2FC194A1146FE
:1047800051F8283FD56A8B4208BF0023002B38BF61
:104790000023CBB194F90E6093F90E0086420FD03E
:1047A000801B00280CDD5968C4E900310C605C6096
:1047B0009068031B58425841BDE87040FFF70ABE9D
:1047C000AB4201D01B68E4E7C4E900152C60D46259
:1047D000EEE700BF2C0C002098010020509C000048
:1047E000168E0000040C002070B504464FF0200324
:1047F000EFF3118583F31188BFF36F8F2548FFF71F
:1048000071FA40B924492548812203F0DDFB81215A
:10481000214803F0A5FC1F48FFF780FA204B214AEE
:10482000986811688842194613D1FFF7A3FC19480C
:10483000FFF766FA40B918491848AC2203F0C4FBE8
:10484000AC21154803F08CFC85F31188BFF36F8F02
:1048500070BD00261660144A1268BAB1C2897F2A58
:1048600014D8427BD20611D1104A90F90E6012681A
:1048700096420BDB0E4A904208D01A69A24202DC33
:10488000FFF75CFFD1E7121B1A61D0E700230B6131
:10489000CDE700BF400C0020508E0000168E0000B7
:1048A000040C00203C0C0020480C0020440C00208C
:1048B0009801002070B590F90D200446002A437B32
:1048C0003FDBDA063DD18569002D3AD163F07F03E5
:1048D00043731C4B98420AD11B491C4840F2B53225
:1048E00003F072FB40F2B531174803F039FC184968
:1048F0000B4653F8280F984218BF0546002D1A465C
:104900002B4638BF0023CD6AB3B194F90E6093F9FA
:104910000E0086420CD0801B002809DD5A68C4E9CD
:10492000003214605C600020BDE87040FFF752BDAB
:10493000AB4201D01B68E7E7C4E900252C60CC62DC
:10494000F1E770BD98010020509C0000168E000019
:10495000040C002038B504464FF02003EFF3118516
:1049600083F31188BFF36F8F1248FFF7BBF940B98B
:1049700011491248812203F027FB81210E4803F0E0
:10498000EFFB0C48FFF7CAF92046FFF793FF0948F1
:10499000FFF7B6F940B908490848AC2203F014FB08
:1049A000AC21054803F0DCFB85F31188BFF36F8F62
:1049B00038BD00BF400C0020508E0000168E000055
:1049C00038B504464FF02003EFF3118583F31188C7
:1049D000BFF36F8F1848FFF785F940B9174918489A
:1049E000812203F0F1FA8121144803F0B9FB124847
:1049F000FFF794F9637B5A0711D40F48FFF780F94A
:104A000040B90E490E48AC2203F0DEFAAC210B4847
:104A100003F0A6FB85F31188BFF36F8F38BD23F039
:104A2000040320466373FFF745FF2946BDE838407D
:104A30000148FFF709BC00BF400C0020508E000069
:104A4000168E000070B504464FF02003EFF3118678
:104A500083F31188BFF36F8F1B48FFF743F940B909
:104A60001A491B48812203F0AFFA8121174803F04D
:104A700077FB1548FFF752F914F80B3C13F0280F99
:104A800010D154F8103CA4F1180513B12846FFF7D3
:104A900083FC14F80B3C284623F0140304F80B3C69
:104AA000FFF708FF0848FFF72BF940B90749084806
:104AB000AC2203F089FAAC21044803F051FB86F3E1
:104AC0001188BFF36F8F70BD400C0020508E000026
:104AD000168E0000F8B504460E464FF02003EFF3A3
:104AE000118783F31188BFF36F8F3848FFF7FAF807
:104AF00040B937493748812203F066FA81213448AA
:104B000003F02EFB3148FFF709F9637B76B2DA0632
:104B100058D1A569002D55D103F07F036373214659
:104B20002D48FFF71BFC637BA67363F07F03637361
:104B30002A4B9C420AD12A49264840F2B53203F05A
:104B400043FA40F2B531264803F00AFB25490B46EB
:104B500053F8280F984218BF0546002D1A462B46D9
:104B600038BF0023CD6A43B394F90E6093F90E0069
:104B700086421ED0801B00281BDD5A68C4E9003223
:104B800014605C600120FFF725FC01240F48FFF74B
:104B9000B7F840B90E490F48AC2203F015FAAC2122
:104BA0000B4803F0DDFA87F31188BFF36F8F2046BF
:104BB000F8BDAB4201D01B68D5E7C4E900252C60E5
:104BC000CC62DFE7A6730024E0E700BF400C0020C2
:104BD000508E0000168E00002C0C00209801002042
:104BE000509C0000040C002038B504464FF0200310
:104BF000EFF3118583F31188BFF36F8F1648FFF72A
:104C000071F840B915491648812203F0DDF9812178
:104C1000124803F0A5FA1048FFF780F8204603F089
:104C20008BFD044628B1FFF7B7FB04F1180000F034
:104C300027FB0948FFF764F840B908490848AC2247
:104C400003F0C2F9AC21054803F08AFA85F3118814
:104C5000BFF36F8F204638BD400C0020508E0000FF
:104C6000168E00000021044B084603F12802C3E918
:104C70000A22FFF795BA00BF040C0020F8B5EFF345
:104C8000058353B1404941484FF4966203F09CF9C3
:104C90004FF496613C4803F063FA3D4D3D4EAB68DE
:104CA000B34267D04FF02003EFF3118783F31188ED
:104CB000BFF36F8F3848FFF715F840B937493348CD
:104CC000812203F081F98121344803F049FA324806
:104CD000FFF724F8A96832484B7B03F07F034B733E
:104CE000FFF73CFBAC68637BB44263F07F03637304
:104CF0000AD12549254840F2B53203F065F940F262
:104D0000B531214803F02CFAAB6A2548E96A8342A1
:104D100008BF0023002B38BF002333B394F90E6083
:104D200093F90E2096421CD0921B002A19DD5A6876
:104D3000C4E9003214605C600120FFF74BFB1648A9
:104D4000FEF7DEFF40B915491048C32203F03CF9D5
:104D5000C321124803F004FA3846BDE8F840FDF7D5
:104D6000B7B98B4201D01B68D7E7C4E900010C60DA
:104D7000EC62E1E74FF02003EFF3118083F3118839
:104D8000BFF36F8FE9E700BF509C0000168E000054
:104D9000040C002098010020400C0020508E0000E0
:104DA0002C0C00202DE9F04106460F46EFF3058359
:104DB00053B13549354840F2D14203F005F940F28C
:104DC000D141314803F0CCF956EA070304D1FFF78B
:104DD00055FF0020BDE8F08103F0B8FC84194FF0C6
:104DE0002003EFF3118883F31188BFF36F8F2848F6
:104DF000FEF778FF40B927492448812203F0E4F800
:104E00008121244803F0ACF9234D2148FEF786FFA9
:104E1000A868224B1860FFF70DFBA86832463B4696
:104E200018301F4900F072F9AA681948537B43F003
:104E300010035373FEF764FF40B916491348C322A9
:104E400003F0C2F8C321134803F08AF94046FDF786
:104E50003FF9AB685B7BDB060AD50B490B4840F298
:104E6000EF4203F0B1F840F2EF41074803F078F960
:104E700003F06CFC201A64EB0401002871F10003BC
:104E8000B8BF0020A6E700BF509C0000168E0000AF
:104E9000400C0020508E0000040C00203C0C002030
:104EA000454A000038B504460D46EFF3058353B17B
:104EB0001149124840F2FE4203F086F840F2FE41EA
:104EC0000D4803F04DF96B1C08BFB4F1FF3F06D14C
:104ED0000B4B9868FFF77EFB4FF0FF3038BD204644
:104EE0002946FFF75FFF4FF47A7380FB0334D80B3A
:104EF00040EA4440F2E700BF509C0000168E0000DC
:104F0000040C0020014B9868704700BF040C00207F
:104F10002DE9F04104464FF02003EFF3118683F3AF
:104F20001188BFF36F8F3E48FEF7DCFE40B93D4964
:104F30003D48812203F048F881213A4803F010F9F6
:104F40003748FEF7EBFE637B1A0712D53448FEF7AD
:104F5000D7FE40B933493448AC2203F035F8AC21D0
:104F6000304803F0FDF886F31188BFF36F8FBDE87A
:104F7000F08123F0200242F00801D20938D1617398
:104F8000A36813B12046FFF707FA04F1180000F0F8
:104F900077F94FF0000804F15807A56DBD4200D025
:104FA00085BB0120FFF716FA204B9B68A342CDD1A9
:104FB000EFF30583002BC9D11948FEF7A1FE40B9D4
:104FC00018491948C32202F0FFFFC321154803F016
:104FD000C7F83046FDF77CF840F2116214491248D8
:104FE00002F0F2FF40F21161114803F0B9F8ADE7A9
:104FF00003F05F0343F0080321460E486373FFF795
:10500000ADF9BDE72846FFF7C7F905F1180000F034
:1050100037F92846C5F87880FFF74CFCBDE700BF9C
:10502000400C0020508E0000168E0000040C002062
:10503000509C00002C0C002008B50648064A074981
:10504000121A03F0CCF9BDE80840054A05490648A4
:1050500003F0C5B90000002098010020D49C000096
:1050600000000000D49C000000000020034B1B68DF
:105070000BB9FCF7D3BC0020704700BF4C0C0020DC
:1050800030B5036868B10A4A5268904209D043B10A
:10509000D3E90421D0E90445121945EB0101C3E924
:1050A0000421426813605A600023C0E9003330BD18
:1050B0005800002038B5134B1C689C4208BF0024E0
:1050C000FFF7D4FF0546BCB1D4E90401401B61EBF6
:1050D000E571012871F1000311DB6FF0004200233C
:1050E000824273EB010400DA1046074B1B6913B1CF
:1050F0009842A8BF184638BD6FF00040F5E7002081
:10510000F3E700BF58000020040C00202DE9F74F02
:105110001D466B1C08BFB2F1FF3F82468B4614460A
:1051200000F09C80036843B14E494F485D2202F075
:105130004BFF5D214B4803F013F8CAF808B04FF05D
:105140002003EFF3118B83F31188BFF36F8F474870
:10515000FEF7C8FD40B946494348812202F034FFBA
:105160008121434802F0FCFF4048FEF7D7FD6FF075
:1051700001034FF0FF32B3EB040862EB0509B8F10D
:10518000000F79F100011CDB3A48D0E900105B1AEE
:1051900062EB00021E1B62EB0507012E77F1000394
:1051A000BCBF01260027CAE90467334AD2E90036AA
:1051B00093421DD1CAE90026C6F800A0C2F804A097
:1051C0002CE0FFF753FF631C009345F100030193AC
:1051D000DDE90023121843EBE073CAE90423E4E796
:1051E000E01B65EB0801B342CAE90401E2D01B6889
:1051F000002BDFD0D3E90478DAE90445BC4275EB33
:105200000801EDDA381B68EB0501C3E904015968B0
:10521000CAE90031C1F800A0C3F804A013689342A2
:105220000BD09A4509D1FFF745FF18B1134B1B6905
:10523000834202D00021FCF7BFFB0C48FEF760FD63
:1052400040B90B490848AC2202F0BEFEAC21084828
:1052500002F086FF8BF31188BFF36F8F03B0BDE8B8
:10526000F08F00BF729C0000168E0000500C0020D2
:10527000508E00009802002058000020040C0020EE
:1052800038B504464FF02003EFF3118583F31188FE
:10529000BFF36F8F1548FEF725FD40B91449154837
:1052A000812202F091FE8121114802F059FF0F483E
:1052B000FEF734FD2368B3B12046FFF7E1FE00247A
:1052C0000A48FEF71DFD40B909490A48AC2202F020
:1052D0007BFEAC21064802F043FF85F31188BFF343
:1052E0006F8F204638BD6FF01504E9E7500C0020A1
:1052F000508E0000168E000038B54FF02003EFF3FB
:10530000118583F31188BFF36F8F1348FEF7EAFC12
:1053100040B912491248812202F056FE81210F48FD
:1053200002F01EFF0C48FEF7F9FCFFF7C3FE04462F
:105330000948FEF7E5FC40B908490948AC2202F0EB
:1053400043FEAC21054802F00BFF85F31188BFF343
:105350006F8F204638BD00BF500C0020508E0000DB
:10536000168E000070B504460D464FF02003EFF393
:10537000118683F31188BFF36F8F1648FEF7B2FCD6
:1053800040B915491548812202F01EFE81211248BC
:1053900002F0E6FE0F48FEF7C1FCFFF78BFE012886
:1053A00005DDA04203DB29462046FCF705FB094842
:1053B000FEF7A6FC40B908490848AC2202F004FEFA
:1053C000AC21054802F0CCFE86F31188BFF36F8F45
:1053D00070BD00BF500C0020508E0000168E0000E3
:1053E0002DE9F04F85B00446FFF7FEF94FF020039A
:1053F000EFF3118983F31188BFF36F8F4C48FEF7E9
:1054000071FC40B94B494C48812202F0DDFD8121FD
:10541000484802F0A5FE494F494EBB464448DFF8D4
:1054200024A1FEF77BFC3460D6F800C0DAF80080D7
:105430006246D7E90034D045CDE902344FEAE27341
:10544000CDE9002311D0B8F1000F0ED0D8E9041235
:10545000DDE900348B4274EB02032ADA009BC81AA0
:10546000019B62EB0301C8E904010024009B029A3E
:1054700003999A18019B346041EB0303CBE90023A5
:10548000FFF718FE2146FCF797FA2948FEF738FC8B
:1054900040B928492848AC2202F096FDAC212548A5
:1054A00002F05EFE89F31188BFF36F8F05B0BDE88F
:1054B000F08F0022DDE9024500236418ACEB010007
:1054C00045EBE1753060C8E904234046C7E9004573
:1054D000FFF7D6FD1648FEF713FC40B915491648EC
:1054E000AC2202F071FDAC21124802F039FE89F3C2
:1054F0001188BFF36F8F4046D8F8083098474FF0B7
:105500002003EFF3118983F31188BFF36F8F0848ED
:10551000FEF7E8FB40B907490748812202F054FD35
:105520008121044802F01CFE0148FEF7F7FB7BE7EF
:10553000500C0020508E0000168E000098020020B3
:105540004C0C00205800002070B54FF02003EFF302
:10555000118683F31188BFF36F8F1648FEF7C2FBE5
:1055600040B915491548812202F02EFD81211248CB
:1055700002F0F6FD0F48FEF7D1FBFCF74FFA104B97
:10558000D3E9004524180B4845F10005FEF7B8FBA8
:1055900040B909490948AC2202F016FDAC21064881
:1055A00002F0DEFD86F31188BFF36F8F2046294697
:1055B00070BD00BF500C0020508E0000168E000001
:1055C00098020020024A0349034802F0FDBC00BFD4
:1055D0004D8F0000969C0000A69C000010B50C4C5E
:1055E000236813B10B4B1B682BB900F099FA30B943
:1055F0000122084B1A6001230020236010BD0138EE
:10560000062801D9044810BD044B53F8200010BDF2
:10561000540C0020580C0020FE8FFFFF6C8C000003
:10562000BFF34F8F0549064BCA6802F4E06213438B
:10563000CB60BFF34F8F00BFFDE700BF00ED00E080
:105640000400FA054FF0FE33002130B4064A074D3E
:10565000074C2B6013602360064A074CEB606368BD
:10566000C2F8001530BC184704148450001484504C
:10567000081484500000845060000020024BD0E9E0
:105680000012C3E900127047600000202DE9F043CA
:10569000154CDFF85C80002818BF0446206883B0F2
:1056A00040451DD016460D4620464FF4DE7104F1EC
:1056B000040900F079FE04F58C77484600F01CF9E7
:1056C000384601F047FA4A4638462B4607490096C5
:1056D00001F052FA08B9C4F8008003B0BDE8F083C5
:1056E000002003B0BDE8F0835C0C00207959000075
:1056F000A5BCC95AF0B50D4C0D4E002808BF204678
:10570000076883B0B7420ED100261D4600F58C70A5
:1057100033460096144601F07FFA002818BF34463D
:105720002C6003B0F0BD0348FBE700BF5C0C002019
:10573000A5BCC95AE88FFFFF48B143682BB1BFF33E
:105740005F8F0023036018467047024870476FF46C
:10575000E0407047EA8FFFFF10B5044628B1636848
:1057600013B100232360636010BD024B02485B68E5
:105770009847F4E760000020888C000010B50446CC
:1057800030B100226368226043F00103636010BD02
:105790000148FFF757FFF4E7B08C000080B1436881
:1057A00063B10122D0E8EF3FC0E8E12F0029F9D131
:1057B000012BF7D0BFF35F8F00207047024870477E
:1057C0006FF4E040704700BFEA8FFFFF70B40B4BEF
:1057D0000668C268D0E90154C3E90242C3E9006522
:1057E000D1E903020E68064BD1E90154C3E9006513
:1057F000C3E902401A6170BC704700BF700000200E
:10580000800000202DE9F043202B1D4606468946E6
:1058100090468BB026D8DBB202AF31688DF8049089
:105820008DF8053006F1040921B9484600F062FE02
:10583000044640B9012302224846336001A900F022
:105840006DFE044638B13846202100F0ADFD2046FB
:105850000BB0BDE8F0832A464146484600F05EFEA4
:105860000446F0E702AF1946104600233A4601F01D
:10587000ADFA04460028E6D12023B8461D46CCE701
:10588000F0B5D0F8F430A7B0002BD8BF02AE2CDDB5
:1058900005460023D0F8084102AE0193A4F10107A8
:1058A0003146D5F8F8409022D0F8FC0001ABB7FAA9
:1058B00087F7A0477F09044610B9019B3BB9A7B100
:1058C0003046902100F070FD204627B0F0BD014623
:1058D00032462846FFF796FF50B9D5F80031019AB5
:1058E0001344C5F80031002FEAD16FF03C04E7E71C
:1058F0000446204627B0F0BD70B500250446294671
:105900001422C0F8F450F83002F094FD164B04F560
:1059100086761B6830469847204640F8045B00F0C6
:10592000CFFD124B30461B689847D8B9D4F8F430F5
:10593000AB4211DC0121202503EB830204EB820240
:10594000C2F8FC000A480B44C2F80451C2F8F8003F
:10595000C2F80811C4F8F430064B3046BDE8704078
:105960001B68184770BD00BFC4000020C80000209D
:10597000BD630000CC0000202DE9F047202A88B04C
:1059800078D83E4B00F5867904461B684846174692
:1059900088469847054640BB40F20116D4F8F430DB
:1059A000002B63D02046FFF76BFF054600285FD130
:1059B000D4F8F430002B07DDD4E94002904203D341
:1059C000D4F80821012A14D0013EE9D16FF03B053B
:1059D0006E463046202100F0E7FC294B48461B6804
:1059E0009847002818BF6FF01D05284608B0BDE88D
:1059F000F0871F28E8D96E4629462022304604F158
:105A0000040A02F017FD3146504600F08FFD0546AE
:105A10000028DED1504600F067FD504600F050FDF2
:105A20002946504600F066FD05460028D1D1504673
:105A30002022314600F072FD05460028C9D10346F8
:105A400032462021304601F0C1F905460028C0D178
:105A5000D4F8F4303A46002BC8BF00234046314604
:105A6000C8BFC4F8003102F0BAFCB2E76FF03F05DE
:105A70006E46AEE76FF03B05B7E700BFC8000020F9
:105A8000CC000020002130B58DB0282202A8019161
:105A900002F0D0FC02A801F0C1F9044610B1204682
:105AA0000DB030BD184D4FF0FF31286800F03AF9C5
:105AB0000446C0B9002000F065F900BB134A02A9F2
:105AC00001A800F063FC0446012000F05BF990B9E6
:105AD000286800F02FF90028E1D00D48FFF7B2FD4B
:105AE00020460DB030BD0B48FFF7ACFD012C08BFC0
:105AF0000524EDD0DEE70848FFF7A4FDE8E70748F6
:105B0000FFF7A0FDDAE700BFC0000020900E0020E4
:105B10002C8D0000D48C00000C8D0000EC8C00005B
:105B200010B582B000F054F828B100F0A3F80324B7
:105B3000204602B010BD00F06FF8D0B900F022F995
:105B4000D8B91E4B1B681B0EF02B0AD11C4A1D4BEB
:105B500012689A4229D000F03DF8072400F08AF834
:105B6000E6E7062400F036F800F084F8204602B09C
:105B700010BD0424204602B010BD00F02BF800F048
:105B800079F8FFF77FFF044658B902460146FFF750
:105B90007DFD30B968220C4901ABFFF7ABFD002851
:105BA000C6D00524204602B010BD012000F0EAF85E
:105BB0000028E2D1054B1860E3E700BF28198450A4
:105BC000241A84500000E020280E00200C1A845073
:105BD0000020704700207047430503D54FF0FF3287
:105BE000024B1A60024B1860704700BF08118450C6
:105BF000081A8450014B1860704700BF041A845083
:105C000008B100F06DB84FF47500704708B100F0AE
:105C10004FB84FF47500704710B5114800F06EF89A
:105C200000B110BD0F4800F069F80028F9D10E4C02
:105C3000204600F063F80028F3D10C4B0C481C60A0
:105C400000F05CF801460028EBD100F02DF8044686
:105C500008B1204610BD00F077F82046FAE700BFF3
:105C6000BC000020B0000020B8000020C0000020D0
:105C7000B400002008B5084800F04AF8074800F0D2
:105C800047F8074800F044F8064800F041F8BDE83E
:105C9000084000F00BB800BFBC000020B00000209E
:105CA000B8000020B400002000207047704700BFFB
:105CB0000246074803681342FCD021B1054B064851
:105CC0001B680B600360054B00201A60704700BF23
:105CD000001A84500411845008118450081A84500A
:105CE000024604490B681A42FCD0034B00201A609C
:105CF000704700BF001A8450081A845008B5034B3F
:105D000002681B6810689847002008BD70000020DA
:105D100008B5034B02685B6810689847002008BD0F
:105D200070000020024B02689B681068184700BF93
:105D30007000002008B5034B0268DB6810689847C4
:105D4000002008BD7000002070B5094C094D206985
:105D5000AB68984718B1084B08485B689847002122
:105D6000074AEB6811602069BDE87040184700BF22
:105D7000800000207000002060000020448D0000A2
:105D8000B010002070B51A4D1A4E0446B26828694A
:105D90009047F0B95CB1184C2368ABB1012B1AD015
:105DA000013B23602869F3689847002070BD124CBE
:105DB000216839B90120114B114AC3F80005136855
:105DC000002BFCD101312160F3682869984700203D
:105DD00070BD0C4870BD0A4A1368002BFCD1074AFD
:105DE0006FF07E40C2F80035FFF704FF2368D7E765
:105DF0008000002070000020B010002000008450BF
:105E000010198450E98FFFFF014B1B68184700BF32
:105E100070000020014B9B68184700BF70000020F5
:105E2000014BDB68184700BF700000202DE9F843E4
:105E3000002878D00C46002975D01D46002B72D062
:105E400006461AB1012200232A6003602B68002B4A
:105E500065D02946204601F0DDF8074600285FD1CD
:105E60002146286801F0B8F80746002858D12B6869
:105E7000082B67D0042B68D0A3F10208B8FA88F881
:105E80004FEA581801239C46314A324913601046A4
:105E90000B60943AC0F800C0636A136011688B42CB
:105EA000F8D14FF000092C4B4FF0FF30C3F80090B1
:105EB000FFF792FE6FF01B02284B48461A60FFF76F
:105EC00099FE274A274BC2F80080186840F480608A
:105ED000FFF790FE0A22244B1A60089A2369012AD0
:105EE000616A24D0214AA2FB03231B09012203FB80
:105EF00001F303EB43031E49DB039B090B60164BC5
:105F000038461A6033682A6823F07F4343EA026305
:105F100033602A6843EA02233360BDE8F883154FF3
:105F20003846BDE8F883144F3846BDE8F8834FF48F
:105F30007F03D3F80C2C013202D0D3F80C3CD1E70C
:105F40001623D3E74FF003089CE74FF0020899E7C8
:105F5000C4118450401184502C118450001184507D
:105F60000C118450041A845038118450ABAAAAAA88
:105F7000D8118450310CF100350CF100F0B400243C
:105F8000C9002646274601F1FF3C06E09F4215D096
:105F90000126654518D82C461F46630950F8233062
:105FA00004F01F01CB401F2904F1010518BF03F0C5
:105FB0000103002CEAD101263546ECE70136964272
:105FC000E7D10348F0BC70470020F0BC704700BF29
:105FD000360CF10000285FD02DE9F0414C1EB4F5DD
:105FE000047F26D22BB322B3CC00012B04F1FF3E59
:105FF0002FD000218C460F460D4603F1FF384C0987
:1060000050F8244001F01F06F4401F2E18BF04F082
:10601000010421B90125AC4629462746EFE7AB42EA
:1060200013D0A74201D10CF1010C454504D16245C2
:1060300002D21A48BDE8F0813C4601318E4505F197
:106040000105EAD20020BDE8F08100254FF0010CE7
:10605000F3E70026B446374631464B0950F8233063
:1060600001F01F05EB401F2D18BF03F0010339B1EC
:106070005FB99C4501D0634608E06346013605E000
:10608000012631469C460127E7E73E46B242D0D37F
:106090000131A142F6D1D5E700487047370CF10035
:1060A0002DE9F04F8DB0189E07460C46179D002E27
:1060B0004CD1D1F810B000211D60169B1960002A48
:1060C00000F022819C4A9D4B1168626A1B689A42CB
:1060D00047D10A2945D1FB7804930423B84602939B
:1060E000974BA3FB0B234FEA930A0AEB4A0305F1F4
:1060F00008020392ABEB430A169BC3F800B0BBF156
:10610000000F00F0C7805D464FF00009039E00F0CD
:1061100091FF00230593B8F1000F00F0E980002CF7
:1061200000F0E680049B002B00F0E080204604A9EC
:1061300000F070FFB8B1834B984240F0AB80029002
:1061400000F078FF02980DB0BDE8F08F4FF47F01AA
:10615000D1F80C0C01300CBF4FF4047BD1F80CBC0F
:10616000A9E77948EBE72146049800F035FF0028BD
:10617000E1D1049F082F00F0BD80042F00F0BC8007
:10618000A7F10207B7FA87F77F09012319466F487D
:10619000036040F8843C6D4B68481960636A036093
:1061A00000688342F7D10023694A4FF0FF30136043
:1061B000FFF712FD00236FF01B011846654B1960B5
:1061C000FFF718FD6449654B0F6018685C4F40F499
:1061D0008060FFF70FFD0A210122574B60481960CC
:1061E0002169636AA7FB01C1090903FB01F303EB02
:1061F0004303DB039B090360554B05A81A60049910
:10620000D8F800200B0243EA016322F07F421343D7
:10621000C8F8003000F0D0FE059B03F01A030343DA
:1062200038D1504BA7FB05271A681433069253F850
:10623000102CB9EB970F079253F80C2C089253F8D7
:10624000082C099253F8042C0A921B680B9302D174
:10625000BAF1000F41D1182230460DEB020100F0D7
:106260001BFE183D183609F10109002D7FF44FAFD0
:10627000BBF5047F5DD8039D594628466269FFF748
:106280007DFE00284BD00023169A13602D4B9842B8
:106290003FF455AF049D082D34D0002204AB2146B5
:1062A00040466D0000920495FFF7C0FD2E4B9842CA
:1062B00024D000287FF443AFD8F80020130A03F459
:1062C0007F03134323F07F43C8F80030029B013B58
:1062D00002937FF411AF002031E73046524606A901
:1062E00000F0DAFDA5EB0A055644BCE71E4822E79C
:1062F0001E4820E7032748E7022746E7236A002BCA
:106300003FF41DAF1A481AE701222146384600968D
:1063100004ABFFF78BFD00283FF4DFAE0FE74FF42F
:10632000806359462846A269FFF754FE0028AAD187
:10633000D1E7169B1D60ADE73811845030118450B1
:10634000ABAAAAAA020CF100300CF100C4118450CF
:106350002C118450001184500C118450041A845064
:10636000D811845014118450310CF100350CF10017
:10637000320CF100002330B4DDE903450493029BA5
:10638000CDE9024530BCFFF78BBE00BF10B501243C
:1063900086B005ABCDE901240093002204ABFFF7E2
:1063A0007FFE06B010BD00BF38B131B100220144FC
:1063B0000346013081421A70FAD170472DE9F0414D
:1063C00088B00592002968D01C46002B65D0154680
:1063D000002A62D0DFF8E4800E46D8F800004FF0C3
:1063E000FF31FFF79FFC00284CD10020FFF7CAFCCB
:1063F000002843D12A4800F011FDE8B101204FF0F8
:10640000FF37FFF7BFFC002834D14FF4087125484F
:10641000FFF7CAFF04212448FFF7C6FF20482821C0
:10642000FFF7C2FFD8F80000FFF784FC00282DD149
:10643000384608B0BDE8F0811A4907AB0246039020
:106440000291009316491848019405ABFFF792FF9B
:106450000028D3D12368AB42D0D3079907462A46F8
:106460003046083100F018FD01202560FFF78AFC56
:106470000028CAD00D48FFF7E5F8C6E70C48FFF73B
:10648000E1F8B7E70B48FFF7DDF8AEE70A48FFF79A
:10649000D9F8384608B0BDE8F0814FF0FF37C7E7BC
:1064A000D8120020B8100020B41000200C8D00007D
:1064B000EC8C0000D48C0000648D0000C000002033
:1064C00010B5044628B12046BDE81040F02100F088
:1064D000E7BC0448FFF7B6F82046BDE81040F021BD
:1064E00000F0DEBC7C8D000010B1F021FFF75CBF36
:1064F000704700BF08B561B1012907D1022100F042
:1065000039F8002818BF6FF0360008BD6FF036006C
:1065100008BD012100F02EF8F3E700BF08B500F038
:106520006BF8002818BF6FF0360008BD70B5E8B1F1
:106530000E46D9B1044600F031F80546B0B92368DB
:10654000012B0BD0022B01D0284670BD30461C22F7
:1065500004F1080100F0A0FC284670BD304620225E
:1065600004F1080100F098FC284670BD6FF0360574
:10657000EAE700BF78B138B50D46F021044600F0D7
:106580008FFC402320462560E36500F099FD00382C
:1065900018BF012038BD0120704700BF70B5056EDF
:1065A000A4B0044604AEE5B901220023626030467F
:1065B0002946CDE9003302AA00F04AFD10B10120BE
:1065C00024B070BD2A46204602A900F0A3FD002891
:1065D000F5D1204600F0C8FE0028F0D1206624B096
:1065E00070BD802D2A46304628BF802204F1640108
:1065F00000F052FC256ED7E7002855D0F0B51546BF
:10660000A5B0B2B10E4651B30446D0E917301A1AFC
:10661000B2FBF3F703FB1727AF4228BF2F46002F2B
:1066200044D1834208D0B5FBF3F703FB07F7CFB99A
:106630006DBB284625B0F0BD802B28BF802304F118
:1066400064011A4604A800F027FC0023CDE90033BA
:1066500004A8E16D02AA00F0FBFC002833D0012061
:1066600025B0F0BD002339463046CDE9003302AAFB
:1066700000F0EEFC0028F2D13A46204602A900F0D4
:1066800049FD0028EBD1ED1B3E44002DD1D0206EFA
:106690002A461930314604EB800000F0FDFB226EE3
:1066A00000202A442266C5E70120704704F16403F4
:1066B00018443A4600F0F0FBD4E9173038443E4421
:1066C000ED1B2066ADE72046E26D02A900F022FD39
:1066D0000028C4D1E36D2066A5E700BF2DE9F04195
:1066E0002022044688B00D4668460021A6186F4651
:1066F00001F0A0FEE27B0132D2B2E273002A4DD15A
:10670000A27B0132D2B2A273002A47D1637B01334C
:10671000DBB26373002B41D1237B0133DBB22373E4
:10672000002B3BD1E37A0133DBB2E372002B35D18E
:10673000A37A0133DBB2A372002B2FD1637A01332A
:10674000DBB2637253BB237A0133DBB223722BBB00
:10675000E3790133DBB2E37103BBA3790133DBB22D
:10676000A371DBB963790133DBB26371B3B9237908
:106770000133DBB223718BB9E3780133DBB2E37011
:1067800063B9A3780133DBB2A3703BB963780133FB
:10679000DBB2637013B92378013323703B46224682
:1067A0000121304600F050FE804600282AD11037E3
:1067B00008AB9F429ED100992B686A684B400199B3
:1067C00030464A40AE68029900937140EB68039EE0
:1067D000019273402A69049E0291564005996A69A4
:1067E00003935140D5E90623069D05915540079A2C
:1067F000694653408022CDE90653049600F00AFE14
:10680000804638B168462021FFF7CEFD404608B0EB
:10681000BDE8F081102220460DEB020101F0DFFD02
:10682000F0E700BF2DE9F04F06468069AFB0B0F544
:10683000C07F00F27C811D46C0F5C073AB42C0F042
:106840007681C5F5C073181A90421746C0F06F8163
:10685000DFF8E8924FF4C07288464846002101F004
:10686000E9FD4946D6F89430B269D6F898009847C1
:10687000002840F05F81B46955B12A464946D6F8F0
:106880009430D6F898009847002840F053812C4463
:10689000B8F1000F02D0002F40F02281B4F5C07F84
:1068A00088BF6FF0370500F21281DFF8A4824FF441
:1068B000D0720021404601F0BDFD11A800F094FD0A
:1068C0002023002165BA2246A8F81010A8F812501B
:1068D0009A4988F8173008F1180001F080FD8022ED
:1068E000974B984D984908EB0400CDE90251027688
:1068F000019311A803F10C3301A9049300F08AFD60
:106900000546002840F0F48004F119070DF1140940
:106910000DF1240B10220021484601F08BFDBA46F0
:106920008A4C9DF8142014F8103C9DF815C014F8FA
:106930000F1C9DF81600534014F80E2C8CEA010C25
:1069400050409DF8171014F80D2C9DF818E0514098
:1069500014F80C2C8DF814308EEA020214F80B3C5B
:106960009DF819E08DF815C08EEA030314F80ACCDF
:106970009DF81AE08DF816008EEA0C0C14F8090C3C
:106980009DF81BE08DF817108EEA000014F8081C23
:106990009DF81CE08DF818208EEA010114F8072CF0
:1069A0009DF81DE08DF819308EEA02029DF81E3028
:1069B00014F806EC8DF81AC083EA0E038DF81B005C
:1069C0008DF81C108DF81D208DF81E309DF81F10BD
:1069D00014F8053C9DF820C09DF821004B4014F8A8
:1069E000042C14F8031C8CEA020241409DF822C0DA
:1069F00014F8020C9DF823E08CEA000014F801CC96
:106A00008DF81F308EEA0C0C8DF820208DF82110A7
:106A10008DF822004B464A46012111A88DF823C06B
:106A200000F012FDBAF1100F94BFAAEB0A0AAAF106
:106A3000100A002879D11034BAF1000F7FF471AF39
:106A40000BEB05001022494601F0C9FC98F8033011
:106A500010350133202D88F803307FF45BAF80229E
:106A6000594611A800F0D6FC0546002844D1334C05
:106A700004F120070DAB1A46012111A800F0E4FC37
:106A80000546002838D1102220460DA9144401F0F3
:106A9000A6FCBC42EED111A800F0B6FC4FF4D071B8
:106AA0002B48FFF781FC58462021FFF77DFC102181
:106AB00001A8FFF779FC48461021FFF775FC304626
:106AC0001E49FFF70BFE054608B9012333614FF459
:106AD000C0711A48FFF768FC28462FB0BDE8F08F58
:106AE00009EB040041463A4601F079FC3C44D5E606
:106AF0000DF114090DF1240B11A800F085FC4FF4E1
:106B0000D0711348FFF750FC58462021FFF74CFC8A
:106B100001A81021FFF748FC48461021FFF744FC6C
:106B200020210648FFF740FCD1E70546E4E76FF077
:106B30003705D1E76FF03305CEE700BFA014002082
:106B4000000102030405060708090A0B10130020C0
:106B50000013002010B5A4220021044601F06AFCB5
:106B60004FF0FF32034B226104F19C001B68BDE82B
:106B700010401847C40000202DE9F04104460E469D
:106B8000154684B01022002100F1200868461F46F7
:106B900001F050FC404600F027FCA269C4E92565DD
:106BA000D2B920222669A261002E2FDB4FF6F073A6
:106BB000694640468022E36100F02CFC054638B966
:106BC000134B04F19C0840461B689847054658B192
:106BD000284604B0BDE8F0812669002EE6DA172ABF
:106BE00014D801325608E1E7334639460A9A20465E
:106BF000FFF718FE074B05461B68404698470028DC
:106C000018BF0546284604B0BDE8F0810026CDE750
:106C1000C8000020CC0000202DE9F047B2F5806FBD
:106C20008CB0149F00F2CB80B7F5807F00F2C48057
:106C3000044615460E462022002104A8984601F07D
:106C4000F9FB2169E269914200F387806369002BB7
:106C500040F08380002F40F0A7806F46002D00F0A9
:106C600098806F4604F120080EE0102DA94628BF39
:106C70004FF01009304639464A4601F0B0FBB5EBFB
:106C800009054E4400F08580E37B0133DBB2E373FA
:106C9000002B4DD1A37B0133DBB2A373002B47D173
:106CA000637B0133DBB26373002B41D1237B013360
:106CB000DBB22373002B3BD1E37A0133DBB2E37207
:106CC000002B35D1A37A0133DBB2A372002B2FD175
:106CD000637A0133DBB2637253BB237A0133DBB2D5
:106CE00023722BBBE3790133DBB2E37103BBA379DE
:106CF0000133DBB2A371DBB963790133DBB26371BA
:106D0000B3B923790133DBB223718BB9E378013353
:106D1000DBB2E37063B9A3780133DBB2A3703BB994
:106D200063780133DBB2637013B9237801332370C6
:106D30003B4622460121404600F086FB8146002862
:106D400093D0202104A8FFF72FFB38461021FFF72E
:106D50002BFB48460CB0BDE8F0871A4B04F19C0AA7
:106D600050461B68984781460028F2D103463A46B0
:106D700041462046FFF756FD134B07461B68504619
:106D8000984781460028E4D1002F3FF466AFB9460A
:106D9000DFE7204604A9FFF7A1FC81460028D0D1F7
:106DA000236901332361CCE7064B04F19C001B6887
:106DB00098476F468146C4E76FF03709C9E76FF01F
:106DC0003509C6E7C8000020CC000020F8B51C46F5
:106DD000054611480E461746FFF772FB21460E483E
:106DE000FFF788FB044620B10B48FFF77DFB2046E8
:106DF000F8BD324629460848FFF790FB04460028B4
:106E0000F2D139460448FFF791FB04460248FFF7E8
:106E10006BFB2046F8BD00BF201600201C2330B5B8
:106E200083B001A90446019300F03EF8054638B945
:106E3000019B1C2B07D0164D20461C2100F030F87A
:106E4000284603B030BD0121D4E90032003B18BF11
:106E50000123E1610AB143F00203A26832B9E2689A
:106E600042B9C4E908328BB90A4DE5E7E26843F05C
:106E700004033AB10022284643F00803C4E908326B
:106E800003B030BD1546C4E90832D9E71546D7E747
:106E9000370CF0000E0CF00001F08ABA01F0CABA0B
:106EA0000A46002101F0C6BA002866D0002964D045
:106EB0000B681C2B61D14FF47F033B4AD3F8101CA5
:106EC00091425CD0D3F8102C013258D0D3F8102C5A
:106ED0004FF47F030260D3F8141C344A914260D00F
:106EE000D3F8142C01325CD0D3F8142C4FF47F0368
:106EF0004260D3F8182C12F5947F4FD0D3F8182C99
:106F000001324BD0D3F8182C4FF47F038260D3F8B2
:106F10001C1C274A91423ED0D3F81C2C01323AD097
:106F2000D3F81C2C4FF47F03C260D3F8002C7032CE
:106F30002FD0D3F8002C01322BD0D3F8002C4FF4F3
:106F40007F030261D3F8042CAF3220D0D3F8042C95
:106F500001321CD0D3F8042C4FF47F034261D3F8E4
:106F6000081C144A91420DD0D3F8082C013209D0E4
:106F7000D3F8083C8361002070470120704740F639
:106F8000FC02A5E740F237338361002070475122AD
:106F9000E2E79022D3E742F60412C3E740F6D86254
:106FA000B2E742F2D002A1E7FCF8FFFFD020FFFFDA
:106FB0000429FFFF37F3FFFF014608B54FF4806057
:106FC000FEF724FE00230249024A0B60136008BD4D
:106FD000C81184502C1184500138072805D8DFE8E7
:106FE00000F00A0E04120404040609487047CB6836
:106FF00000204B6270470B6800204B6270474B6863
:1070000000204B6270478B6800204B62704700BFC6
:10701000310CF1000B6802E0082B0B6006D8026A05
:1070200013424FEA4303F7D00020704700487047EF
:10703000310CF10000230449044A0B604FF48060D6
:107040001360FEF7C9BD00BF2C118450C4118450D9
:107050002DE9F041002682B0B0F1005F8DF80760A5
:10706000099E27D30C460444B4F1804F054621D82D
:107070001746984601220DF1070300F00FFA044667
:10708000C0B99DF807303D603B71AEB1B8F1000F5B
:1070900009D00246089940460DF1070300F0FEF9B9
:1070A00040B99DF807302046C6F80080337102B021
:1070B000BDE8F0814FF47504204602B0BDE8F081D0
:1070C000E8B110B50468012C04D0022C10D044B1F2
:1070D0000C4810BD20220C490830FFF7DDFE0020CF
:1070E00010BD142209490830FFF7D6FE204610BD16
:1070F000202207490830FFF7CFFE002010BD4FF4D3
:10710000730070470100F300C08D00008C8D0000FB
:10711000A08D00002DE9F041002900F0EF80044629
:10712000002800F0EF80036817460E46002B00F0A1
:10713000B980013B012B00F2CD804FF0FF31734845
:107140004FF00208FEF7EEFD002840F0B580002069
:10715000FEF718FE0546002840F0B8806C4A136818
:10716000002BFCD16B480368002BFCD14FF0FF30A3
:10717000FEF732FD684B186820F04000FEF73AFD3C
:1071800001230720654A66491360086042F8543CB1
:10719000A16C644B483A1960E16C116043F80C8CA7
:1071A000236863B1013B012B18D8616A5E4BA2F5DD
:1071B000BC721960216A1160E26943F8082CA16968
:1071C0005A4B5B4A196061691160216943F8081CD8
:1071D000E16842F8081CA26843F8102C554A13686D
:1071E000002BFCD1002F59D063684020012B04BF35
:1071F000514A13603168514A514B11601F60FEF7CC
:10720000FFFC05464B4A1368002BFCD1414A13682A
:10721000002BFCD123685BB1013B012B16D8424BFC
:10722000484A1968083B6162126822621B68E36180
:107230003E4B3F4A1968083AA1619168103B616171
:10724000996821611268E2601B68A3600121002334
:1072500034483D4A0068A0641068E06442F80C1CA1
:1072600035483A49036002F5A0720B601368002BA1
:10727000FCD12A4A1360002D3AD1274B186840F000
:107280004000FEF7B7FC0120FEF77CFD60BB1F4805
:10729000FEF750FD10BB2846BDE8F08104222B4BC1
:1072A0001A60AFE74FF0FF3118484FF00108FEF7C2
:1072B00039FD00283FF44BAF2548FEF7C3F9002005
:1072C000FEF760FD054600283FF448AF2148FEF771
:1072D000B9F943E7204D2846BDE8F0811F48FEF785
:1072E000B1F92846BDE8F0811D48FEF7ABF9CEE7BD
:1072F000102104F10800FFF7D3FDBEE7194D284621
:10730000BDE8F0814FF47305C5E700BFBC00002065
:107310001C198450201C8450041A8450181884505E
:1073200000198450CC1784505C1684505016845039
:107330004C1684501019845084168450281C845094
:107340002C1C845058168450D0178450C817845071
:10735000D48C0000EC8C00000100F3002C8D0000A8
:107360000C8D00000300F30000283AD02DE9F04115
:10737000D0E9062392FA82F893FA83FE026A436AFE
:10738000D0E9044112BA24BA1BBA04610262846AC9
:10739000826B4362C36BD0E9026509BA36BA2DBA73
:1073A000C76A8660C560066B456B416194FA84FCD0
:1073B00019BA14BA436C026C3FBA36BA2DBA12BA73
:1073C0001BBAC0E90C65C0E90E41C0F81880C0F8CE
:1073D0001CE0C0F828C0C762C0E910230020BDE847
:1073E000F0814FF47300704710B5044630B10022AD
:1073F0000123C4E91522C4E9173310BD0148FEF783
:1074000021F9F4E7E08D000018B174220021FFF7A4
:1074100045BD704788B199B110B50024802A8463B6
:1074200080F83C4006D1046310221030FFF734FD91
:10743000204610BD6FF01F0010BD6FF02100704797
:107440006FF01F00704700BF28B322B31BB30129A0
:1074500021D870B50446816B86B017D0012917D1A9
:10746000102500210DEB05066163104629460095A5
:1074700002AA0196FFF7ECFD50B92B463246204692
:1074800002A900F0EBF818B906B070BD0029E7D0EA
:107490006FF02100F8E76FF02100704700201870AE
:1074A000704700BF00284DD038B5044690F83C0026
:1074B000022816D003283DD0002830D02348244D80
:1074C0002A68244B126824491A602B68234A5C6896
:1074D000234B0C602968896811602A68D2681A6099
:1074E00038BD216B206C00F0CBFB194D0028E7D193
:1074F0002A68184B1068184918602868174A4068AD
:1075000008602968896811602A68D268DA60216B8E
:10751000206C00F0D9FB0028D2D1002038BD2169B1
:107520000C4A0D4B116061691960A1699160E269B3
:107530009A6038BD216B206C00F0B8FB0028BED1EA
:10754000034DD5E74FF47100704700BF0900F1000B
:10755000AC0000200014845004148450081484509B
:107560000C14845010B50446314A1368002BFCD12A
:10757000304A1368002BFCD12F4A1368002BFCD132
:107580002E4A1368002BFCD12D4A1368002BFCD126
:107590002C4A1368002BFCD14FF0FF30FEF71CFB88
:1075A000636B23F00403032BE36D36D0012B264BD2
:1075B00018680CBF20F0800020F02000FEF71AFBB6
:1075C0000121224B1A4A19601368002BFCD1194A79
:1075D0001368002BFCD11E49154A0B601368002B61
:1075E000FCD1144A1368002BFCD1626B22F0040119
:1075F000032918BFA36B4FEA820218BF03F00103EF
:10760000144902F01C0213430B60636B072B02D179
:107610000122114B1A60002010BD012B0A4B186883
:107620000CBF20F0400020F01000FEF7E3FAC7E79F
:107630001019845070148450201D8450201C8450D4
:10764000381D8450381C8450041A8450001984500A
:10765000BC148450C01484507C1484502DE9F04F25
:1076600087B0002900F0A5801646002A00F0A1800E
:107670000446002800F041811F46C36D0D46002BD3
:1076800050D1B7F5805F52D294F83C30042B00F013
:107690000B814FF000084FF0FF31A948FEF742FB85
:1076A000002840F0E0800020FEF76CFB002840F04E
:1076B000E3800121A34BA44A19601368002BFCD17D
:1076C000636B032B39DC002B3ADADFF8C8929E4A51
:1076D0001368002BFCD1B8F1000F40F0DC80636B25
:1076E00023F00403032BE36D58D0012B974B18684C
:1076F0000CBF40F0800040F02000FEF77BFA002233
:10770000904B01201A60FEF73DFB002840F0BF803F
:107710008B48FEF70FFB002840F0B280484607B0C8
:10772000BDE8F08F012BAFD1B7F5803FACD3DFF8C8
:107730006892484607B0BDE8F08F063B012BC4D8DD
:10774000A36B012B00F2D680E36D012B37D8236E9B
:10775000012B00F234812046FFF704FF8146002808
:10776000B5D12046FFF79EFE81460028AFD1636B5E
:10777000072BAAD801A252F823F000BFDB77000044
:10778000C577000037790000C5770000CB76000090
:10779000CB76000037790000C5770000012B6B4BDA
:1077A00018680CBF40F0400040F01000FEF722FACD
:1077B000A5E7DFF8E891484607B0BDE8F08FDFF8AD
:1077C000E09184E72168624A624B11606168196048
:1077D000A1689160E2689A60636B23F00403032B55
:1077E0002A6809D0216E3368012907BF5A485B49CE
:1077F0005B485C4903600F60E36D012B0BBF5A4B84
:107800005A4B5B495B490A601F60636B23F00403BA
:10781000032B75D0236E012B0CBF80202020FEF798
:10782000EFF9814600287FF452AF474B1A68002ACF
:10783000FCD1636B9146013B062B11D8DFE803F0C6
:1078400004BC041010BC0400414A424B11680832C9
:1078500021601968083361601268A2601B68E360E8
:107860000123A36533E74448FDF7ECFE0020FEF753
:1078700089FA00283FF41DAF4048FDF7E3FE18E702
:107880003F48FDF7DFFE484607B0BDE8F08F3D48B2
:10789000FDF7D8FE3CE70423202184F83C3004F1B6
:1078A0001000FFF7FDFA1AE7216B206C00F0D2F907
:1078B000E8B9DFF8F080DFF8F0B0D8F80030DFF892
:1078C000ECA01B68DFF8E890CBF80030D8F8003067
:1078D0002D4A5B68CAF80030D8F800309B68C9F8B8
:1078E0000030D8F80030DB681360216B71B14FF0C5
:1078F0000108D0E6DFF8BC90E9E64FF471090DE726
:10790000E36D012B0CBF4020102088E7D4E913322F
:107910000093102304F11000CDE90120039305909A
:10792000D4E91123206C00F04DFA00284AD100233D
:1079300084F83C30DBE72168144A154B45E700BF6B
:10794000BC0000201018845010198450041A845070
:107950004014845044148450281D84502C1D84509D
:10796000301D8450341D84502C1C8450341C845091
:10797000281C8450301C8450D48C0000EC8C0000F7
:107980002C8D00000C8D00000C1484506014845069
:10799000641484500100F1000500F1000B00F100B7
:1079A0000300F100AC000020001484500414845043
:1079B000081484500200F1000F4A104B46E7DFF82C
:1079C000449084E6D8F8003005981B680C4ACBF840
:1079D0000030D8F8003010215B68CAF80030D8F8C1
:1079E00000309B68C9F80030D8F80030DB681360BD
:1079F000FFF756FA9BE700BF60148450641484506C
:107A00000C1484500400F1002DE9F04101B3FAB1E7
:107A1000044600287AD01D46436B0E46072B1BD028
:107A20005DB9032B10D1836D73B9C0E91955C0E955
:107A30001B55102500F164030B602B463146204690
:107A4000BDE8F041FFF70ABE2F463846BDE8F08199
:107A5000684F3846BDE8F081C36D002B59D1B5F5AC
:107A6000805F5BD215B9A36D002B57D14FF0FF316A
:107A70006148FEF757F9002840F09A800020FEF791
:107A800081F9002840F0908001215C4B5C4A19602C
:107A90001368002BFCD1636B032B20DD063B012B0D
:107AA0001FD8A36B012B3BD8E36D012B00F288801C
:107AB000236E012B00F286802046FFF753FD074618
:107AC00080B92046FFF7EEFC074658B9636B072BD9
:107AD00007D8DFE803F03127552706065527002B86
:107AE000DFDA484F464A1368002BFCD1434A012095
:107AF0001360FEF747F900285ED13F48FEF71AF9F8
:107B00000028A2D04048FDF79DFD9EE74FF4710785
:107B10009BE7012BA6D1B5F5803FA3D33B4F94E75C
:107B20003B4FDFE721683B4A3B4B116061681960BE
:107B3000A1689160E2689A6001233849384A0B6075
:107B40001560002D40D1A26D0AB9364A13602C4B46
:107B50001F68002FFCD1636B013B062BC2D801A22A
:107B600052F823F0897B0000A37B0000897B000092
:107B7000E57A0000E57A0000A37B0000897B000025
:107B80002168294A294BD0E7224A234B1168083241
:107B900021601968083361601268A2601B68E360A5
:107BA000A0E7214A214BF1E72148FDF74BFD6BE7A8
:107BB0002048FDF747FD61E71F48FDF743FD9CE7BF
:107BC0001E4F8FE71E4F8DE7E26D3368012A0AD002
:107BD00010201C491C4A0B601560FEF711F807467F
:107BE0000028B4D07EE71949194A0B60402015607F
:107BF000F3E700BF0B00F100BC0000201018845018
:107C0000101984500100F1002C8D00000500F100D6
:107C10000200F10040148450441484507C148450B9
:107C2000BC1484502415845060148450641484500F
:107C3000EC8C0000D48C00000C8D00000300F100DF
:107C40000400F100301C8450341C8450281C8450E3
:107C50002C1C84507F280CD849B1032901D0064838
:107C6000704706497F280CBF084600207047084629
:107C700070470248704700BF0300F7000100F7009B
:107C8000831E7D2B0CD849B1032901D005487047CC
:107C900005497F280CBF08460020704708467047FA
:107CA000014870470300F7000100F70028B9044BB2
:107CB000002918BF19460846704702490846704710
:107CC0000300F7000100F700002858D009B133483D
:107CD000704730B40124324B324A84B0C2F80045B8
:107CE000C3F80811D3F8082105190292029AC3F8C3
:107CF0000011D3F8002180300292029AC3F80411D7
:107D0000D3F80411284A02910299C3F8005552F899
:107D10003010264A03910399914236D11A461C60CD
:107D200005E09DF80630DBB99DF80730C3B9D2F8FD
:107D30000031003B18BF01238DF80530D2F808311F
:107D4000003B18BF01238DF80630D2F80431003B08
:107D500018BF01238DF807309DF80530002BE0D0C7
:107D60009DF80630ABB99DF8073003F0FF0293B9D8
:107D700010460B4BC3F8002504B030BC70470122FD
:107D80000B490C4B08601A6070470B4804B030BCBC
:107D900070470A48F0E70A48EEE700BF0C00F10020
:107DA00000900350000084500080FF0000148450B5
:107DB000381A8450781484500600F7000100F70048
:107DC0000200F7002DE9F04F0024CDB00546DDE9B3
:107DD000589688461746214674220EA89B4600F006
:107DE00029FB214680222CA82B9400F023FB84231E
:107DF000B6F57F6FCDE90A44CDE90C4405935DD813
:107E000005AB0DF1AC0A01935946DDE9562338461E
:107E10000296CDF800A000F061F8002855D1A542E7
:107E20000CBF4FF0030C4FF0020C00220123072778
:107E3000012410211C900EA8CDE92423CDF86880E0
:107E40008DF874C01B971E952694FFF729F8102211
:107E50000DF120080092504605990AAB06AACDF80C
:107E60000480FFF7F5F80746C8B10EA87422002178
:107E7000FFF714F838464DB0BDE8F08F102E3546A8
:107E800028BF10250EA92A46FFF706F810210EA8D4
:107E9000FFF706F80134761B2F44E4B213D0059B9C
:107EA000424606A90EA88DF8AC40FFF7ADFD03468B
:107EB00009EB0700002BE1D01F46D6E7054F3846F7
:107EC0004DB0BDE8F08F3746CFE7034F38464DB091
:107ED000BDE8F08F0F00F1000E00F1002DE9F04138
:107EE000002682B00A9D0196B5F57F6F3BD8EE0063
:107EF000B6F5807F1F4634BF032304234D1E3F2D5C
:107F00000C4600932FD870B3904617B15AB3402F48
:107F100029D8089A3AB3099A116821B3E21913448F
:107F2000994220D3089B22460146581CFEF7B4FF15
:107F30000022089B23445A70023407BBFF2E009690
:107F400015D9089B3502ADB21819022245EA16254B
:107F500001A90195FEF7A0FF02340020099B1C60D7
:107F600002B0BDE8F0810A4802B0BDE8F081089B8C
:107F7000012218196946FEF78FFF0134EDE7089BCF
:107F8000414618193A46FEF787FF3C44D6E700BF42
:107F90000600008008B5F9F72FFEBDE80840F9F7A4
:107FA000CBBD034658B1426802F00302012A03D058
:107FB000032A04D1026812B10020986070476FF064
:107FC00015007047002070470FB407B504A951F899
:107FD000040B0191F8F7F2FA03B05DF804EB04B07A
:107FE0007047838B13F0070305D10368002B0CBF88
:107FF000002003207047022B05D1C38B002B14BF38
:10800000002004207047012B05D10368002B0CBF12
:10801000002005207047002070472DE9F0410D46F3
:1080200007461946281D90461E46F8F79BFA044657
:1080300038B13346424629463846A446BDE8F041A9
:108040006047BDE8F08110B50C4640B139B1081D5C
:10805000FFF7A7FF28B9A36833F0030301D06FF03F
:10806000150010BD38B50C46054658B151B10B6826
:1080700043B14B6833B12022002100F0DBF900202E
:108080002C6138BD6FF01500FBE7044608B50846C3
:1080900011461A46A047FCF735FFFAF75BFC2DE9BD
:1080A000F74F9946D37814466F2BA3F14102064649
:1080B0000F4601922DD028D8582B14BF0A25102521
:1080C000AA464FF0000BDDF8308052465B46304642
:1080D0003946F8F7B3F8092AD3B21FD830335F45D1
:1080E000DBB208BF564508F8013D01D3C84512D898
:1080F00023789B0605D5082D16D1A37843F00803F5
:10810000A370404603B0BDE8F08F03F0F703702B77
:10811000D3E70825D4E706460F46D6E7019A192A81
:1081200094BF37335733DAE7102DEAD1A37843F001
:108130001003E5E72DE9F0410746884615461E463F
:108140001446B442A4EB050002D33EB923782BB108
:10815000414614F8010BB8470028F2DABDE8F08177
:10816000404080F311884FF0040002DF70477047F1
:10817000FBF78CB884B004AB03E90700002383F35A
:108180001188BFF36F8F04B070470FB407B504A90F
:1081900051F8040B0191F8F711FA03B05DF804EB04
:1081A00004B070470022C0E900228260704710B519
:1081B0004FF02003EFF3118283F31188BFF36F8F29
:1081C000036803F00704012C06D10160002082F34C
:1081D0001188BFF36F8F10BD03F0C0038B4214BF33
:1081E0004FF0FF306FF07700F1E74FF02003EFF32F
:1081F000118283F31188BFF36F8F036803F0C0030C
:1082000043F00203036082F31188BFF36F8F70475E
:108210000069CBB200EB4310002110470020FBF7B0
:1082200055B90020FBF7A2B98022F9F741B91046F1
:10823000FBF700BF2DE9F0410C24C9B24C4305699E
:10824000064604F148008021284490461F46FFF767
:10825000AEFF002806DB2544C5E9108773681B596B
:1082600098470020BDE8F081704738B505460C46B8
:1082700051B96FF01500BDE838407146724673463B
:10828000F4468EF3008C744700F061F80128F0D1B9
:10829000204600F05CF80128EBD02846F9F792FD63
:1082A000014628B13C22204600F099F80020E2E780
:1082B0006FF00D00DFE7FEE700210120F9F7F0BFC6
:1082C000024643B20846C1B9002B27DB01205B09F7
:1082D0009B0003F1604303F56143D3F8801202F081
:1082E0001F02904021EA0001C3F88012D3F88002F7
:1082F000D04000F00100C0B27047002B0DDB01211F
:108300005B099B0003F1604303F56143D3F88002EE
:1083100002F01F0291400143E6E700207047436EE0
:1083200083F30B88704701460068F9F7B9BF08B5B9
:10833000F9F7E4FFBDE80840FAF7BCBA40E800F3FB
:1083400013F4803FD8B208BF6FF01500704740E8C3
:1083500000F0C0F380507047034600201A5C02B959
:1083600070470130FAE7034600201A5C0AB18842E0
:1083700000D170470130F8E7431E013913F8012F8F
:1083800011F8010F824201D1002AF7D1101A70476B
:1083900010B55AB10139841810F8012B11F8013FBA
:1083A000A04201D09A42F7D0D01A10BD1046FCE787
:1083B000431A934210B500EB020308D30246013979
:1083C0009A420BD011F8014F02F8014BF8E70A442A
:1083D00012F8014D8A4203F8014DF9D110BDF0B5F4
:1083E00081EA0004A50703460BD0013B0A449142F1
:1083F0001BD1F0BD002AFCD011F8014B013A03F863
:10840000014B9C07F6D122F003041D1F96080F199B
:10841000B94205D16FF00305234405FB0622E4E7CA
:1084200051F804CB45F804CFF2E711F8014B03F8FB
:10843000014FDCE7034670B5C9B29C0711D141EA90
:10844000012422F0030644EA04451E449408B34282
:108450000DD16FF0030505FB04221A44934209D1A4
:1084600070BD002AFCD003F8011B013AE5E743F890
:10847000045BECE703F8011BF0E74FF0FF307047B7
:1084800043681B68D3F80423D10518D5D3F82021FD
:10849000AAB14FF02001EFF3118281F31188BFF3ED
:1084A0006F8FD3F8201131B10021C3F82011D3F818
:1084B00020110121D96082F31188BFF36F8F4268C8
:1084C0005268D20615D54FF02001EFF3118281F3E7
:1084D0001188BFF36F8FD3F8581111B10021C3F881
:1084E00000154FF48001C3F8081382F31188BFF31D
:1084F0006F8F70470B460269D2E9010183E80300E0
:108500000020704743681B68D3F88004C3F88004D8
:10851000704742681368D3F8580140B9526812078F
:1085200006D4D3F82001003818BF0120704701207D
:108530007047436802691B68D3F8100148B10020F6
:10854000527C0A70C3F81001D3F8102101221A607E
:1085500070474FF0FF3070474368F7B51C68002341
:108560000769C4F800350B683860064601A80D4657
:108570000193FAF71DFD0123019A934083602B6854
:1085800001A80193FAF714FD0322019B803340F800
:1085900023206B685A1C08D001A80193FAF708FD44
:1085A0000C22019B803340F82320D5E90023C4F836
:1085B0000C25C4F81435AB68581C08D001A80193E9
:1085C000FAF7F6FC0C22019B803340F82320EB687D
:1085D000591C11D001A80193FAF7EAFC0123019A72
:1085E00093408360EB6801A80193FAF7E1FC032252
:1085F000019B803340F823203169D5E902323046AF
:10860000C4F808250431C4F81035FAF71BFC40BB48
:108610000823C4F800356B6801330BD0C4F810018F
:10862000D4F8103107F11103C4F834350123C4F82C
:1086300038352360736810375B681A075CBF4FF4E6
:108640008072C4F80423DB0644BF4FF48003C4F8EF
:1086500004330023C4F84475C4F848350123A360EB
:10866000E36003B0F0BDFCF7B9BF08B5F9F76EFCE5
:10867000F9F718FDBDE80840FCF7B0BF004700F06F
:1086800069B87047C3681888C0F30800A0F5807304
:108690005842584170474FF02002EFF3118382F3A4
:1086A0001188BFF36F8FFEE730B50024C46184608A
:1086B00041EA020414F00304C0E9033241610CD121
:1086C0008461A34203D1C0E90000002030BD856968
:1086D00001340D6081611144F3E76FF01500F5E797
:1086E000EFF30580003818BF012070470020704765
:1086F00008B5F8F713FEBDE80840FFF7B5BD03461F
:108700000020C3E90033C3E902007047034620B9E3
:10871000EFF305820AB9F9F7DBBC83F31188BFF3E5
:108720006F8F70474FF02003EFF3118083F31188B0
:10873000BFF36F8FFFF7EABF03460068834203D0A1
:10874000002838BF002070470020704708B5FCF7AC
:10875000FBFE08BD08B1F8F77BBD70477047FFFF0F
:108760000C7BFF7F010000002912000000000000C8
:108770007D39000000000000678600000000000056
:1087800051150000D000002009310000E800002051
:10879000D930000000010020B9310000180100208C
:1087A000DD1300000000000065190000300100200A
:1087B0006B86000000000000D531000000000000C2
:1087C00000000000B982000000000000B982000033
:1087D00000000000B982000000000000B982000023
:1087E00000000000B9820000393600007D860000DC
:1087F00000000000B982000000000000B982000003
:108800000001002081840000E80000208184000035
:1088100000000000B982000000000000B9820000E2
:1088200000000000B982000000000000B9820000D2
:1088300000000000B982000000000000B9820000C2
:1088400000000000B982000000000000B9820000B2
:1088500000000000B982000000000000B9820000A2
:1088600000000000B982000000000000151900009F
:1088700000000000B982000000000000B982000082
:1088800000000000B982000000000000B982000072
:1088900000000000B982000000000000B982000062
:1088A00000000000B982000000000000B982000052
:1088B00000000000B982000000000000B982000042
:1088C00000000000B982000000000000B982000032
:1088D00000000000B982000000000000B982000022
:1088E00000000000B982000000000000B982000012
:1088F00000000000B982000000000000B982000002
:1089000000000000B982000000000000B9820000F1
:1089100000000000B982000000000000B9820000E1
:1089200000000000B982000000000000B9820000D1
:1089300000000000B982000000000000B9820000C1
:1089400000000000B982000000000000B9820000B1
:1089500000000000B982000000000000B9820000A1
:1089600000000000B982000000000000B982000091
:1089700000000000B982000000000000B982000081
:1089800000000000B982000000000000B982000071
:1089900000000000B982000000000000B982000061
:1089A00000000000B982000000000000B982000051
:1089B00000000000B982000000000000B982000041
:1089C00000000000B9820000FB8E000003000000E0
:1089D0007698000003000000989B00000300000050
:1089E000A58E0000030000007C8E00000300000044
:1089F0007599000001000000FF7FFF7FFF7FFF7F70
:108A0000FF7FFF7FFF7FFF7FFF7FFF7FFF7FFF7F76
:108A1000FF7FFF7FFF7FFF7FFF7FFF7FFF7FFF7F66
:108A2000FF7FFF7FFFFFFFFFFFFFFFFFFFFFFFFF56
:108A3000DEE61E284CBBCE8F025B00001D0000004E
:108A40001C0000001A0000001B00000001000000D4
:108A5000000000000F0000000E000000DEE61E28EF
:108A6000EAAC45B8025B0000DEE61E284CBBCE8FA8
:108A7000025B000000000000000000000000000099
:108A80000338FDD870470000C51600002982000099
:108A900035820000000000007D1400003D1600003B
:108AA000A1160000EF8E00001D820000238200004E
:108AB000F58E0000311400002915000000000000B0
:108AC0003B910000420100004291000005010000BE
:108AD0004C910000140100005591000015010000A8
:108AE0005E9100003901000067910000090100005B
:108AF000729100000A0000007D9100000A01000050
:108B0000879100000B010000919100000F0100000F
:108B10009C91000010010000A791000011010000CD
:108B2000B29100000E010000BC9100002101000084
:108B3000C591000022010000CE9100002301000039
:108B4000D791000024010000E0910000180100000E
:108B5000E89100002A010000F09100003A010000B5
:108B6000F89100002C010000009200001C010000A0
:108B7000099200001D010000129200001701000080
:108B80001C920000040100002B920000260100004E
:108B900033920000280100003B92000031010000E8
:108BA00000000000000200000004000000080000B7
:108BB0000010000000000000B7820000E51F000068
:108BC0009D1F000055200000591F000020000020BC
:108BD0000800002018000020000000001000002005
:108BE000000000200000000006000100020000005C
:108BF000F48B0000000000002C990000060000002B
:108C0000E0FF0F0000000020349900002100000068
:108C1000E0FF0020338500001530000005850000CE
:108C2000452E0000F5840000008000500300000085
:108C300000900050030000003931000000000000E7
:108C400068870000A8870000B0870000C087000088
:108C5000C0870000F5FFFFFF499B0000579B000005
:108C60006B9B00007A9B0000869B0000FF8FFFFF3C
:108C7000FF8FFFFFFE8FFFFFFE8FFFFFFD8FFFFFC8
:108C8000FC8FFFFFFC8FFFFF6D757465785F667268
:108C900065652063616C6C65642077697468204E3B
:108CA000554C4C20706172616D65746572000000F6
:108CB00043616E277420696E697469616C697A65B5
:108CC000206D757465782C20776173204E554C4C5F
:108CD0000D0A00004661696C20746F206163717534
:108CE000697265206D757465780A00004661696C6B
:108CF00020746F20696E63726561736520504D202A
:108D0000636F756E7465720A000000004661696CDD
:108D100020746F20646563726561736520504D2017
:108D2000636F756E7465720A000000004661696CBD
:108D300020746F2072656C65617365206D75746554
:108D4000780A0000436F756C64206E6F74206C6F3E
:108D5000636B20706F7765722073617665206D7527
:108D6000746578004661696C20746F20756E6C6F55
:108D7000636B206D757465780A0000000A6374786F
:108D8000206973204E554C4C0A00000001234567B2
:108D900089ABCDEFFEDCBA9876543210F0E1D2C345
:108DA000D89E05C107D57C3617DD703039590EF7CE
:108DB000310BC0FF11155868A78FF964A44FFABE94
:108DC00067E6096A85AE67BB72F36E3C3AF54FA55C
:108DD0007F520E518C68059BABD9831F19CDE05B88
:108DE0006374782063616E6E6F74206265204E55E7
:108DF0004C4C00574553545F544F504449522F7ABE
:108E000065706879722F6C69622F6F732F6E6F7443
:108E10006966792E6300415353455254494F4E20A1
:108E20004641494C20402025733A25640A005745A5
:108E300053545F544F504449522F7A657068797289
:108E40002F6C69622F6F732F6F6E6F66662E6300D3
:108E5000574553545F544F504449522F7A657068B8
:108E600079722F696E636C7564652F7370696E6CAF
:108E70006F636B2E6800286E696C2900736F630046
:108E8000574553545F544F504449522F7A65706888
:108E900079722F7375627379732F706D2F706F777E
:108EA00065722E6300706F77657200554152545F92
:108EB0003000574553545F544F504449522F7A6500
:108EC000706879722F647269766572732F636C6F44
:108ED000636B5F636F6E74726F6C2F636C6F636B29
:108EE0005F636F6E74726F6C5F6E72662E63006884
:108EF00066636C6B006C66636C6B00636C6F636BBA
:108F00005F636F6E74726F6C00574553545F544FBC
:108F1000504449522F7A65706879722F647269766D
:108F20006572732F74696D65722F7379735F636CEB
:108F30006F636B5F696E69742E63007379735F632F
:108F40006C6F636B005365637572650909004E6F42
:108F50006E2D5365637572650900574553545F5410
:108F60004F504449522F6E72662F73756273797336
:108F70002F73706D2F73706D2E6300253032752046
:108F800025303275203078253035782030782530FE
:108F9000357820090025630053504D3A204E532068
:108FA000696D61676520617420307825780A005307
:108FB000504D3A204E53204D53502061742030784C
:108FC00025780A0053504D3A204E53207265736540
:108FD0007420766563746F72206174203078257810
:108FE0000A0053504D3A20707265706172652074AA
:108FF0006F206A756D7020746F204E6F6E2D5365F3
:109000006375726520696D6167652E0A004E6F6E2B
:109010002D53656375726500466C617368207265D7
:1090200067696F6E730909446F6D61696E09095054
:1090300065726D697373696F6E730A005745535497
:109040005F544F504449522F6D6F64756C65732F98
:1090500068616C2F6E6F726469632F6E7266782F11
:1090600068616C2F6E72665F7370752E68004E6F4C
:109070006E2D7365637572652063616C6C61626CE3
:109080006520726567696F6E203020706C61636562
:109090006420696E20666C61736820726567696F11
:1090A0006E20256420776974682073697A652025AD
:1090B000642E0A00436F756C64206E6F7420696EB5
:1090C000697469616C697A6520736563757265207E
:1090D00073657276696365732028657272202564F2
:1090E000292E0A005352414D20726567696F6E093F
:1090F00009446F6D61696E09095065726D6973731A
:10910000696F6E730A005065726970686572616C90
:109110000909446F6D61696E09095374617475734F
:109120000A002530327520252D3231732573000950
:10913000534B49500A00094F4B0A004E52465F50AC
:1091400030004E52465F434C4F434B004E52465FF9
:1091500052544330004E52465F52544331004E52F7
:10916000465F4E564D43004E52465F554152544560
:1091700031004E52465F554152544532004E5246E0
:109180005F5457494D32004E52465F5350494D335C
:10919000004E52465F54494D455230004E52465F94
:1091A00054494D455231004E52465F54494D455247
:1091B00032004E52465F5341414443004E52465F97
:1091C00050574D30004E52465F50574D31004E5271
:1091D000465F50574D32004E52465F50574D330058
:1091E0004E52465F574454004E52465F495043002A
:1091F0004E52465F564D43004E52465F4650550014
:109200004E52465F45475531004E52465F454755E1
:1092100032004E52465F4450504943004E52465F22
:10922000524547554C41544F5253004E52465F50A1
:10923000444D004E52465F493253004E52465F47FE
:1092400050494F544531006D757465785F696E699A
:10925000742063616C6C65642077697468204E5576
:109260004C4C20706172616D6574657200436F755E
:109270006C64206E6F7420616C6C6F636174652028
:109280006D75746578206265666F726520696E69B8
:109290007469616C697A696E6700574553545F540D
:1092A0004F504449522F7A65706879722F6172630A
:1092B000682F61726D2F636F72652F6161726368D1
:1092C00033322F6972715F6D616E6167652E630065
:1092D00025633A2072302F61313A202030782530D2
:1092E0003878202072312F61323A202030782530B2
:1092F0003878202072322F61333A202030782530A0
:1093000038780A0025633A2072332F61343A2020DE
:10931000307825303878207231322F69703A202029
:10932000307825303878207231342F6C723A202012
:109330003078253038780A0025633A202078707319
:10934000723A20203078253038780A0025633A2098
:109350004661756C74696E6720696E7374727563AB
:1093600074696F6E20616464726573732028723152
:10937000352F7063293A203078253038780A002557
:10938000633A202A2A2A2A2A204D50552046415540
:109390004C54202A2A2A2A2A0A0025633A2020200F
:1093A000537461636B696E67206572726F722028F7
:1093B000636F6E746578742061726561206D696792
:1093C0006874206265206E6F742076616C69642910
:1093D0000A0025633A202020556E737461636B691F
:1093E0006E67206572726F720A0025633A20202032
:1093F00044617461204163636573732056696F6CC7
:109400006174696F6E0A0025633A2020204D4D4635
:10941000415220416464726573733A203078257834
:109420000A0025633A202020496E737472756374B4
:10943000696F6E204163636573732056696F6C6159
:1094400074696F6E0A0025633A202020466C6F61B4
:1094500074696E672D706F696E74206C617A792003
:109460007374617465207072657365727661746976
:109470006F6E206572726F720A00574553545F54C5
:109480004F504449522F7A65706879722F61726328
:10949000682F61726D2F636F72652F6161726368EF
:1094A00033322F636F727465785F6D2F6661756CF0
:1094B000742E630025633A202A2A2A2A2A2042553C
:1094C00053204641554C54202A2A2A2A2A0A00258C
:1094D000633A202020537461636B696E6720657264
:1094E000726F720A0025633A20202050726563690A
:1094F0007365206461746120627573206572726F98
:10950000720A0025633A20202042464152204164DD
:1095100064726573733A20307825780A0025633ABF
:10952000202020496D7072656369736520646174E1
:109530006120627573206572726F720A0025633A4A
:10954000202020496E737472756374696F6E206297
:109550007573206572726F720A0025633A202A2A99
:109560002A2A2A205553414745204641554C54202C
:109570002A2A2A2A2A0A0025633A202020446976CA
:109580006973696F6E206279207A65726F0A0025AF
:10959000633A202020556E616C69676E6564206DAA
:1095A000656D6F7279206163636573730A0025636B
:1095B0003A202020537461636B206F766572666C6D
:1095C0006F772028636F6E746578742061726561AF
:1095D000206E6F742076616C6964290A0025633AF5
:1095E0002020204E6F20636F70726F636573736FFE
:1095F0007220696E737472756374696F6E730A009A
:1096000025633A202020496C6C6567616C206C6F83
:109610006164206F66204558435F52455455524E51
:1096200020696E746F2050430A0025633A20202081
:10963000496C6C6567616C20757365206F6620747A
:10964000686520455053520A0025633A2020204186
:109650007474656D707420746F20657865637574BB
:109660006520756E646566696E656420696E7374E5
:1096700072756374696F6E0A0025633A202A2A2A7C
:109680002A2A20534543555245204641554C5420E3
:109690002A2A2A2A2A0A0025633A202020416464C3
:1096A000726573733A20307825780A0025633A2072
:1096B0002020496E76616C696420656E7472792031
:1096C000706F696E740A0025633A202020496E7617
:1096D000616C696420696E7465677269747920735E
:1096E00069676E61747572650A0025633A202020EF
:1096F000496E76616C696420657863657074696F22
:109700006E2072657475726E0A0025633A202020FF
:109710004174747269627574696F6E20756E6974D4
:109720002076696F6C6174696F6E0A0025633A2058
:109730002020496E76616C6964207472616E736971
:1097400074696F6E0A0025633A2020204C617A7993
:1097500020737461746520707265736572766174CC
:10976000696F6E0A0025633A2020204C617A7920C7
:109770007374617465206572726F720A005265734A
:10978000657276656420457863657074696F6E20D4
:10979000280053707572696F757320696E746572F5
:1097A000727570742028495251200025633A202098
:1097B000205320696E737472756374696F6E2061D3
:1097C0006464726573733A2020307825780A002526
:1097D000633A202A2A2A2A2A204841524420464114
:1097E000554C54202A2A2A2A2A0A0025633A202086
:1097F00020427573206661756C74206F6E207665EB
:1098000063746F72207461626C6520726561640AB2
:109810000025633A2020204661756C7420657363CF
:10982000616C6174696F6E20287365652062656C78
:109830006F77290A0025633A202A2A2A2A2A2044F7
:1098400065627567206D6F6E69746F7220657863ED
:10985000657074696F6E202A2A2A2A2A0A002563F5
:109860003A202A2A2A2A2A20257320256429202AF8
:109870002A2A2A2A0A006D70750025633A2046615B
:10988000696C656420746F20616C6C6F63617465D2
:10989000206E6577204D505520726567696F6E2088
:1098A00025750A0A0025633A20506172746974694B
:1098B0006F6E2025753A2073616E69747920636834
:1098C00065636B206661696C65642E0A0025633AE6
:1098D00020496E76616C696420756E6465726C797E
:1098E000696E6720726567696F6E20696E6465785E
:1098F0002025750A00574553545F544F5044495230
:109900002F7A65706879722F617263682F61726D4A
:109910002F636F72652F616172636833322F6D70D0
:10992000752F61726D5F6D70752E6300464C4153EB
:10993000485F30005352414D5F3000574553545FEC
:10994000544F504449522F6D6F64756C65732F6886
:10995000616C2F6E6F726469632F6E7266782F6808
:10996000616C2F6E72665F6770696F2E680055417B
:1099700052545F3100756172745F6E7266785F7504
:109980006172746500574553545F544F50444952B7
:109990002F6E72662F647269766572732F656E74AE
:1099A000726F70792F656E74726F70795F63633355
:1099B00031302E630043525950544F43454C4C00B4
:1099C0004552524F523A2043616E6E6F7420667555
:1099D0006C66696C6C204558545F41504920726533
:1099E00071756573742E0D0A005741524E494E47EA
:1099F0003A204F7074696F6E616C204558545F4116
:109A000050492072657175657374206E6F7420669D
:109A1000756C66696C6C65642E0D0A00574553546D
:109A20005F544F504449522F6D6F64756C65732FAE
:109A300068616C2F6E6F726469632F6E7266782F27
:109A400068616C2F6E72665F636C6F636B2E68006B
:109A5000574553545F544F504449522F6D6F6475AE
:109A60006C65732F68616C2F6E6F726469632F6E03
:109A70007266782F647269766572732F7372632FC2
:109A80006E7266785F636C6F636B2E630025633A5A
:109A90002048616C74696E672073797374656D0A10
:109AA00000556E6B6E6F776E206572726F72007507
:109AB0006E6B6E6F776E0025633A203E3E3E205AF5
:109AC000455048595220464154414C204552524F2E
:109AD000522025643A202573206F6E204350552074
:109AE00025640A0025633A204661756C742064750C
:109AF00072696E6720696E74657272757074206821
:109B0000616E646C696E670A0A0025633A204375CA
:109B10007272656E74207468726561643A20257093
:109B200020282573290A00574553545F544F504449
:109B300049522F7A65706879722F6B65726E656C09
:109B40002F666174616C2E63004350552065786305
:109B5000657074696F6E00556E68616E646C6564E3
:109B600020696E7465727275707400537461636BF2
:109B7000206F766572666C6F77004B65726E656CF0
:109B8000206F6F7073004B65726E656C2070616E34
:109B90006963006D61696E006F7300574553545FD0
:109BA000544F504449522F7A65706879722F6B6513
:109BB000726E656C2F6D656D5F736C61622E6300F4
:109BC000574553545F544F504449522F7A6570683B
:109BD00079722F6B65726E656C2F74687265616443
:109BE0002E6300574553545F544F504449522F7AC7
:109BF00065706879722F6B65726E656C2F6D757408
:109C000065782E6300574553545F544F5044495272
:109C10002F7A65706879722F6B65726E656C2F692B
:109C20006E636C7564652F6B73636865642E680082
:109C3000574553545F544F504449522F7A657068CA
:109C400079722F6B65726E656C2F73656D2E630074
:109C5000574553545F544F504449522F7A657068AA
:109C600079722F6B65726E656C2F73636865642EF5
:109C70006300574553545F544F504449522F7A65FF
:109C8000706879722F6B65726E656C2F74696D6583
:109C90006F75742E630076322E362E302D7263313E
:109CA0002D6E637331002A2A2A20426F6F74696E09
:109CB00067205A6570687972204F53206275696C0D
:109CC00064202573202573202A2A2A0A0000000018
:109CD00000000000C57F00000100000048010020D6
:109CE000010000005C010020010000007001002064
:109CF0000100000084010020010000007B840000BE
:109D00000000000000C2010000010300000000008C
:109D1000000000000000000000C20100000103007C
:109D200000000000000000000090D0035800002058
:109D3000580000200000000021560000180E0020EE
:109D4000010000007D570000595700009D5700009A
:109D500039570000A4000020680000209C0000206B
:109D600000000000940000201C0E002001000000F4
:109D7000200E002001000000240E00200100000041
:109D8000280E002084000020900000208800002081
:109D900080000020B8000020095E0000155E000071
:109DA000215E0000469100009C8A0000888A000025
:109DB000BC020020D00200201A8A00006E99000028
:109DC000308C0000148C0000340A00204000002079
:109DD000108A0000AB8E0000288C0000148C00005C
:109DE000380A00202C000020068A0000B5990000E7
:109DF00000000000388C00003C0A00200000000039
:109E0000FE8900003B8F0000000000000000000001
:109E10003003002000000000F88900004801002005
:109E20004801002000000000000000000F000000BA
:109E30005C0100205C010020000000000000000028
:109E40000F000000700100207001002000000000E1
:109E5000000000000F0000008401002084010020A9
:109E600000000000000000000F000000FFFFFFFFE7
:109E7000FFFFFFFFFFFFFFFFFFFFFFFFFFFFFFFFF2
:109E800000000000000000000000000000000000D2
:109E900000000000000000000000000000000000C2
:109EA00000000000000000000000000000000000B2
:10FFE0007FE97FE9F8F741B97FE97FE9F1F74CBF95
:10FFF0007FE97FE9F1F76CBF7FE97FE9F1F70EBF99
:020000040001F9
:10000000F0940220694C020047950500A54C0200BF
:10001000A54C0200A54C0200A54C0200A54C020014
:100020000000000000000000000000009D480200E9
:10003000A54C020000000000054802000545020032
:10004000294C0200294C0200294C0200294C0200D4
:10005000294C0200294C0200294C0200294C0200C4
:10006000294C0200294C0200294C0200294C0200B4
:10007000294C0200294C0200294C0200294C0200A4
:10008000294C0200294C0200294C0200294C020094
:10009000294C0200294C0200294C0200294C020084
:1000A000294C0200294C0200294C0200294C020074
:1000B000D527040029D70500294C0200294C02004D
:1000C000294C0200294C0200294C0200294C020054
:1000D000294C0200294C0200294C0200294C020044
:1000E000294C0200294C0200294C0200294C020034
:1000F000294C0200294C0200294C0200294C020024
:10010000294C0200294C0200294C0200294C020013
:10011000294C0200294C0200294C0200294C020003
:10012000294C0200294C0200294C0200294C0200F3
:10013000294C0200294C0200294C0200294C0200E3
:10014000294C020000000000000000000000000038
:10015000000000000000000000000000000000009F
:10016000000000000000000000000000000000008F
:10017000000000000000000000000000000000007F
:10018000000000000000000000000000000000006F
:10019000000000000000000000000000000000005F
:1001A000000000000000000000000000000000004F
:1001B000000000000000000000000000000000003F
:1001C000000000000000000000000000000000002F
:1001D000000000000000000000000000000000001F
:1001E000000000000000000000000000000000000F
:1001F00000000000000000000000000000000000FF
:10020000DEE61E284CBBCE8F025B00003C000000E7
:10021000844307000100000000000100000001000D
:10022000FFFF02910000000000000000000000003D
:10023000000000000000000000000000FFFFFFFFC2
:1002400081F0004102E000BF83F0004330B54FEA87
:1002500041044FEA430594EA050F08BF90EA020FF4
:100260001FBF54EA000C55EA020C7FEA645C7FEA87
:10027000655C00F0E2804FEA5454D4EB5555B8BFAA
:100280006D420CDD2C4480EA020281EA030382EA1B
:10029000000083EA010180EA020281EA0303362DAD
:1002A00088BF30BD11F0004F4FEA01314FF4801C80
:1002B0004CEA113102D0404261EB410113F0004F92
:1002C0004FEA03334CEA133302D0524263EB430349
:1002D00094EA050F00F0A780A4F10104D5F1200EE7
:1002E0000DDB02FA0EFC22FA05F2801841F1000142
:1002F00003FA0EF2801843FA05F359410EE0A5F116
:1003000020050EF1200E012A03FA0EFC28BF4CF046
:10031000020C43FA05F3C01851EBE37101F00045FC
:1003200007D54FF0000EDCF1000C7EEB00006EEB09
:100330000101B1F5801F1BD3B1F5001F0CD3490893
:100340005FEA30004FEA3C0C04F101044FEA4452EA
:1003500012F5800F80F09A80BCF1004F08BF5FEA71
:10036000500C50F1000041EB045141EA050130BD51
:100370005FEA4C0C404141EB0101013C28BFB1F563
:10038000801FE9D291F0000F04BF01460020B1FAAE
:1003900081F308BF2033A3F10B03B3F120020CDA81
:1003A0000C3208DD02F1140CC2F10C0201FA0CF05F
:1003B00021FA02F10CE002F11402D8BFC2F1200CC4
:1003C00001FA02F120FA0CFCDCBF41EA0C0190407A
:1003D000E41AA2BF01EB0451294330BD6FEA0404C3
:1003E0001F3C1CDA0C340EDC04F11404C4F12002AE
:1003F00020FA04F001FA02F340EA030021FA04F3C0
:1004000045EA030130BDC4F10C04C4F1200220FA16
:1004100002F001FA04F340EA0300294630BD21FA54
:1004200004F0294630BD94F0000F83F4801306BF1A
:1004300081F480110134013D4EE77FEA645C18BF0E
:100440007FEA655C29D094EA050F08BF90EA020FA5
:1004500005D054EA000C04BF1946104630BD91EA9D
:10046000030F1EBF0021002030BD5FEA545C05D1A0
:100470004000494128BF41F0004130BD14F58004DF
:100480003CBF01F5801130BD01F0004545F0FE4153
:1004900041F470014FF0000030BD7FEA645C1ABF88
:1004A000194610467FEA655C1CBF0B46024650EABF
:1004B000013406BF52EA033591EA030F41F40021EB
:1004C00030BD00BF90F0000F04BF0021704730B571
:1004D0004FF4806404F132044FF000054FF0000146
:1004E00050E700BF90F0000F04BF0021704730B507
:1004F0004FF4806404F1320410F0004548BF4042DC
:100500004FF000013EE700BF42004FEAE2014FEA30
:1005100031014FEA02701FBF12F07F4393F07F4F0B
:1005200081F06051704732F07F4208BF704793F00E
:100530007F4F04BF41F40021704730B54FF4607421
:1005400001F0004521F000411CE700BF50EA010224
:1005500008BF704730B54FF000050AE050EA0102CD
:1005600008BF704730B511F0004502D5404261EB3D
:1005700041014FF4806404F132045FEA915C3FF47E
:10058000D8AE4FF003025FEADC0C18BF03325FEA1B
:10059000DC0C18BF033202EBDC02C2F1200300FACC
:1005A00003FC20FA02F001FA03FE40EA0E0021FAF1
:1005B00002F11444BDE600BF70B54FF0FF0C4CF4DF
:1005C000E06C1CEA11541DBF1CEA135594EA0C0F91
:1005D00095EA0C0F00F0DEF82C4481EA030621EACC
:1005E0004C5123EA4C5350EA013518BF52EA033507
:1005F00041F4801143F4801338D0A0FB02CE4FF0B9
:100600000005E1FB02E506F00042E0FB03E54FF0E8
:100610000006E1FB03569CF0000F18BF4EF0010EE0
:10062000A4F1FF04B6F5007F64F5407404D25FEADC
:100630004E0E6D4146EB060642EAC62141EA55518F
:100640004FEAC52040EA5E504FEACE2EB4F1FD0CD1
:1006500088BFBCF5E06F1ED8BEF1004F08BF5FEA4F
:10066000500E50F1000041EB045170BD06F0004601
:1006700046EA010140EA020081EA0301B4EB5C04AE
:10068000C2BFD4EB0C0541EA045170BD41F48011A6
:100690004FF0000E013C00F3AB8014F1360FDEBFCB
:1006A000002001F0004170BDC4F10004203C35DAA7
:1006B0000C341BDC04F11404C4F1200500FA05F32A
:1006C00020FA04F001FA05F240EA020001F00042CB
:1006D00021F0004110EBD37021FA04F642EB060141
:1006E0005EEA430E08BF20EAD37070BDC4F10C046B
:1006F000C4F1200500FA04F320FA05F001FA04F22F
:1007000040EA020001F0004110EBD37041F100011A
:100710005EEA430E08BF20EAD37070BDC4F1200525
:1007200000FA05F24EEA020E20FA04F301FA05F28D
:1007300043EA020321FA04F001F0004121FA04F235
:1007400020EA020000EBD3705EEA430E08BF20EA05
:10075000D37070BD94F0000F0FD101F0004640003F
:1007600041EB010111F4801F08BF013CF7D041EAC1
:10077000060195F0000F18BF704703F000465200C5
:1007800043EB030313F4801F08BF013DF7D043EA96
:100790000603704794EA0C0F0CEA135518BF95EA4C
:1007A0000C0F0CD050EA410618BF52EA4306D1D1D3
:1007B00081EA030101F000414FF0000070BD50EAF2
:1007C000410606BF1046194652EA430619D094EA7C
:1007D0000C0F02D150EA013613D195EA0C0F05D166
:1007E00052EA03361CBF104619460AD181EA0301BA
:1007F00001F0004141F0FE4141F470014FF0000072
:1008000070BD41F0FE4141F4780170BD70B54FF00C
:10081000FF0C4CF4E06C1CEA11541DBF1CEA13558C
:1008200094EA0C0F95EA0C0F00F0A7F8A4EB05046E
:1008300081EA030E52EA03354FEA013100F0888065
:100840004FEA03334FF0805545EA131343EA12632E
:100850004FEA022245EA111545EA10654FEA0026E3
:100860000EF000419D4208BF964244F1FD0404F59C
:10087000407402D25B084FEA3202B61A65EB0305F8
:100880005B084FEA32024FF480104FF4002CB6EBB5
:10089000020E75EB030E22BFB61A754640EA0C0035
:1008A0005B084FEA3202B6EB020E75EB030E22BF75
:1008B000B61A754640EA5C005B084FEA3202B6EBB6
:1008C000020E75EB030E22BFB61A754640EA9C0075
:1008D0005B084FEA3202B6EB020E75EB030E22BF45
:1008E000B61A754640EADC0055EA060E18D04FEA03
:1008F000051545EA16754FEA06164FEAC30343EAA3
:1009000052734FEAC2025FEA1C1CC0D111F4801F6F
:100910000BD141EA00014FF000004FF0004CB6E768
:1009200011F4801F04BF01430020B4F1FD0C88BF07
:10093000BCF5E06F3FF6AFAEB5EB030C04BFB6EB12
:10094000020C5FEA500C50F1000041EB045170BD05
:100950000EF0004E4EEA113114EB5C04C2BFD4EB32
:100960000C0541EA045170BD41F480114FF0000EB6
:10097000013C90E645EA060E8DE60CEA135594EA32
:100980000C0F08BF95EA0C0F3FF43BAF94EA0C0F35
:100990000AD150EA01347FF434AF95EA0C0F7FF4AA
:1009A00025AF104619462CE795EA0C0F06D152EAFE
:1009B00003353FF4FDAE1046194622E750EA4106E2
:1009C00018BF52EA43067FF4C5AE50EA41047FF4F3
:1009D0000DAF52EA43057FF4EBAE12E74FF0FF3C58
:1009E00006E000BF4FF0010C02E000BF4FF0010C29
:1009F0004DF804CD4FEA410C7FEA6C5C4FEA430CA2
:100A000018BF7FEA6C5C1BD001B050EA410C0CBFF0
:100A100052EA430C91EA030F02BF90EA020F002052
:100A2000704710F1000F91EA030F58BF994208BFB9
:100A300090422CBFD8176FEAE37040F00100704776
:100A40004FEA410C7FEA6C5C02D150EA013C07D1CD
:100A50004FEA430C7FEA6C5CD6D152EA033CD3D018
:100A60005DF8040B704700BF8446104662468C4612
:100A70001946634600E000BF01B5FFF7B7FF002845
:100A800048BF10F1000F01BD4DF808EDFFF7F4FF6E
:100A90000CBF012000205DF808FB00BF4DF808EDF9
:100AA000FFF7EAFF34BF012000205DF808FB00BF1C
:100AB0004DF808EDFFF7E0FF94BF012000205DF83E
:100AC00008FB00BF4DF808EDFFF7CEFF94BF0120F3
:100AD00000205DF808FB00BF4DF808EDFFF7C4FFEC
:100AE00034BF012000205DF808FB00BF4FEA410C35
:100AF0007FEA6C5C02D150EA013C0AD14FEA430C18
:100B00007FEA6C5C02D152EA033C02D14FF0000054
:100B100070474FF0010070474FEA410212F5001292
:100B200015D211D56FF47873B3EB625212D94FEA34
:100B3000C12343F0004343EA505311F0004F23FA1E
:100B400002F018BF404270474FF00000704750EA73
:100B5000013005D111F0004008BF6FF00040704730
:100B60004FF00000704700BF4FEA4102B2F1E0438E
:100B700024BFB3F5001CDCF1FE5C0DD901F0004C84
:100B80004FEAC0024CEA5070B2F1004F40EB8300D4
:100B900008BF20F00100704711F0804F21D113F100
:100BA0003872BCBF01F00040704741F480114FEA39
:100BB0005252C2F11802C2F1200C10FA0CF320FAC2
:100BC00002F018BF40F001004FEAC1234FEAD323DF
:100BD00003FA0CFC40EA0C0023FA02F34FEA430349
:100BE000CCE77FEA625307D150EA01331EBF4FF0D2
:100BF000FE4040F44000704701F0004040F0FE40ED
:100C000040F40000704700BF80F0004002E000BFE9
:100C100081F0004142001FBF5FEA410392EA030FE7
:100C20007FEA226C7FEA236C6AD04FEA1262D2EB31
:100C30001363C1BFD218414048404140B8BF5B4236
:100C4000192B88BF704710F0004F40F4000020F0CF
:100C50007F4018BF404211F0004F41F4000121F0E5
:100C60007F4118BF494292EA030F3FD0A2F101022F
:100C700041FA03FC10EB0C00C3F1200301FA03F16D
:100C800000F0004302D5494260EB4000B0F5000F90
:100C900013D3B0F1807F06D340084FEA310102F14F
:100CA0000102FE2A51D2B1F1004F40EBC25008BF01
:100CB00020F0010040EA03007047490040EB0000CB
:100CC000013A28BFB0F5000FEDD2B0FA80FCACF1CC
:100CD000080CB2EB0C0200FA0CF0AABF00EBC250F9
:100CE00052421843BCBFD0401843704792F0000FE7
:100CF00081F4000106BF80F400000132013BB5E73A
:100D00004FEA41037FEA226C18BF7FEA236C21D0AF
:100D100092EA030F04D092F0000F08BF0846704714
:100D200090EA010F1CBF0020704712F07F4F04D1E2
:100D3000400028BF40F00040704712F100723CBFF5
:100D400000F50000704700F0004343F0FE4040F41F
:100D5000000070477FEA226216BF08467FEA2363DD
:100D60000146420206BF5FEA412390EA010F40F4C8
:100D7000800070474FF0000304E000BF10F0004314
:100D800048BF40425FEA000C08BF704743F09643FB
:100D900001464FF000001CE050EA010208BF704716
:100DA0004FF000030AE000BF50EA010208BF70479D
:100DB00011F0004302D5404261EB41015FEA010CB2
:100DC00002BF84460146002043F0B64308BFA3F1AA
:100DD0008053A3F50003BCFA8CF2083AA3EBC2538C
:100DE00010DB01FA02FC634400FA02FCC2F12002AB
:100DF000BCF1004F20FA02F243EB020008BF20F0E2
:100E00000100704702F1200201FA02FCC2F1200247
:100E100050EA4C0021FA02F243EB020008BF20EA3C
:100E2000DC7070477BB972B90029BEBF00204FF05B
:100E3000004106E008BF00281CBF6FF000414FF0E2
:100E4000FF3000F0EDB9ADF1080C6DE904CE0029DA
:100E500009DB002B1ADB00F083F8DDF804E0DDE9A4
:100E6000022304B07047404261EB4101002B1BDBC1
:100E700000F076F8DDF804E0DDE9022304B040423A
:100E800061EB4101524263EB43037047524263EB13
:100E9000430300F065F8DDF804E0DDE9022304B067
:100EA000404261EB41017047524263EB430300F063
:100EB00057F8DDF804E0DDE9022304B0524263EBA9
:100EC0004303704753B94AB9002908BF00281CBF23
:100ED0004FF0FF314FF0FF3000F0A2B9ADF1080C38
:100EE0006DE904CE00F03CF8DDF804E0DDE9022312
:100EF00004B0704738B50022002304460D46FFF7C2
:100F0000CDFD28B920462946BDE8384000F00AB892
:100F1000204605F1004100F005F8404261EB410137
:100F200038BD00BFD0B500220B4B06460F46FFF779
:100F300043FB00F077F90446FFF7C4FA0022074BA1
:100F4000FFF73AFB02460B4630463946FFF77CF97D
:100F500000F068F92146D0BD0000F03D0000F041EE
:100F60002DE9F047089D04468846002B7DD18A4232
:100F700017463FD9B2FA82F242B1C2F12000914045
:100F8000974024FA00F0944040EA01084FEA174CD9
:100F9000230C1FFA87FEB8FBFCF60CFB168106FB40
:100FA0000EF043EA0143984205D9FB1802D2984259
:100FB00000F22481013E191AA3B2B1FBFCF00CFB34
:100FC000101100FB0EFE43EA0144A64505D93C1969
:100FD00002D2A64500F20F81013840EA0640A4EB98
:100FE0000E0400261DB1D4400023C5E9004331465C
:100FF000BDE8F08702B9FFDEB2FA82F2002A50D1D2
:10100000CB1B4FEA174E1FFA87F80126210CB3FBC2
:10101000FEFC0EFB1C300B4608FB0CF941EA0041BC
:1010200089450AD979182CBF01230023894502D9A3
:10103000002B00F0D9800CF1FF3CA1EB0901A3B219
:10104000B1FBFEF00EFB101108FB00F843EA01446F
:10105000A04505D93C1902D2A04500F2C98001384B
:10106000A4EB080440EA0C40BCE78B4209D9002DF0
:1010700000F0B1800026C5E9000130463146BDE8E8
:10108000F087B3FA83F6002E46D18B42C0F0A680DB
:10109000824240F2A3803046002DA8D0C5E9004826
:1010A000A5E79740C2F1200301FA02F04FEA174E7C
:1010B000D94024FA03F31FFA87F894400343B1FBA5
:1010C000FEF01E0C0EFB101100FB08FC46EA01416D
:1010D0008C4509D979182CBF012600268C4502D9E8
:1010E000002E00F093800138A1EB0C019BB2B1FB04
:1010F000FEF60EFB161106FB08FC43EA01418C4587
:1011000005D9791802D28C4500F28780013EA1EB07
:101110000C0346EA004679E7C6F1200703FA06F415
:1011200002FA06FC01FA06FEFA4020FA07F8F94036
:1011300000FA06F3224348EA0E044FEA12484FEA47
:10114000144E1FFA82F9B1FBF8FA08FB1A110AFBD8
:1011500009F04EEA014E70450AD912EB0E0E2CBF73
:1011600001210021704501D9002952D00AF1FF3A2E
:10117000AEEB000EA4B2BEFBF8F008FB10EE00FBD5
:1011800009F944EA0E4EF14505D912EB0E0E01D2D3
:10119000F14538D8013840EA0A40AEEB090EA0FB11
:1011A0000C89CE4541464C4602D306D1434504D274
:1011B0000138B8EB0C0169EB020415B35A1A6EEB57
:1011C000040EF2400EFA07F72EFA06F30026174334
:1011D000C5E900730BE72E46284608E7841A61EB41
:1011E00003010120884657E7ACF1020C394424E79B
:1011F00002383C4434E702383C44EEE6023E3B44CD
:10120000D9E62E46F3E602389644C4E7023839445C
:101210006AE7AAF1020A9644AAE7023E394476E751
:10122000704700BF4A0011D212F5001211D20DD53D
:101230006FF47873B3EB62520ED44FEAC12343F0DC
:10124000004343EA505323FA02F070474FF0000086
:10125000704750EA013002D14FF0FF3070474FF035
:101260000000704710F8012B11F8013B012A28BF3C
:101270009A42F7D0D01A7047034613F8012B002A80
:10128000FBD1181A013870472DE9F047A4B04FF090
:10129000FF324FF0FF33A0483EF062F9DFF8C8821A
:1012A0009E4C9F480023D822214600684EF0D5F975
:1012B0000028234605DC00214FF480403FF060FF0A
:1012C000EEE72278022A00F00481032A00F052811E
:1012D000012AE5D198F80030022B14D1914D2868ED
:1012E00088B1914B1B784BB114A90BF04DFA8F4884
:1012F00000218F4A006814AB46F083FF00232B6067
:101300000BF02AFACCE7DFF864A29AF80030002B41
:1013100000F0C38094F84430844D864F864E13F01D
:10132000010F14BF3B4633460021844A286846F02B
:1013300068FF94F84430002113F0020F14BF3B46BD
:1013400033467F4A286846F05CFF94F84430002119
:1013500013F0040F14BF3B4633467A4A286846F020
:1013600050FF94F84430002113F0080F14BF3B469F
:101370003346754A286846F044FF94F84430734A6F
:1013800013F0100F14BF3B4633460021286846F087
:1013900038FF94F84430A946DA074BD5238E6C4ABF
:1013A000059394F82E300021049394F82D30039384
:1013B00094F82C300293238D019394F82A300093F3
:1013C000286894F82B3046F01CFF206CFFF79CF83F
:1013D000CDE91201E06BFFF797F8CDE91001A06BA2
:1013E000FFF792F8CDE90E01606BFFF78DF8CDE9BC
:1013F0000C01606AFFF788F8CDE90A01206AFFF75F
:1014000083F8CDE90801E069FFF77EF8CDE9060130
:10141000A069FFF779F8D4E90423CDE90401CDE907
:101420000223D4E90223CDE900230021494A286898
:1014300046F0E7FE9AF80030012B2ED90026374DF2
:10144000DFF82CA1B5F8467017B395F85030C3F308
:10145000C002C3F340030692059395F84830049305
:10146000B5F94E300393B5F94C300293B5F84A0004
:10147000FFF738F826A3D3E90023FFF79DF8CDE95D
:1014800000013B4652460021D9F8000046F0B9FE63
:1014900001360C2E05F10C05D4D198F80030022B42
:1014A0007FF4FEAE94F84430DB077FF5F9AE4EF0E2
:1014B0009AFA4FF47A730A46A0FB030103FB021168
:1014C000184AC30B43EA4143234813603EF0DCFC57
:1014D000E6E6224A1278002A3FF4E2AE002203F147
:1014E000080111F8010B0D2801D00A280AD1134474
:1014F00000221A720D480021194B1A4A006846F062
:1015000080FECDE60132532AEBD1F3E7AFF3008042
:101510009A9999999999B93FE876012060890120B3
:10152000B46A0120B8A301201B05022088A2012073
:10153000D1F106007BCD060080CD0600F1F106005A
:101540000AF2060022F206003AF2060052F2060003
:101550006AF2060099F20600188801201E05022092
:1015600068890120A67D06001F050220177301204F
:1015700042F306002E4B1B78002B3FF491AE4EF049
:1015800032FA4FF47A75A0FB052305FB0133D00B2B
:1015900040EA434014A90BF0F7F8002326698DF8C0
:1015A000603016F0010F18AD04D0302228462149D2
:1015B0004EF00FFFB70704D5302228461E494EF0E3
:1015C00008FF700704D5302228461C494EF001FF61
:1015D000310704D53022284619494EF0FAFEF206AA
:1015E00004D53022284617494EF0F3FEB30604D541
:1015F0003022284614494EF0ECFE2846FFF73CFE08
:1016000080B9284611494EF009FFE368104801935C
:10161000A3680295009300210E4A006814AB46F0BF
:10162000F0FD3DE624AB1844002300F8333CECE722
:101630001B0502208BF3060092F306009AF30600C6
:10164000A1F30600A9F30600B0F30600B7F3060005
:1016500088A20120BCF3060001282DE9F0470D46C1
:1016600009D004283AD047F0BDFF162303604FF09D
:10167000FF30BDE8F0871E4B9E68D3E900484EF06E
:10168000B2F90B461B4FA0FB070107FB031116A382
:10169000D3E900234FEAD03949EA41494FEAD13A28
:1016A00048465146FFF70EFC0FA3D3E90023041967
:1016B00041EB080848465146C5E90048FFF702FCDF
:1016C0000D4B32449A42AA6006D9013448F1000118
:1016D000C5E90041D21BAA600020CAE700263446B3
:1016E000B046CCE7AFF3008000CA9A3B0000000090
:1016F000208D012000CA9A3BFFC99A3B00000000E0
:10170000012870B50C4606D047F06CFF1623036025
:101710004FF0FF3070BD4EF066F90E46184D22684E
:101720006168A2FB052305FB0133A168521843EB56
:10173000E173A0FB050105FB0611C40B44EA41441B
:10174000141B4FEAD13563EB050520460AA3D3E904
:1017500000232946FFF766FB07A3D3E90023094EC0
:10176000C6E9000120462946FFF75CFB0020B26075
:10177000D0E700BFAFF3008000CA9A3B0000000032
:1017800000CA9A3B208D01202DE9F04F00272DED56
:10179000028B08EE902A0122044608EE101ABB467E
:1017A0003D46BA463E469A4B87B01A60002318EE73
:1017B000901A009318EE100A964B974A48F0E9FAEF
:1017C000431C0BD12178632940F01083BAF1000F3C
:1017D00000F012830322914B1A6000E3013876284F
:1017E00000F28D80DFE810F00A01D502DF02E3028B
:1017F000EA010A01DB028B000A010A012B028B00BD
:101800008B008B008B00E702EF02690239028B002C
:101810004B016D028B00B6028B008B008B008B009E
:101820008B008B008B008B008B008B008B008B0060
:101830008B008B008B008B008B008B008B008B0050
:101840008B008B008B008B00CF00C1018B000B0243
:101850008B0010028B008B008B008B008B008B00A9
:101860008B008B008B008B000A01E4010A01C90088
:101870008B0084028B008B00A202D7008B000A0130
:10188000F60107027902AA018B00B6011402980240
:101890008B00D3008B003F028B005F028B008B001C
:1018A0008B008B008B008B008B002401F7009E02C5
:1018B0008B0085008B008B00A1008B009B01A40195
:1018C000F70292018B0077008B008B00EC00860101
:1018D0000401DB00CB01524B18684EF052F94FF671
:1018E000FE73421E9A4202D91A224C4B06E06064F3
:1018F0005CE74B4B1B682BB91822484B1A604FF022
:10190000FF306CE21B78D4F8B82182F8603023F005
:101910002003473BDBB20D2BEED842F2510222FAF4
:1019200003F3DA073FF542AFE6E73D4B18684EF0A8
:1019300025F935A3D3E9002359EC108B84ED3C0B3A
:1019400084ED3A0B10EE100A4946FFF7A7F840B9AC
:10195000002240464946334BFFF7BEF800283FF4CB
:1019600025AF0022002340464946FFF78DF80028A6
:101970007FF41CAF0922294BC0E70123C4F88C3047
:101980004FF0010A12E70123C4F89030F8E7012371
:10199000C4F8A0300AE70123C4F8A43006E716F023
:1019A0001DF903901AF016FB02901AF017FBDDE9FF
:1019B000023200901C491D4842F082FD00200EE2D8
:1019C0002378632B02D10122144B97E77321204621
:1019D00048F09AFBEAE62378732BF4D02046632183
:1019E00048F092FB0E4B2046196848F0A5FBDDE657
:1019F0000221204616F040FC0125D7E60D22074BB8
:101A00007CE700BFAFF300809A9999999999B93F03
:101A1000446D0120646D0120D22D07004CCF0120C0
:101A200034CF012000004E40456007004F2D0700D5
:101A3000B34D2F2128684EF0E4FC90B1002300F84C
:101A4000013BD4F8B8814EF09CF8D4F8B831C8F80E
:101A50003C00DB6B013BB3F57A7F02D30F22A94B2D
:101A60004CE7286802F094FA51EC100BFFF75AFA91
:101A7000D4F8B8514FF0010BC5E90401BCE7DFF819
:101A800080A22F21DAF800004EF0BBFC28B300231F
:101A900000F8013BD4F8B8814EF070F888ED080BDF
:101AA000D4F8B8310022D3E90889002340464946DA
:101AB000FEF7EAFF88B990A3D3E9002340464946E0
:101AC000FEF7ECFF30B90022404649468E4BFFF747
:101AD00003F810B11C228B4B10E7DAF8000002F07B
:101AE00057FA51EC100BFFF71DFAD4F8B881C8E98A
:101AF000060145E7824B18684EF043F8834BE064DB
:101B0000984240F3718105227E4BF7E67C4BD4F876
:101B1000B85118681AF006FEC5E914016CE7784B55
:101B2000D4F8B85118681AF0FDFDC5E9160163E74D
:101B3000734B18681AF0F6FD06465DE7704B18689F
:101B40004EF01FF88028C4F848017FF755AF0622F1
:101B50006C4BD3E6D4F89C3013B11922694BCDE617
:101B60000121204648F0EFFA46E7D4F89830002BE0
:101B7000F3D10125FF23C4F89C50637016E6604B37
:101B800018681AF083FD59EC108B002210EE100A31
:101B900049465F4BFEF7A0FF10B10822594BADE656
:101BA00040464946FEF7B8FFD4F8B851686023E7CD
:101BB000534B18684BF048FDE061F7E5504B18684F
:101BC0004DF0DFFF4FF6FE73421E9A423FF68CAE99
:101BD0002064EBE54A4BD4F8B85118684DF0D1FFBA
:101BE000D4F8B83128641B6CB3F5105F7FF704AFED
:101BF0000A22444B82E60125C4F89450D6E501221E
:101C0000D4F8B8311A60D1E50222D4F8B831F9E736
:101C10003B4D0022286805A9D4F8B88143F09EFE08
:101C20002B68059AC8F848009A4205D0D4F8B83114
:101C30009B6CFF2B7FF6E0AE1522324B5EE6304BFD
:101C4000D4F8B851186816F07FFAD4F8B831A864FF
:101C50009B6C002BBFF6D0AEEEE7294B18684BF01B
:101C6000F3FC2066C8E6102041F028FC804610B93D
:101C70008B22244B42E6102200214EF05FF8204BCD
:101C800018684BF0E1FCC8F800000028F0D00023F1
:101C9000C8F80830E36B08F10800C8F80C30C3F846
:101CA0000080E06382E548F073FF10B90B22154B0A
:101CB00024E60125C4F8A85078E50125C4F8C050F1
:101CC00074E50123C4F8C4300D4B196819B12046DE
:101CD00048F012FA6AE50F49F9E7094B18684DF028
:101CE00050FF3C28A0647FF687AE0C22054B05E62A
:101CF000034B1B68236559E59A9999999999B93FBE
:101D000034CF01204CCF012000004E408051010013
:101D10000000C041642D0700864B18684BF094FC0E
:101D2000E06569E60123C4F8AC303FE5DFF80482E2
:101D3000D8F800004BF088FCC4F8CC0000287FF4F1
:101D400035ADD8F800107C4845F02AFB4FF4977267
:101D50007A4BD3E5DFF8DC8105A90022D8F8000032
:101D600043F0FCFDD8F80010059B8B4201D0002801
:101D700003DA734845F014FBC1E508464BF064FCF8
:101D8000C4F8D00000287FF411ADD8F800106D48D9
:101D9000DAE7684B18684BF057FC606706E50123EB
:101DA000C4F8B83002E50125C4F8B050FEE40123C0
:101DB000C4F8B430FAE45F4B18681AF0B3FCD4F8F6
:101DC000B831986318E65B4B18681AF0ABFCD4F88E
:101DD000B831986610E616F02DFA6FF0010007B0E2
:101DE000BDEC028BBDE8F08F012705E6732903D116
:101DF00015B10422514BEFE4E3681B6846BB022B8C
:101E000005D00C2B40F6D45608BF4FF48036D4F8DA
:101E1000B851AE60BBF1000F07D1022B14BF0022F6
:101E20004FF480120023C5E90423D5E9148958EA48
:101E3000090371D1D5E9162313436DD10022424B1A
:101E400001F0EF0163291A600BD002223B4BC3E47F
:101E5000022B52D0721EB2F5801FD8D30722374B07
:101E6000BAE4D5E908670022002330463946FEF778
:101E70000BFEC8B9D4E93A89304642464B4639464A
:101E8000FEF716FE78BB42464B4630463946FEF713
:101E9000BDFC41EC100B40F069FB51EC100BFEF760
:101EA0003BFED4F8B8319862D4F8A430002B3FF44C
:101EB00085ADD4F8B83193F86030612B15D1D4F8E2
:101EC000A0303BB1214816F0CBF9D4F8A430002B58
:101ED0003FF474ADD4F8AC30002B3FF46FAD1C4828
:101EE00016F0BEF96AE50120DBE71A4816F0B8F9EA
:101EF000D4F8A430002BE2D160E5B6F5801FADDC4C
:101F0000002E84DD4FF6D372A6F1100595427FF6C0
:101F10007EAF1422094B5FE447B90023E36458EA1B
:101F200009038BD0D5E91623134387D01022034B26
:101F300052E400BF34CF0120682D07004CCF0120B0
:101F4000942D0700A92D0700446D0120312E0700B4
:101F5000692E0700FB2D07002DE9F04F2DED028BB8
:101F600003780446732B87B010D1C06F16F016F9B2
:101F7000054670B97522A24B1A60D4F8AC3013B183
:101F8000A04842F09DFA4FF0FF3681E016F056FA75
:101F9000EEE79D4947F0E3FF9C498146284647F01C
:101FA000DEFF9B498046284647F0D9FF99490746FE
:101FB000284647F0D4FFD4F8AC300646B9F1000FFC
:101FC00004D0B8F1000F01D007B148B975218C4A8F
:101FD000116013B1904842F073FA4FF0FF364BE0B6
:101FE00053B1284647F0A7FF824601468B4842F08E
:101FF00067FA504616F0A2F8D9E90823C4E94C2341
:10200000D8E90823C4E94E23D7E90823C4E95023BB
:1020100094F90130B2698BB9C4E90123284680499B
:1020200047F09DFF824668B9D4F8AC3013B17D48C3
:1020300042F046FA7522724B1A60CEE7013308BFB0
:10204000A260EBE74FF0000947F07BFF4E469FEDA3
:102050006A8B0390039B994520DB2378632B0BD17C
:10206000D4F8B03043B128466F4947F0A9FF0028A3
:1020700000F09280C4F8E80128466C4947F06FFFF1
:1020800018B100694BF0E0FAE066284615F0BCFD97
:10209000304607B0BDEC028BBDE8F08F4946504694
:1020A00047F057FF074670B97522554B1A60D4F8B0
:1020B000AC3023B94FF0FF3609F10109CAE75C489B
:1020C00042F0FEF9F6E75B4947F049FF5A490590AF
:1020D000384647F044FF59498346384647F03FFFAA
:1020E00057490090384647F03AFF56490190384624
:1020F00047F035FF54490490384647F030FF5349C4
:102100000290384647F02BFF51498046384647F049
:1021100026FF059A4AB15B463BB1009B2BB1019B60
:102120001BB1049B0BB1029941B97522344B1A6063
:10213000D4F8AC30002BBDD04648C1E79769D4F83D
:10214000B4211AB9D0222E4B1A60B3E71169B942F3
:102150002FD0D2F8B020F4E701999B6991ED087B6C
:10216000136682ED127BC2F83CE063465A46C7E92B
:102170000023B8F1000F09D040B1D8E90823D0E915
:102180000801FEF761F8C7E91C0195E787ED1C8B94
:1021900092E787ED1A8B8FE728462F4947F0DFFE3D
:1021A00000283FF469AF00694BF04EFAC4F8E4012F
:1021B00062E70299D769D1F818E05169DBE906BCFA
:1021C0000029C9D1009B59469B69C2F83CE0624690
:1021D000FB62C7E90212B8F1000FDAD00028D8D0AC
:1021E000D8E90823D0E90801FEF72EF8C7E91A015B
:1021F00062E700BFAFF300800000000000000000B5
:102200004CCF0120072F0700252F0700342F070090
:10221000422F0700522F0700692F0700872F070062
:10222000972F07009F2F07001C3007004230070040
:10223000BD2F0700DA4D0700561208005D2F07007A
:10224000DB2F0700DCAD0700E22F0700EA2F0700B5
:10225000F52F0700FE2F07002F30070000000000B9
:102260002DE9F04F0FF2DC29D9E900892DED0E8B15
:1022700000230446D3B0D0F8B4A1DFF8D0B216934F
:10228000BAF1000F0DD1169B002B41D1D4F8AC3020
:1022900013B1A14842F014F953B0BDEC0E8BBDE868
:1022A000F08FDAF81C30DB6F5B681D686DB320AA15
:1022B00005F1100105F1080048F042FB20A801F0EB
:1022C0004BFED4F8AC3057EC106B3BB12B6810EEE2
:1022D000102A009358463B4642F0F2F8D4E93A01FE
:1022E00042464B46FEF768F932463B46FEF7E0FBB6
:1022F00018B9D5E90023134307D0D4F8AC3013B193
:10230000864842F0DDF801231693DAF8B0A0B7E76B
:10231000D4F8A430002B00F0EE8015F003FF8246C5
:102320000028B9D00146D4F8DC0147F01BFE15F0B7
:10233000EDFE0CEE100A0028AED002467849504659
:1023400047F012FE94F901305A1C40F0D7802378F0
:10235000632B0CBF4FF0FF3300231C93169B08BF69
:10236000002316939FED6AAB169B1C9A934293DB56
:102370006C4A24AB5168106803C31189927A1980A2
:102380009A701C9B5B43189394F90130013340F021
:10239000B880654A1899654B2078002918BF134604
:1023A0006349644A632818BF0A460021CDE9003218
:1023B0002AA82022604B4DF0ADFF0023B0EE4AEA80
:1023C000F0EE6AEACDE91A33D4F8B4B11993179351
:1023D0001D93BBF1000F40F0BB80D4F84831012BB6
:1023E00004DCD4F8A430002B00F05583D4F8B451A9
:1023F000002D00F05083DDE91A01EB6942AEDB6F7E
:102400004AAF5B68D3F800B0FEF7A0F88046894673
:10241000412249EC108B2021304601F011FEDBF8FF
:102420001800FEF771F802460B4640464946FEF793
:10243000EDF9D4F8B83141EC100B93F8602041EC81
:102440001B0B2021384601F0FBFDE86920AA0BF1A7
:1024500008014C3048F074FA20A801F07DFDE869CD
:1024600020AA0BF110014C3059EC108B48F068FA9F
:1024700020A801F071FDE368D4F8A4201B68B0EE39
:10248000408AF0EE608A012B1E9202D00C2B40F0A5
:102490005B836368012B40F00283189B002B00F0E4
:1024A000FE821E9BDBF84020002B00F0E182189B8F
:1024B000CDE90A231D9B1946DA1713460A4651EC4B
:1024C0001B0BCDE9082300221C4BFEF775F81A9B65
:1024D000CDE9060104931B9B0593DBF81800FEF77A
:1024E00013F88DED008B42464B46CDE902011448AE
:1024F00048F0A3FAF3E20CEE10AA23E716931C931C
:1025000030E700238DF8A8308DF8903055E700BFF4
:102510000000000000000000DD370700C73707009B
:10252000972F0700053B07009B3707009E370700E2
:10253000779D0700B49C0700033807000000204087
:10254000983A07009A9999999999B93FA137070044
:10255000DBF81430189A934240F07682B44A27ABE5
:102560005168106803C31189927A19809A7094F99E
:10257000013001332AD1AF4A1899AF4B2078002996
:1025800018BF1346AD49AE4A632818BF0A4600215A
:10259000CDE900324AA82022AA4B4DF0BBFEDBF861
:1025A0001C00C36F5B681D68B5B92046A64918F0CA
:1025B000C5FDDBF81C30DB6F5B681B68002B40F04F
:1025C0002F822046A14918F0B9FD65E600238DF859
:1025D00028318DF89C30E2E7D4F8A43005F10808E2
:1025E000FBB9D4F8B4319B451BD141464C3048F07F
:1025F00095F9002840F0C580E3681B68012B02D0E4
:102600000C2B40F0B3806268D4F89C30012A40F073
:10261000A880002B00F0A3808D4A20468D4916F03B
:10262000D1FCD5E90001FDF791FF412241EC100BEF
:10263000202132A801F004FD95ED068AB5EEC08A8E
:10264000F1EE10FA40F3A480D5E90001FDF77EFF1A
:10265000064618EE100A0F46FDF756FF02460B46D7
:1026600030463946FEF7D2F841EC1D0BD4F8B831AC
:102670000DF1E80993F86020B0EE4D0AF0EE6D0A16
:102680002021484601F0DCFCDBF81C00414622AA70
:102690004C3048F055F922A801F05EFCDBF81C0034
:1026A00022AA05F110014C30B0EE408AF0EE608AAB
:1026B00048F046F922A801F04FFCE368B0EE409ADA
:1026C000F0EE609A1B68D4F8A480012B02D00C2B8A
:1026D00040F0F0806368012B40F08380DBF8143019
:1026E000002B7ED0286DB8F1000F56D0DBF80C60BF
:1026F00015932B6CC1171493AA6EF717D317CDE956
:1027000012236A6ED317CDE910232A6ECDE90C018E
:10271000D317CDE90E23AA6C51EC1D0BD317CDE9CD
:102720000A2300224C4BFDF747FFCDE90801D5E90C
:102730000023CDE90623A869FDF7E6FE8DED029B97
:10274000CDE904018DED008B32463B46434848F00D
:1027500074F901461CEE100A47F004FC29E7404AD0
:102760005BE70BB13F4A58E73F4A56E794F901301F
:10277000012B01D13D4A50E70BB93D4A4DE73D4A97
:102780004BE7D4F84831012B7FF74BAF3A4A44E787
:10279000B0EE4ADAF0EE6ADA68E7FDF7A3FE42AE81
:1027A00041EC100B41222021304601F049FCA96C7C
:1027B000324B2D6C3248DBF80C20002D08BF03464D
:1027C0008DED029B8DED008BCDE907633AAB069151
:1027D00005932C4932AB04934AAB204616F0F2FB2A
:1027E000E7E6DBF80C20296CB8F1000F4ED0DBF8DF
:1027F00014301646CDE90A13D71751EC1D0B0022F1
:10280000154BFDF7D9FECDE90801D5E90023CDE947
:102810000623A869FDF778FE8DED029BCDE9040142
:102820008DED008B32463B46174848F006F990E79D
:10283000053B07009B3707009E370700779D070081
:10284000B49C0700033807000B3807005F3A070005
:102850006A590700DC580600000020404238070093
:1028600028590700B758070088580700C95B0700B8
:10287000E55A07003B5B07006C5A0700C25C070083
:10288000CD190700EC580700E6380700A048A14B17
:102890008DED029B002908BF034606933AAB0593D2
:1028A00032AB04938DED008B20469B494AAB16F06A
:1028B00089FB7EE62A6CDBF81430EE69DBF80C70DD
:1028C0001E92002B3AD0B8F1000F22D0B8464FEA42
:1028D000E7790D930C9251EC1D0B00228F4BF717EB
:1028E000CDE90A67FDF768FECDE90801D5E90023C7
:1028F000CDE90623A869FDF707FE8DED029BCDE922
:1029000004018DED008B42464B46854848F095F812
:102910001FE77F4A1E997F4B8DED020B002908BFF0
:102920001346CDE9076327ABCDE9059332AB04939A
:102930008DED008B3A467B494AAB4EE76B6A002E21
:102940001F934BDD1846FDF7CDFD0022764BFDF7BA
:1029500033FE41EC1B0B3046FDF7C4FD02460B462F
:1029600051EC1B0BFDF752FF41EC1B0BD5E90C01A1
:1029700000226E4BFDF720FEB8F1000F33D000238C
:1029800013931E9BB84612931F9B4FEAE779F717E4
:10299000CDE90E67DF171A463B46CDE90A01CDE9BE
:1029A0000C2351EC1D0B00225C4B8DED10BBFDF791
:1029B00003FECDE90801D5E90023CDE90623A86986
:1029C000FDF7A2FD8DED029BCDE904018DED008B9D
:1029D00042464B46564848F030F8BAE6B0EE4ABA9E
:1029E000F0EE6ABAC2E74B4A1E9D494BCDE906019B
:1029F000002D18BF13460C931F9B8DED0ABB089347
:102A00003AAB059332AB04938DED029B8DED008BB9
:102A10003A462046474909964AAB16F0D3FAC8E52C
:102A20001A98D3E9002182181A921B9A41EB0202EC
:102A30001B92E2681268012A09D16268012A03D157
:102A40001D9A9B6C1A441D92DBF8B0B0C1E4DA69A0
:102A50001799114417915A6A199911441991D3E998
:102A60000C2351EC1E0BFDF7F1FB41EC1E0BEBE7C9
:102A70002749284B8DED028B002A08BF0B46079390
:102A80001D9B2046CDE90573CDE900892A490496AE
:102A90002AAA16F097FA1C9B01331C9364E41E9B30
:102AA000D4F8E4200BB3189B51EC1B0BCDE90823A1
:102AB00000221A4BFDF780FD1A9BCDE90601049315
:102AC0001B9B0593DBF81800FDF71EFD8DED008BB9
:102AD000CDE9020142464B46184847F0AEFF024698
:102AE0001749504647F040FAD5E70949094B8DEDA3
:102AF000028B002A08BF0B462046CDE90573CDE9BD
:102B00000089104904962AAA16F05CFAC3E700BFB0
:102B1000CD190700C25C07004C5807000000204098
:102B20004A390700975B07000000594000408F407A
:102B3000BB3907009F5A0700F05D0700F238070015
:102B4000013B0700B45D0700189BD4F8E450002B4C
:102B50003AD01E9B0BB3189BCDE90A53179B19461D
:102B6000DA1713460A4651EC1B0BCDE90823002265
:102B7000524BFDF721FD1A9BCDE9060104931B9BE7
:102B80000593DBF81800FDF7BFFC8DED008BCDE958
:102B9000020142464B464A48AAE44A4B4A4A8DED56
:102BA000020B002D14BF1D461546179B20460793A8
:102BB00024ABCDE90573CDE9008944490895049615
:102BC0002AAA16F0FFF966E7D4F84801FDF78AFC57
:102BD0000B46024651EC1E0BFDF718FE179B0646EE
:102BE000002B0F4648DD1998FDF77CFC0022384B7E
:102BF000FDF7E2FC41EC190B1798FDF773FC024658
:102C00000B4651EC190BFDF701FE41EC190B314B52
:102C1000002230463946FDF7CFFC1E9B8BB30023C4
:102C2000CDE91053179BCDE90801DE171A4633464C
:102C3000CDE90C23199B51EC1B0BDE171A463346CA
:102C4000CDE90A2300221D4B8DED0E9BFDF7B4FC50
:102C50001A9BCDE9060104931B9B0593DBF8180032
:102C6000FDF752FC8DED008BCDE9020142464B464B
:102C7000194847F0E2FE32E7B0EE4A9AF0EE6A9A5F
:102C8000C5E7104A104BCDE90601002D14BF1546CB
:102C90001D46179B8DED0A9B0993199B8DED028BA9
:102CA00008934AAB059342AB2046CDE900890B4916
:102CB0000C9504932AAA16F085F9ECE60000204052
:102CC00056390700C25C0700CD190700725E070085
:102CD0000000594000408F40C73907002C5E0700B4
:102CE0002DE9F04700F1100104460122C06F88B0C1
:102CF0000AF0D8FB002805DC0CBF6D227022A64B21
:102D00001A601FE094F910300233122B00F23A815E
:102D1000DFE813F01B011801380163001E003801C1
:102D200038013801380138013801130023000C0143
:102D30003801FF00030138011E00204616F0A4FBF5
:102D4000002802DA4FF0FF30C6E0D4F8C8310BB9E2
:102D50000020C1E020469847FAE794F901104B1C87
:102D600006D10121204647F015FD0028EADB0021AD
:102D7000204647F00FFD0028E4DBE3681B68022BC8
:102D800002D0D4F8B4510DBB0026D4F8B451DFF80A
:102D900024A204F1DC0804F1E009002DD8D0EB688E
:102DA00041461846059346F052F949460746E868F9
:102DB00046F04DF93246CDE9007051462046059B5C
:102DC00016F000F90136D5F8B050E6E7E8680121C1
:102DD00019F050FBD5F8B050D5E7D4F8AC301BB1A2
:102DE000E16F6E4841F06CFB0121E06F19F042FB8E
:102DF000204615F0DFFD0028A4DB06A847F07DFD86
:102E0000002802DA6522644B7AE70023E26CC4E909
:102E10004333C4F8043192B1C4F808310293A36C6F
:102E20005F491A445F4B06A882FB0323CDE90023C8
:102E3000224619F083FBC4F804010028E2D0D4E94B
:102E40003A670022002330463946FDF71DFEA8B937
:102E500001233046029339464DA3D3E90023FDF701
:102E6000ABFBFEF747F82246CDE900014E4906A824
:102E700019F064FBC4F80C010028C3D0D4E93C6706
:102E80000022002330463946FDF7FEFDA8B9012394
:102E90003046029339463EA3D3E90023FDF78CFB6D
:102EA000FEF728F82246CDE90001404906A819F0AE
:102EB00045FBC4F810010028A4D0A36C7BB9C4F86A
:102EC0000031C4F8E43094F90130002B3FF440AFF6
:102ED000204615F09FFDC01708B0BDE8F08706A892
:102EE00047F00BFD00288DDB0123C4F8E4300023FC
:102EF0000293A26C2B4B2E4982FB032306A8CDE93B
:102F00000023224619F01AFBC4F800010028DAD188
:102F100078E7204647F076F9DDE7D4F8CC310BB1FD
:102F200020469847204617F015FF11E778221A4BE4
:102F300020461A600E232374D4F8FC3098470B23E4
:102F40002374FFE67922144BDAE601230422E06FB2
:102F500006A947F0D1FD00280F4D02DA6C232B6043
:102F6000F0E6069B04221BBA2B60E06F012306A942
:102F700047F0C2FD0028F1DB069B1CBA46F032FB8D
:102F80000460DFE66E22044BBAE600BFAFF30080B8
:102F90000000000080842E414CCF0120BB40070080
:102FA0006BA7050040420F0075A7050085A7050027
:102FB000F5AB02008F40070030B505464FF4807234
:102FC0000021E34887B04CF0B9FED02D00F3B28168
:102FD000002D07DA2B464FF48071DE4ADC4841F0C1
:102FE00021FC30E2D02DF5D801A353F825F000BF25
:102FF000593301009D330100A7330100AB330100B9
:10300000AF330100B3330100C3330100C933010002
:10301000D1330100D93301002B34010033340100D6
:10302000373401003B3401003F3401004B340100D0
:1030300053340100573401005B340100FD330100BB
:1030400001340100173401001B3401001F3401005A
:10305000233401005B350100273401005F35010096
:10306000D52F0100D52F0100D52F0100D52F01004C
:10307000D52F0100D52F0100D52F0100D52F01003C
:10308000D52F0100D52F0100D52F0100D52F01002C
:10309000D52F0100D52F0100D52F0100D52F01001C
:1030A000D52F0100D52F0100D52F0100D52F01000C
:1030B000D52F0100D52F0100D52F0100D52F0100FC
:1030C000D52F0100D52F0100D52F0100D52F0100EC
:1030D000D52F0100D52F0100D52F0100D52F0100DC
:1030E000D52F0100D52F0100D52F0100D52F0100CC
:1030F000D52F0100D52F0100D52F0100D52F0100BC
:10310000D52F0100D52F0100D52F0100D52F0100AB
:10311000D52F0100D52F0100D52F0100D52F01009B
:10312000D52F0100D52F0100D52F0100D52F01008B
:10313000D52F0100D52F0100D52F0100D52F01007B
:10314000D52F0100D52F0100D52F0100D52F01006B
:10315000D52F0100D52F0100D52F0100D52F01005B
:10316000D52F0100D52F0100D52F0100D52F01004B
:10317000D52F0100D52F0100D52F0100D52F01003B
:103180005F3401006B340100733401009734010097
:103190009B3401009F340100A3340100A7340100D7
:1031A000AB340100AF340100B3340100B734010087
:1031B000BB340100BF340100C3340100C734010037
:1031C000CB340100CF340100D3340100D7340100E7
:1031D000DB340100DF340100E3340100E734010097
:1031E000EB340100EF340100F3340100F734010047
:1031F000FB340100FF3401000335010007350100F5
:103200000B3501000F3501003F350100433501004A
:10321000473501004B3501004F350100D52F010026
:1032200053350100573501006F340100D52F0100DF
:10323000D52F0100D52F0100D52F0100D52F01007A
:10324000D52F0100D52F0100D52F0100D52F01006A
:10325000D52F0100D52F0100D52F0100D52F01005A
:10326000D52F0100D52F0100D52F0100D52F01004A
:10327000D52F0100D52F0100D52F0100D52F01003A
:10328000D52F0100D52F0100D52F0100D52F01002A
:10329000D52F0100D52F0100D52F0100D52F01001A
:1032A000D52F0100D52F0100D52F0100D52F01000A
:1032B000D52F0100D52F0100D52F0100D52F0100FA
:1032C000D52F0100D52F0100D52F0100D52F0100EA
:1032D000D52F0100D52F0100D52F0100D52F0100DA
:1032E000D52F0100D52F0100D52F0100D52F0100CA
:1032F000D52F0100D52F0100D52F0100D52F0100BA
:10330000D52F0100D52F0100D52F0100D52F0100A9
:1033100013350100173501001B3501001F35010071
:1033200023350100273501002B3501002F35010021
:1033300033350100A5F59673032B3FF64BAE032BF7
:103340003FF648AEDFE813F0F700F9008D008F007C
:10335000DA050220984F0700914992484DF05EF837
:103360002C4646F03FF90368002B00F0FA80002D50
:1033700000F0F78046F036F9006841F0D5FC059082
:103380008848FDF779FF4FF48073C0F1FF0205997B
:1033900084484DF08BF8834807B030BD824981489E
:1033A0004DF03CF827E08149F9E78149F7E7814989
:1033B000F5E7814B814A4FF480717A4841F032FA47
:1033C00019E080237E4AF6E74FF480137D4AF2E746
:1033D0004FF000537C4AEEE700227C4B4FF48071A3
:1033E000CDE902236CA3D3E900236E48CDE9002385
:1033F000774A41F017FA00242546B2E77549CEE72F
:103400004FF6E3734FF480710093734A10236548BD
:1034100041F008FAEFE77149C1E77149BFE7714927
:10342000BDE77149BBE77149B9E74FF41053704AE2
:10343000C1E77049B3E77049B1E77049AFE7704938
:1034400058484CF0EBFF002418E04FF47A736D4AB3
:10345000B1E76D49A3E76D49F2E76D499FE76D4913
:10346000EEE76D49ECE76D49EAE76D49E8E76D493C
:1034700095E76D494B484CF0D1FF01244948FDF7D1
:10348000FBFE4FF48073C0F1FF02684945484DF0E0
:103490000DF8012565E76649ECE76649EAE7664904
:1034A000CEE76649CCE76649CAE76649C8E7664998
:1034B00075E7664973E76649C2E76649C0E766494A
:1034C000BEE76649BCE76649BAE76649B8E76649B8
:1034D000B6E76649B4E7664961E766495FE766496A
:1034E0005DE76649ACE76649AAE76649A8E7664929
:1034F000A6E76649A4E7664951E76649A0E7664939
:103500009EE766499CE7664949E7664998E7664948
:1035100096E76649AEE76649ACE76649AAE76649B9
:10352000A8E766498CE766498AE7664988E76649FD
:1035300035E7664933E7664982E7664980E76649C9
:103540002DE766497CE766497AE7664978E7664988
:1035500076E7664974E7664921E766491FE76649E9
:103560001DE7002C3FF417AF644C206800283FF49F
:1035700012AF0FF02FFE05900A48FDF77DFE4FF4C5
:103580008073C0F1FF02059906484CF08FFF0023BD
:10359000236000E7AFF300809A9999999999B93F10
:1035A0009B430700DA050220A4430700C543070038
:1035B000F1430700224407008051010053440700F3
:1035C00081440700B5440700DF44070000004E4077
:1035D00011450700464507006E450700AA4507004C
:1035E000DE4507002846070076460700B546070077
:1035F000E74607000E470700304707004747070028
:103600007E47070095470700B8470700F2470700C5
:103610000A48070024480700404807006848070098
:1036200096480700B1480700CB480700C4FF0700D1
:10363000F4480700104907003849070058490700B7
:103640007B490700A1490700C8490700EF49070067
:10365000134A0700324A0700544A0700784A070015
:10366000A14A0700BB4A0700D24A0700EC4A0700FC
:10367000FA4A0700144B07002E4B0700614B070066
:10368000804B07009B4B0700BC4B0700D14B07004A
:10369000F24B0700104C0700324C0700574C070054
:1036A000784C0700904C0700AB4C0700C54C070056
:1036B000E34C0700FF4C07001F4D0700384D070083
:1036C0005B4D07007C4D07009E4D0700C44D070071
:1036D000DD4D0700F84D07000F4E07006E4E070046
:1036E000874E0700A74E0700CC4E0700F94E070093
:1036F000154F07003A4F0700634F070048CF0120DE
:103700002DE9F04F436F04468DB063B9616D481CDD
:1037100010D0204615F046FC60B16FF00105284638
:103720000DB0BDE8F08F46F021FD0028EEDA4FF035
:10373000FF35F4E7D4F8A43083B3204615F0A0FB9E
:103740000028EADBD4F8A43043B3C048D4F8D451FD
:1037500014F0C4FCBE490246284646F005FCD4F8E5
:10376000D45118F037FC14F0B9FCBA490246284687
:1037700046F0FAFB204617F017FE0028CDDB0026A6
:103780000F23B246B34623740596D4F88851F5B199
:10379000204647F06BF81B22AF4B3BE0D4F8A0303B
:1037A000002BE7D02046A94AAC4915F00BFCAC4AE7
:1037B000AC49204615F006FC18F00CFCA74902465F
:1037C000204615F0FFFB204646F0CDFFD2E7D4F8A7
:1037D000DC3008A80693D4F8E030079347F08DF862
:1037E00008A818F0DBFE0746D4F8D8002B4600974F
:1037F00007AA06A9013045F04AFC00280CDA45F07A
:10380000F1FE0368042B00F0BA81204647F02EF841
:103810007622914B1A608AE700F0B881D4F88000D4
:1038200006A945F014FCC8B194F910300A2B15D044
:10383000204617F023FE002803DA204647F016F84A
:1038400075E706A9D4F8800045F00EFC94F9013024
:10385000D4F848A1591C40F099805646E06F06A95B
:1038600045F0F5FB40B1204617F07CFE0028E4DB74
:10387000E06F06A945F0F8FB94F910300A2B40F0F0
:103880006881D4F8840006A945F0E1FB00283AD00D
:10389000E36820469B689847B0F10008CDDB47F00D
:1038A000A7F8024650BB059B9E4276D00133059394
:1038B0004146204615F074FA81460028BDD0D9F85B
:1038C0001430002B6FD004F1E001404645F0D6FBE8
:1038D000D4F8D8304345E368B8BFC4F8D8801B6833
:1038E000022B02D1D9F814301BB90121404618F03F
:1038F000C1FDD4F8C0310BB148469847D4F88400D4
:1039000006A945F0B1FB059BB34240F02281D345A7
:1039100040F01F81E3681B68012B47D0D4F8840076
:1039200004F1DC0145F0A0FBD4F8840009F0F2FDBD
:103930004FF0FF33C4F8843094F90130D4F8B80163
:10394000013308BF4FF0020ED0E9068918BF4FF0CF
:10395000010E58EA090361D0D0E904C0D4F8481137
:103960004843CB170CFB0303ACFB01011944A0FB3C
:103970000E230EFB0133994508BF90454ED22046D9
:10398000CDE90089384917F0D9FB01E7002B0ABFC0
:10399000564600264FF0000A60E7DA45AED0012215
:1039A0000BF1010B84E704F1DC018EE7D4F89430CD
:1039B00033B9D4F8B8311A6C12B95B68002BB7D0A0
:1039C00004F1DC084146D4F8800045F04DFBD4F802
:1039D000800009F09FFD0023C4F88030636CD4F8A8
:1039E000B81100930122E3692046096818F074FCBD
:1039F000031E05DA204646F039FF6622164B09E71A
:103A0000C4F88030414645F039FBD4F88030D4F812
:103A1000D8209342C8BFC4F8D83089E70121204696
:103A200015F0ACFC804600287FF407AF204614F068
:103A3000C1FF0028FFF601AF0AA846F05EFF00288C
:103A400014DA6522044B1A60F7E600BF45600700F0
:103A5000CCD10700E24007004CCF0120A67D060034
:103A6000CD190700DC5806007C610700E26CC4E950
:103A70004388C4F80481A2B1A36C6B491A446B4B10
:103A8000283282FB0323C4F80881CDE90023CDF856
:103A9000088022460AA818F051FDC4F80401002845
:103AA000CFD0D4E93A8900230022C4E94333404609
:103AB00000234946FCF7E8FFA8B9012340460293DA
:103AC000494657A3D3E90023FCF776FDFDF712FA28
:103AD0002246CDE9000156490AA818F02FFDC4F886
:103AE0000C010028ADD0D4E93C89002200234046D7
:103AF0004946FCF7C9FFA8B901234046029349464D
:103B000047A3D3E90023FCF757FDFDF7F3F922465D
:103B1000CDE9000147490AA818F010FDC4F81001CA
:103B200000288ED0A36C002B50D1C4F80031C4F80B
:103B3000E43094F901302BB1204614F06BFF0028DB
:103B4000FFF67BAE0221204615F018FC00287FF41A
:103B500074AE94F91030022B11D194F901305A1C33
:103B60004FD1204606A914F039FC0028FFF665AEB7
:103B7000204607A914F096FB0028FFF65EAE5FB161
:103B8000D7E90023134307D1BB682BB908A846F037
:103B9000B4FE08A818F050FD94F91030102B7FF4F3
:103BA000F4AD204646F062FED4F8A43083BB204634
:103BB00046F0D9FDA36D01333FF4B1AD204615F0B9
:103BC000F9F9003818BF01204542A8E50AA846F0D7
:103BD00094FE0028FFF635AF0123C4F8E43000233B
:103BE000A26C0293114B144982FB03230AA8CDE96E
:103BF0000023224618F0A2FCC4F80001002898D146
:103C00001FE7012BB4D0204606A914F0E7FBB3E769
:103C1000204615F079F90028C9DA88E5AFF300806D
:103C20000000000080842E412FA8050040420F00B4
:103C30000FA805001FA8050049B3020000000000FE
:103C400070B5C6690446874DB0B0AEB150220021B0
:103C500008A84CF073F8D4F8B83100211B6830463E
:103C60000A93012308AA0B9303AB45F055F828608B
:103C700010B1CB227C4B4FE05022002108A84CF021
:103C80005DF8D4F8B8310C211B68784A0A930123F7
:103C900005A80B93636C40F0C5FDD4F8D030C3B1D8
:103CA0004FF4A052009309920C21636C704A05A84E
:103CB00040F0B8FD606904AB08AA05A945F02CF8EE
:103CC000286068B1E369002BD3D0039845F026F84B
:103CD000CFE7D4F8CC30002BECD01CAB0893E9E74D
:103CE000049B9868062201210FF080FA051E06DA6F
:103CF000E36913B1039845F011F80498E6E7D4F8A6
:103D0000D01079B118F0DAF8C0B1D4F8D010594811
:103D100040F0D6FBCA22544B4FF0FF351A602846BC
:103D200030B070BDD4F8CC1041B118F077F828B19C
:103D3000D4F8CC10504840F0C3FB9AE7E169236CFB
:103D400000293DD00398C3F30722816942EA032387
:103D50004B804269284644F0F6FF00280FDA45F010
:103D600041FC0468284609F0D5FB039844F0D6FFCF
:103D7000049844F0D3FF45F035FC046079E70398DC
:103D800044F0CCFFD4F89430002B56D001221C9282
:103D900004230621009328461CAB45F003F90028B4
:103DA0004BDA45F01FFC0468284609F0B3FB049881
:103DB00044F0B4FF45F016FC7A222B4B0460ABE7CD
:103DC000002BDFD0049A9268012A16D1ADF870203A
:103DD000C3F3072242EA03230822ADF872301D9193
:103DE00028461CA944F0AFFF0028CBDA45F0FAFBC7
:103DF0000468284609F08EFBBAE7022A0ED1ADF816
:103E00007020C3F3072242EA0323ADF872301B4B44
:103E10001DAE0FCB86E80F001822E1E745F0E2FB6C
:103E20000468284609F076FB049844F077FF45F0D3
:103E3000D9FB83220C4B04606EE7D4F8B8311A6CBE
:103E40001C92EAB145F0CEFB0468284609F062FBFB
:103E5000049844F063FF45F0C5FB7B22024B0460ED
:103E60005AE700BF48CF01204CCF0120AEFE07002B
:103E700013620700196207006BDD0600E82B0600DD
:103E800059681C9129B1D4F8AC3013B12C4840F0DA
:103E900017FBD4F8A430CBB1D4F8B8315868FCF78C
:103EA00021FB41EC100B2749D4F8D40146F0A7F8C8
:103EB0009FED210B2449D4F8D40146F0A0F89FEDE2
:103EC0001E0B2249D4F8D40146F099F8D4F8B83141
:103ED000D3E90413C90851EA437105D0D4F8AC30D2
:103EE00013B11B4840F0ECFA049BD3E905212846A6
:103EF00044F050FF002805DA45F074FB0368772B87
:103F00007FF474AF049844F009FF0123252228466A
:103F100004F5C67146F015FE0028BFF600AF45F067
:103F200061FB0468284609F0F5FA45F05BFB69225D
:103F3000084B0460F0E600BF000000000000000035
:103F4000A0620700E3620700F0620700FE6207005C
:103F50007E6207004CCF0120D0B504464068FCF7D4
:103F6000B1FA09A3D3E90023FCF750FC0646206808
:103F70000F46FCF7A7FA02460B4630463946FCF7D7
:103F800065F941EC100BD0BD0000000080842E418B
:103F90001FB500238DF8073028B98621224B234A0C
:103FA00023483EF035FB0DF10703224902AA40F0F9
:103FB0008DFC9DF80730672B21D010D84D2B22D0D7
:103FC00006D8472B1BD04B2B04D100221A4B0FE0F5
:103FD000542B0AD09DED020B05B05DF804FB6D2B50
:103FE00011D0742B01D06B2BEEE709A3D3E900238A
:103FF000DDE90201FCF7E0FACDE90201EAE706A3F8
:10400000D3E90023F4E706A3D3E90023F0E700BFD8
:10401000000000A2941A6D420000000065CDCD4161
:104020000000000080842E41D3650700576607001A
:10403000DD6507000066070000408F4000000000BB
:104040002DE9F04F2DED028B574B0546D65C08EE5F
:10405000101A06F00306012E5BEC10AB144685B077
:104060000BD05946002210EE100A504BFCF7A4FA70
:1040700082468B46022E08BF203C4D2C10DC412C82
:1040800010DD423C0B2C0DD8DFE804F07D0C0C0C4D
:104090000C4F0C0C0C060C7F0124012E15D158E09E
:1040A000542C74D0012E5F4656464FF000044FF05A
:1040B00000085BD0DFF8189142464B46304639463F
:1040C000FCF700FD08B1042C53D1394B504603EBEB
:1040D000C403D3E900235946FCF76EFA06460F469F
:1040E000344B53F8244030462BA3D3E90023394600
:1040F000FCF7D4FC00284CD129A3D3E90023304697
:104100003946FCF7CBFC2C4B2C4A002818BF1A462A
:1041100018EE101A2846CDE90067029440F082FBA1
:1041200005B0BDEC028BBDE8F08F0324B5E7304647
:10413000394642464B46FCF73FFA06460F460134E5
:104140000022304639461E4BFCF7BCFC08B1042C5B
:10415000EDD11C4B504603EBC403D3E90023594671
:10416000FCF72AFA184B06460F46BAE7DFF86490C8
:10417000E6E73046394642464B46FCF747FB0134FA
:1041800006460F4698E7002487E7022485E70424C3
:1041900083E70E4ABCE700BF3D0AD7A370FD23406A
:1041A000CDCCCCCCCCFC58403E27080000002040B1
:1041B000681C0600847001200F660700186607005F
:1041C00000009040901C06009870012006660700D1
:1041D00000408F400000503F0EB433B5059B0446AD
:1041E00098B103F4700106AAB1F5800F019200F0B6
:1041F0008F820CDCB1F5001F00F0AB80B1F5401FE1
:1042000000F0AA81B1F5801F30D0302087E1B1F5F0
:10421000A00F00F0A682B1F5C00FF6D1111D1268F3
:104220000191002AF1D0C5498B4200F224820A395B
:104230008B42EAD9A3F5C003073B092BE5D801A1BE
:1042400051F823F09F460100A5460100AB4601004E
:10425000B14601000B4201000B4201000B4201007C
:1042600095460100B7460100C5460100111D1268C0
:104270000191002AC9D0B2498B4235D80C398B4202
:1042800011D80B398B424BD003318B424BD01439B0
:104290008B42BAD1D0F85836AA49002B08BF0B463A
:1042A000136000203BE1A3F580131E3B0B2BACD821
:1042B00001A151F823F000BF2D4301003343010059
:1042C000394301000B4201000B4201000B42010087
:1042D000474301000B4201000B4201000B42010069
:1042E0000B4201004143010097498B422ED0093116
:1042F0008B428AD1D0F8A434002BD1D190F94E361C
:10430000002B09DB90F8C83B023BDBB2042B05D83D
:104310008E4951F82330C3E78D4BC1E78D4BBFE782
:10432000D0F8443CBCE7D0F85834B9E7D0F8503B5B
:10433000B6E7D0F8483CB3E700F658441460B0E75D
:1043400000F68C44FAE7D0F85835A9E7D0F8C03C1D
:10435000A6E71568111D0191002D3FF456AFA3F596
:104360000013023B392B3FF650AF01A252F823F065
:10437000594401000B4201000B4201000B420100B5
:104380000B4201000B4201000B4201000B420100F5
:104390000B42010093440100994401009F44010035
:1043A000674401000B4201000B4201000B42010077
:1043B0000B4201000B420100A54401000B42010029
:1043C00061440100AB440100B1440100B744010065
:1043D000BD4401000B4201000B420100C344010037
:1043E0000B4201000B4201000B4201000B42010095
:1043F0000B420100DF4401000B420100F7440100C1
:10440000FD44010003450100CD4401000B420100C1
:10441000D34401000B4201000B4201000B4201009A
:10442000094501000B420100374501000B42010024
:104430000B4201000B4201000B4201000B42010044
:104440000B4201000B4201000B4201000B42010034
:104450000B420100D9440100D0F8103C2B6020E74A
:10446000D0F8143CFAE700F54264D4E90023B2F135
:10447000004F73F1000102DB6FF00043EEE7B2F191
:10448000004F73F1FF3102DA4FF00043E6E72A6094
:1044900007E7D0F8283CE1E7D0F8303CDEE7D0F879
:1044A0001434DBE7D0F86031D8E7D0F83C3CD5E7EE
:1044B000D0F8383CD2E7D0F88C38CFE7D0F8403C81
:1044C000CCE7002118F078FA2860EAE6D0F8883CBA
:1044D000C4E7D0F8BC3CC1E790F8D03CBEE7D0F8C8
:1044E000103CB3F5987F01D10123B7E790F8D13C98
:1044F00003F00103B2E7D0F8783BAFE7D0F87C3B9C
:10450000ACE7D0F8803BA9E7D0F8183C142B10D0CA
:104510000ADC0A2BE8D00B2B09D00020286002B05F
:10452000BDE8304003B070471E2B97D0F5E702235B
:1045300094E7032392E7D0F8C43C8FE710006000B3
:1045400029001000CD19070031001000A02E060030
:10455000C46E070010B107001568111D0191002DF0
:104560003FF453AEA3F54013033B1E2B3FF64DAE75
:1045700001A252F823F000BFF54501000D460100ED
:10458000134601001F4601002B4601003D46010075
:1045900043460100494601000B4201000B42010065
:1045A0000B4201000B4201004F4601005D46010035
:1045B000254601000B420100714601000B4201003B
:1045C0000B4201000B4201000B4201000B420100B3
:1045D0000B4201000B4201000B4201000B420100A3
:1045E0000B4201000B4201000B4201000B42010093
:1045F0001946010000F5D564D4E90001FBF7AEFFD0
:1046000063A3D3E90023FCF701F914E000F5D864B3
:10461000F2E700F5D964EFE700F5DA64ECE700F5BE
:10462000DB64E9E700F5DC64E6E700F5D264D4E991
:104630000001FBF793FFC5E9000132E600F5D16404
:10464000F5E700F5D664F2E700F5D764EFE7D0F8B8
:10465000A4365B0609D500F5CF64E8E7D0F8A436A8
:10466000980602D504F5D064E1E700204449E2E76A
:1046700000F5DD64C0E7A3F5C003323B072B3FF62E
:10468000C4AD072B3FF6C1ADDFE803F02A2D30366D
:10469000393C333F00F54264D4E900011DE000F5E8
:1046A000D264F9E700F5D164F6E700F5D664F3E7E4
:1046B00000F5D764F0E7D0F8A436590609D500F51F
:1046C000CF64E9E7D0F8A4369B0602D500F5D064A4
:1046D000E2E74FF0FF304FF0FF31C2E90001E0E5C3
:1046E00004F5D564D8E704F5D864D5E704F5D964B2
:1046F000D2E704F5DA64CFE704F5DB64CCE704F530
:10470000DC64C9E704F5DD64C6E704F54564C3E786
:1047100004320192069A002A3FF477AD19498B4280
:104720001CD009D807398B4203D001318B427FF46A
:104730006CAD00201060F2E613498B4203D00231C9
:104740008B427FF462AD04F6D843136048F0F1FA6F
:1047500084F8D80C0020C4F8DC0CE0E600F6C8446D
:10476000ECE51468111D0191002C3FF44EAD074A91
:1047700093427FF44AAD002118F01EF9206090E5C5
:104780000000F0BF220040002B0040002C00500031
:104790000000000080842E412DE9F04788B0CDE96B
:1047A0000623DDE90634012B74F10003804605DAA7
:1047B0003D4908B0BDE8F0474BF030BE0023DDE9CD
:1047C00006013A4A82428B4132DB4FF46162002398
:1047D000FCF728FB06460F46354A414202FB07110B
:1047E000A6FB02230B440699079D541843EB0505CD
:1047F0003C22002320462946FCF714FB6FF03B02C5
:10480000C0F1000C02FB01CCA0FB0223141963448D
:1048100043EB0505CDE90201CDE9044509214046F8
:10482000CDE90067234A47F026FA08B0BDE8F087D3
:104830000023DDE90601204AFCF7F4FA18A3D3E9C6
:10484000002381468A46DDE9060182428B411CDB5A
:104850001A4EC9F1000306FB0A33A9FB0667069945
:104860001F44701807994FF461624FF0000347EB43
:104870000101FCF7D7FACDE9009ACDE90201104A0F
:104880000921404647F0F7F9CFE709214046CDE935
:10489000009A0C4A47F0EFF9C7E700BFAFF300807A
:1048A000FF5B260500000000847A07003F7E0500BC
:1048B000F0F1FFFF8D7A07008051010080AEFEFF0E
:1048C000A17A0700B07A0700F0B585B004460D461E
:1048D00010461946DDE90A2352EA030C03D10020F1
:1048E000014605B0F0BD261A65EB01078D4208BFF1
:1048F0008442F4D01CA5D5E90045B44275EB07010C
:104900001BDB4FF47A74A6FB040104FB0711FCF7D0
:1049100089FA04460D460CAB0FCB8DE80F0010ABA7
:104920000FCB00F06DFB0B46A04273EB0501024676
:10493000D5DAA01A65EB0301D3E730463946FCF718
:1049400071FA84420B4675EB0101A8BF4FF47A71EE
:104950000246ADBFA2FB01454FF0FF346FF00045AA
:1049600001FB0355D7E700BFF653E3A59BC4200026
:104970002DE9F04F2DED068BBDB028AE04681B90DD
:10498000304647F088FF1B9B0DF1B00C1D6896E880
:104990000F008CE80F00DDE92823CDE9182305F589
:1049A000D163D3E90023CDE9142305F5D263D3E91C
:1049B0000023CDE91623DDE91823CDE92C2305F5E5
:1049C000DE630FCB8DE80F009CE80F0000F054FB76
:1049D0000023C14AC5F8A806C5F8AC16814688462A
:1049E000FCF720FA4FF47A72002306460F46484639
:1049F0004146FCF717FAB6A3D3E9002382468B465B
:104A0000DDE91401824273EB0101CDE91C23C0F200
:104A1000C2804FF47A73149ABAF1010FA2FB03011A
:104A2000159A7BF1000C03FB021152465B4601DA3A
:104A300001220023FCF7F6F91490149A8846C5F871
:104A4000B026C5F8B416DDE91C23DDE91601824263
:104A50008B41C0F2AB804FF47A73169AA2FB03012C
:104A6000179A03FB02115246012A7BF100065B46AE
:104A700001DA01220023FCF7D5F9DDE9189A8C460A
:104A8000C5F8BC1605F5CE61D1E90023534508BF32
:104A90004A450746C5F8B80600F0A580DDE91823A9
:104AA0004FF0060BD5F8F06705F5D16096FBFBFAE1
:104AB0000BFB1A6AC1E900230BC8D5F89426C3186A
:104AC00005EBCA0942EB010109F5EC69C9E90031BE
:104AD00001360AF1790A05EB0A1A0DF1B00E012E22
:104AE0009EE80F008AE80F00C5F8F06705F5D36A65
:104AF00072D0052ECABF96FBFBF34FF0000B0BFBE9
:104B0000136B0BF1790305EB03130FCB8DE80F004B
:104B10009EE80F0000F074FA0246D9E900060B4641
:104B20000BF1EC0B52EA030105EBCB05D5E90015BF
:104B300004BF01220023411A129166EB0501139173
:104B40000021DDE912566548A842B14139DA314603
:104B50002846CDE91423FBF701FDDDE914230646C1
:104B60000F4610461946FBF7F9FC00225C4BFBF799
:104B70004DFE02460B4630463946FBF747FEFCF732
:104B8000B9F90126CAE90001D4F8A45615F01005B8
:104B90002BD000275AE0012E77F100013246DDE9E3
:104BA00014013B46BCBF0122002343E7012E77F1ED
:104BB00000013246DDE916013B46BCBF012200235D
:104BC00059E74FF47A751299139EA1FB050105FB75
:104BD0000611FCF727F9D4E7149BFF184CEB0801EA
:104BE000CAE90071D0E70026CEE7D4F89C81B8F17D
:104BF000000F31D00121204647F01AFA04F5D263A4
:104C0000D3E90023CDE9042304F5D063D3E90023DD
:104C1000CDE9022304F5D163D3E90023CDE90023D4
:104C200004F5CF60D4F89C11D0E90023D4F8D0016A
:104C3000884729460746204647F0FAF9294B9F4204
:104C400054D01FB12046284947F075FC38463DB086
:104C5000BDEC068BBDE8F08FD4F89831002B45D021
:104C60000121204647F0E4F904F5D263D3E90001BD
:104C7000FBF774FC04F5D06341EC1A0BD3E9000197
:104C8000FBF76CFC04F5D16341EC190BD3E900018F
:104C9000FBF764FC04F5CF6341EC180BD3E900018A
:104CA000FBF75CFCB0EE4A3AF0EE6A3A41EC100BCE
:104CB000B0EE492AF0EE692AB0EE481AF0EE681A12
:104CC000D4F89831D4F8D001984741460746B2E766
:104CD000F653E3A59BC4200040420F0037894100F2
:104CE00000408F4001000010FA7A0700002E3FF4C8
:104CF00050AF1B9BBD4A1C68002304F5D561D1E968
:104D00000001FCF78FF8D4F8A43618901F061B9109
:104D100016D404F53763D3E9002352EA030104D023
:104D2000B349D4F830011EF03DFCB249D4F830014B
:104D30001EF038FCD4F8A43643F08003C4F8A4363F
:104D4000D4F8A456AE0640F1178104F5D763D3E931
:104D50000023012A73F10001C0F20E8104F5D06135
:104D6000D1E9008940464946FCF75CF842F21072EE
:104D70000023424573EB09030F46129004F5D266F7
:104D800080F2EA806422002340464946FCF74AF854
:104D900002460B46D6E90001FCF744F81490169140
:104DA000680640F1038104F5D663D3E90023012AA4
:104DB00073F10001C0F2FA8004F5CF61D1E90089F6
:104DC00040464946FCF72EF842F210720023424555
:104DD00073EB090382468B4604F5D16580F2D680D9
:104DE0006422002340464946FCF71CF802460B4665
:104DF000D5E90001FCF716F806460D46DDF84880B7
:104E0000B946D04577EB0B03BCBFD046D946B8F1C5
:104E1000010F79F10003C0F2D380189BB8EB0302B5
:104E20001B9B69EB03031FA8FFF7B6FC42464B46EA
:104E300022A8FFF7B1FC189A1B9B25A8FFF7ACFC32
:104E4000D4F8A416D4F8887611F0200F04F5D263B4
:104E500008BFD3E9002ED4F88C061CBFD4F88026F6
:104E6000D4F884E6490659BF39468446D4F8781602
:104E7000D4F87CC6521810924EEB0C021192D3E972
:104E80000023BF1842F2107240EB03080023DDE953
:104E9000100182428B4180F2968064220023FBF74E
:104EA000C1FF02460B4638464146FBF7BBFF804632
:104EB0000F46DDE9100131AAD4F830B120F0B6F880
:104EC00004F5D16310902CAAD3E9000120F0AEF8CC
:104ED00004F5D26312900DF1BA02D3E9000120F07B
:104EE000A5F804F5D6638146D3E900010DF1CE02A1
:104EF00020F09CF804F5D7638246D3E9000136AA76
:104F000020F094F804F5D36118900DF1E202D1E994
:104F1000000120F08BF8189B1FAACDE909A3149B70
:104F20000D920693169B25AA0793129B0C9204934D
:104F3000109B22AA0E900B92009342463B46584685
:104F4000CDE902652C49CDF820901EF02BFBD4F85A
:104F500030013DF0EDFC1CE6B8F1010F79F10003E2
:104F600010DB6423D4F890067268A0FB030103FBF6
:104F7000021142464B460FE700231F46129314933B
:104F800016930DE700231493169309E7B8F1010F68
:104F900079F1000311DB6423D4F888066A68A0FB6A
:104FA000030103FB021142464B4623E74FF0000A80
:104FB0004FF0000B56465D4620E7002635461DE7BC
:104FC000002213462FE7DDE91023012A73F10003C5
:104FD00007DB6423A7FB030103FB0811DDE91023B2
:104FE00063E74FF00008474663E700BF40420F0009
:104FF0000B7B0700397B0700DB7B0700000000000C
:1050000030B585B00DF1100C0CE90F00089B009A2B
:10501000D41A019A099B62EB030513A3D3E9002379
:10502000A242AB4116DB12A3D3E90023944275EBF5
:10503000030314DB0A9A029B9B1A4FF47A7293FBC8
:10504000F2F3A4FB020102FB0511C01841EBE3716E
:1050500005B030BD4FF0FF306FF00041F8E70020A1
:105060004FF00041F4E700BFF653E3A59BC42000D6
:105070000AAC1C5A643BDFFF30B585B00DF1100C53
:105080000CE90F00089B009AD41A019A099B62EB65
:10509000030514A3D3E90023A242AB4115DB13A3FC
:1050A000D3E90023944275EB030313DB0C4BA4FB01
:1050B000030103FB05110A9BC01A61EBE371029B1C
:1050C000C01841EBE37105B030BD4FF0FF306FF019
:1050D0000041F8E700204FF00041F4E7AFF3008013
:1050E00040420F00F55AD07B630800000BA52F84C7
:1050F0009CF7FFFF000000002DE9F04788B0CDE9E4
:105100000623DDE90634012B74F10003804605DA3D
:105110003D4908B0BDE8F0474BF080B90023DDE918
:1051200006013A4A82428B4132DB4FF4616200232E
:10513000FBF778FE06460F46354A414202FB07114F
:10514000A6FB02230B440699079D541843EB050563
:105150003C22002320462946FBF764FE6FF03B0209
:10516000C0F1000C02FB01CCA0FB02231419634424
:1051700043EB0505CDE90201CDE90445092140468F
:10518000CDE90067234A46F076FD08B0BDE8F08718
:105190000023DDE90601204AFBF744FE18A3D3E90A
:1051A000002381468A46DDE9060182428B411CDBF1
:1051B0001A4EC9F1000306FB0A33A9FB06670699DC
:1051C0001F44701807994FF461624FF0000347EBDA
:1051D0000101FBF727FECDE9009ACDE90201104A53
:1051E0000921404646F047FDCFE709214046CDE979
:1051F000009A0C4A46F03FFDC7E700BFAFF30080BE
:10520000FF5B260500000000847A07003F7E050052
:10521000F0F1FFFF8D7A07008051010080AEFEFFA4
:10522000A17A0700B07A070070B52DED028B00233C
:1052300086B0CDE9043304230D46064601930028C9
:1052400000F0F780002900F0F480062104A848F05F
:1052500012FD044690B17A4A1368590709D0794B78
:105260000146D21A92089201774842F0010242F0B8
:10527000F4FB204606B0BDEC028B70BD014604AACB
:10528000304648F0F5FC044688B16D4A13685B0768
:1052900009D06C4B0146D21A920892016B4842F039
:1052A000010242F0DAFB04A848F0F8FCE1E7032130
:1052B00001AB02AA04A848F0ECFD044660B1604AC4
:1052C00013685E07EFD05F4B0146D21A9208920135
:1052D0005F4842F00102E4E7019B06AA134401463D
:1052E00003F8100C022202A840F05CFC6A46064655
:1052F000012104A848F096FD044660B1504A1368A5
:105300005D07D0D04F4B0146D21A92089201514806
:1053100042F00102C5E7009B042B2FD0052B11D0D2
:10532000474928700B6813F0060F08D0454B4A48D0
:10533000C91A8908890141F0020142F07FFB6FF030
:105340007F04B0E709239FED458A2B702C1D54D0B4
:10535000F0B20F2851D8072B15D0092B49D06FF088
:105360007F04374A136858079DD0364B2146D21A1E
:10537000920892013A4842F0010292E707239FED1A
:10538000398A2B70E2E7384B33F81000002832D00E
:10539000FBF7A8F828A3D3E90023FBF70DF9FBF7E7
:1053A000E3FB042168600DEB010302AA04A801914C
:1053B00048F06FFD044618BB019B06AA1344014642
:1053C00003F8100C022202A840F0ECFBC1B20F2936
:1053D00024D91B4A13685B0708D01A4B2348D21AFA
:1053E0009208920142F0010242F037FB6FF015047F
:1053F00059E71F4BC8E71F48D3E76FF01504B0E724
:105400000F4A136859073FF44EAF0E4B0146D21AAC
:1054100092089201184842F0010242E70130C0B2FE
:1054200007EE900AF8EEE77A67EE887AC5ED027A21
:1054300039E76FF015041CE77B14AE47E17A24408E
:105440006474012038740120A5EE0700A0F5070060
:10545000CCF50700F8F507001AF607000AD7234035
:1054600042F607000AD7A33F8058060091F60700CE
:10547000A05806000AD7A34066F607000000000007
:105480002DE9F04F1F46A3B0002304468846199229
:105490001E934FF0000AA34B4FF0000B1B681846F9
:1054A0000793FBF7E9FE0546CDF874801D9B1A783B
:1054B0002B2A4CD039D80D2A32D8082A32D8002AC3
:1054C0003CD000230E931D9E3378302B40F0B580E6
:1054D000737803F0DF03582B6CD10E9B1DA9029744
:1054E000204601931EAB904A00931FAB40F024FE70
:1054F00010F00707054605D0062F2AD101360023F4
:105500001D960E93199B002B40F09A850E9BDBB1E4
:1055100052460BF1004343EC102B23B0BDE8F08F53
:10552000202ACED101331D93C0E72D2AC9D10122F3
:105530000E925A1C1D925B78002BC4D1199BCDF89A
:105540007480002B40F07A8552465B46E3E70022E8
:10555000EEE71E9A3AB1352120A84BF0D5FD1E99F1
:1055600020464BF0CEFA013F052F07D8DFE807F0C1
:105570000E0B181D0E034FF0000BDA462807C1D59D
:105580004BF0004BBEE7DDE920ABF7E7DDE920A3F8
:105590001F9A23F4801302F2334243EA025BEDE7E1
:1055A000DFF888B14FF0000AE8E76FF0004B4FF0EA
:1055B000FF3AE3E71D9B5A1C1D925B78302BF9D014
:1055C000002B9FD001234FF0000904930A221D9B5A
:1055D0004F46CDF824900A931D980678A6F1300323
:1055E000D9B209292BD92A4607994AF081FF002808
:1055F00034D0002033463D4602460790652B01D04B
:10560000452B18D11DB9049B034397D00025DDF825
:10561000748008F101031D9398F801302B2B75D08D
:105620002D2B7BD04FF0000CA3F13001092940F263
:105630008380CDF8748000269EE00023C3E7082F06
:1056400000F1010007F10107D4BF099902FB0939F4
:105650001D90DCBF02FB01330993BDE71D9B5A1966
:105660001D925B5D002F36D03D460790A3F13002BE
:10567000092A12D90122C1E71D9B01305A1C1D9233
:105680005B78302BF8D0A3F13102082A00F2DD84D8
:10569000079000201D9A05460A92303B00F1010256
:1056A00013D0079900EB050E11442A4607910A21F1
:1056B000724512D12A180135082A05441CDC0999C3
:1056C0000A2202FB0133099300221D9B1046591C3C
:1056D0001D915B78CAE73846D3E7082A04DC099EA7
:1056E0004E4309960132E3E702F1010CBCF1100FC1
:1056F000D8BF01FB09F9F5E7102DDCBF0A2202FB38
:105700000939E1E70023012207937CE74FF0000C01
:1057100008F102031D9398F8023085E74FF0010C61
:10572000F6E700BF08580600E45606000000F07FC8
:105730001D9B591C1D915B78302BF9D0A3F13101D1
:1057400008293FF678AFA3F1300E1D9B08931D9BEF
:10575000591C1D915B78A3F13006092E37D9089E9C
:10576000891B44F61F66082902DC7645A8BF7646E9
:10577000BCF1000F00D07642002D4FD104990143B7
:105780007FF4C0AE002A7FF4D9AE692B27D024DC89
:10579000492B24D04E2B7FF4D1AE9F491DA84BF04E
:1057A000B6F800283FF4CAAE1D9B1B78282B2DD1DC
:1057B00020AA9A491DA84BF0BEF8052826D1219BA6
:1057C000DDF880A043F0FF4B4BF4E00B9AE60A2192
:1057D00001FB0E3EAEF1300EB9E76E2BDBE79049D0
:1057E0001DA84BF094F800283FF4A8AE1D9B1DA8FF
:1057F0008C49013B1D934BF08AF810B91D9B013376
:105800001D93DFF830B24FF0000A7BE6864801F0C6
:1058100023FA8DED040BDDE904AB73E6079B002F43
:1058200008BF2F46102D0998A6EB0303A846A8BF72
:105830004FF010080893FAF745FE092D82468B4673
:1058400013DD7A4B03EBC80353E91223FAF7B4FED6
:1058500082468B464846FAF735FE02460B465046CE
:105860005946FAF7F3FC82468B460F2D38DC089B2D
:10587000002B3FF447AE24DD162B0BDC6B4D52465C
:1058800005EBC3055B46D5E90001FAF795FE8246B4
:105890008B4637E6C5F12503089A934220DBC5F114
:1058A0000F05624C52465B4604EBC501D1E900018D
:1058B000FAF782FE089B5D1B04EBC504D4E90023C4
:1058C000E3E7089B16330BDB079B5046574A5946C4
:1058D0009E1B02EBC606D6E90023FAF797FFD6E730
:1058E000A5EB0808089B9844B8F1000F71DD18F08B
:1058F0000F030AD04D49524601EBC3015B46D1E983
:105900000001FAF759FE82468B4638F00F084DD059
:10591000B8F59A7F22DD00252E46099507952223AA
:10592000DFF810B14FF0000A2360099B002B3FF411
:10593000E9AD1E9920464BF0E4F8079920464BF05C
:10594000E0F8314620464BF0DCF8099920464BF050
:10595000D8F8294620464BF0D4F8D3E500234FEA87
:105960002818504659469946B8F1010F21DC0BB171
:1059700082468B462E4BABF1547B524603EBC90952
:105980005B46D9E90001FAF717FE2A4B0A46824620
:105990000B4029498B42BED8A1F580118B4286BFAE
:1059A000DFF898B04FF0FF3A02F1547B00230493E4
:1059B00082E018F0010F07D01D4B03EBC903D3E9B8
:1059C0000023FAF7F9FD012309F101094FEA6808FC
:1059D000CAE7EBD0C8F1000818F00F020AD0134B49
:1059E0005046594603EBC203D3E90023FAF70EFFF2
:1059F00082468B465FEA2818D8D0B8F11F0F1FDD0A
:105A000000252E460995079522234FF0000A4FF0F6
:105A1000000B236089E700BF6D2F0800F8560600D1
:105A20005F070700A54C0700CD190700381D0600C9
:105A3000101D06000000F07F0000A07CFFFFEF7F3C
:105A400018F0100350465946DFF8B49318BF6A2384
:105A50000493002318F0010F04D0D9E90023FAF7CA
:105A6000ABFD01235FEA680809F10809F2D10BB127
:105A700082468B46049BBBB1CBF30A535946C3F114
:105A80006B03002B10DD1F2B40F32781342B4FF0CD
:105A9000000ADBBF203B4FF0FF324FF05C7B02FA85
:105AA00003F3D8BF03EA010B0022002350465946F6
:105AB000FAF7EAFF0028A3D1099B3A460A99204643
:105AC00000932B464BF073F8099000283FF423AF66
:105AD000079B00259E1B089B002BB4BF3346002369
:105AE0002E461093089B23EAE3731893099B2046E4
:105AF00059684AF0D2FF079000283FF410AF099B85
:105B00000C301A6903F10C01023292004AF0DCF801
:105B100020AA1FA920464BEC10ABCDE90AAB4BF0F5
:105B200070FA1E9000283FF4FAAE012120464BF097
:105B3000CCF8064600283FF4F2AE1F9B0499002BD8
:105B4000A3EB0108A9BF109A189A03EB0209189F4A
:105B5000B8BFD71A209AA54B9044B8BFDDF8409043
:105B6000C2F1360208F1FF38984580F2CA80A3EBF3
:105B7000080301211F2BA2EB030200F3B58001FAF9
:105B800003F3119300230C9309EB0208049B1744C1
:105B9000C1451F444B46A8BF4346BB42A8BF3B4636
:105BA000002BC2BFA8EB0308FF1AA9EB0309109B47
:105BB000002B17DD31461A46204640F027FD0646E9
:105BC00000283FF4ACAE01461E9A20464BF086F802
:105BD0000F9000283FF4A3AE1E9920464AF091FF93
:105BE0000F9B1E93B8F1000F00F39080089B002BD1
:105BF00008DD189A2046079940F008FD0790002814
:105C00003FF48DAE002F08DD3A46079920464BF051
:105C100000F9079000283FF482AEB9F1000F08DDCB
:105C200031464A4620464BF0F4F8064600283FF439
:105C300076AE079A20461E994BF066F90546002875
:105C40003FF46DAEC36831460F930023C3604BF041
:105C50003FF9002864DA0F9B53EA0A0340F086807C
:105C6000CBF31303002B40F081802BF000431B0D7E
:105C70001B05B3F1D66F79D96B6913B92B69012B69
:105C800074DD2946012220464BF0C3F83146054613
:105C90004BF01EF9002869DD04995B46544A00293F
:105CA00000F0848002EA0B01B1F1D66F7EDCB1F125
:105CB0005C7F7FF7A9AE00234E4A50465946CDE996
:105CC0001632DDE91623FAF777FC0B4682468B463F
:105CD000034304BF222323602BE64FF0FF3202FA76
:105CE00003F303EA0A0ADFE6C8F17F48119108F5D9
:105CF0007F0808F57B4808F1E20801FA08F30C93E5
:105D000042E700230C93012311933DE742461E997D
:105D100020464BF07EF81E9000287FF467AFFEE52A
:105D20005F466FD10F9ACBF3130342B3324A9342CB
:105D300028D1049B5046EBB12D4A4FF0FF313A4039
:105D4000B2F1D46F19D8120DC2F16B0301FA03F34B
:105D5000984217D1294B9F4202D101303FF4DFAD69
:105D6000234B4FF0000A3B4003F5801B049B002BA4
:105D7000A1D1DEE54FF0FF33EAE70B46E8E753EA4F
:105D80000A0389D00C9BDBB13B42EFD00F9B5046FE
:105D9000049A5946C3B14AF032FC02460B46DDE98B
:105DA0000A01FAF753FA82468B46DFE713404FF0B9
:105DB000FF3AA3F580136FEA135B6FEA0B5BD5E73D
:105DC000119B13EA0A0FE0E74AF019FC02460B4662
:105DD000DDE90A01FAF738FA0022002382468B46F1
:105DE000FAF752FE0028C1D00EE600BF02FCFFFF0A
:105DF0000000F07F00005039FFFF0F00FFFFEF7F32
:105E0000E81C0600314628464BF04BF900224FF0C3
:105E1000804310EE100A59EC108B4946FAF748FE01
:105E200000287CD00F9B002B4CD00022944B4FF0CD
:105E30000008DFF84C92CDE90C23924B3B401193C4
:105E4000119A914B9A4240F0B280A7F1547BDDE960
:105E50000A23DDE90C014BEC10ABCDE91623CDE9AB
:105E60000C0140F021FCDDE90C0153EC102BFAF79A
:105E7000A3FB52465B46FAF7E9F90B468149824695
:105E8000824A194091425ED90B9B02F154729342AF
:105E900003D10A9B01333FF442ADDFF8FCB14FF070
:105EA000FF3A1E9920464AF02CFE079920464AF0F8
:105EB00028FE314620464AF024FE294620464AF074
:105EC00020FE13E6BAF1000F1BD1CBF31303F3B995
:105ED00000226B4B40464946FAF7E0FDD0B94046F8
:105EE000494600226A4BFAF767FB8046894609F16A
:105EF0000043CDF868801B93DDE91A23CDE90C231C
:105F00009BE7BAF1010F02D1002F3FF47DAD0022D3
:105F1000604B8CE74FF00008DFF87491E7E75C4BCB
:105F2000404649460022FAF747FB0F9B80468946C8
:105F300033B901F1004312901393DDE91223DDE739
:105F4000CDE91289F9E703F1547B049B002BA8D11A
:105F50002BF00043119A1B0D1B059A42A1D140461C
:105F60004946FAF7C7FFFAF7F9FA02460B464046E8
:105F70004946FAF769F9CBF313030F9A804643EACF
:105F80000A038946134353D035A3D3E90023FAF714
:105F900085FD00287FF4CDAC4046494632A3D3E9C5
:105FA0000023FAF799FD00283FF47BAFC1E4049B7E
:105FB00033B3119BB3F1D46F22D8404649462CA38A
:105FC000D3E90023FAF774FDA0B149464046FBF738
:105FD00029F9012838BF0120FAF774FA0F9B80468F
:105FE000894613BB01F1004314901593DDE9142396
:105FF000CDE90C230D9B119A03F1D6639B1A0D93E7
:10600000DDE90C019DED0A0BCDE90C0140F04CFBE4
:10601000DDE90C0153EC102BFAF7CEFADDE90A2387
:10602000FAF714F982468B468FE7CDE91489DDE74C
:1060300011A3D3E90023FAF731FDB4E700230E934F
:106040001D9B199A1360FFF761BA652B3FF45AAB99
:10605000452B3FF457AB0122FFF790BBAFF3008015
:106060009535A094FFFFDF3F35E5AF350000E03FF9
:106070000000C0FFFFFFDF419535A094FFFFCF3F39
:106080000000F03F0000F07F0000E07FFFFF9F7CFA
:106090000000E03F0000F0BFFFFFEF7F00000000C6
:1060A0002DE9F04F456A04462DED028B95B057EC73
:1060B000106BDDF88080059109920F93CDE902679E
:1060C0003DB910203DF0FAF960620560C560C0E995
:1060D0000155636A196851B15A68012320469340FB
:1060E0004A608B604AF00DFD636A00221A603B1E15
:1060F000B7BF23F00043002301220393A8BFC8F8D1
:106100000030DDF80C90B64BB8BFC8F8002033EA79
:1061100009031BD142F20F730F9A1360C9F31303E3
:10612000334300F07285219B63B9AE4B25E0AE4B43
:1061300000930833219A1360009815B0BDEC028BD0
:10614000BDE8F08FA74B00930333F3E79DED027B8F
:106150000022002351EC170B8DED0A7BFAF794FC1B
:10616000804660B101230F9A1360219B002B00F041
:1061700049859E4B219A1360013B0093DCE7C9F3EC
:106180000A5512AA13A920469DED0A0B4AF039FFC1
:106190008246002D7CD00B9BA5F2FF35CDF84080C8
:1061A000C3F31303DDE90A6743F07F5747F4401751
:1061B00000228F4B30463946FAF746F882A3D3E9DE
:1061C0000023FAF7F9F982A3D3E90023FAF73EF89E
:1061D00006460F462846FAF785F97FA3D3E9002340
:1061E000FAF7EAF902460B4630463946FAF72EF836
:1061F00006460F46FAF790FC0022814600233046FF
:106200003946FAF74BFC48B14846FAF76BF9324683
:106210003B46FAF739FC08B909F1FF39B9F1160F15
:1062200055D8744B03EBC903DDE90A01D3E9002318
:10623000FAF734FC00284CD009F1FF3900230E9303
:10624000129B5D1B6B1E049345BF0023C5F1010823
:106250004FF000080493B9F1000F3CDB049BCDF82C
:1062600034904B44049300230693059B092B00F2C2
:106270009980052BC5BF043B002501250593059B8F
:10628000023B032B00F29A80DFE803F02D7E7C8A2C
:10629000DDE912531D4405F23243202BC6BFC3F182
:1062A000400305F21240C3F1200305F1FF35C5BFDD
:1062B00009FA03F326FA00F006FA03F01843FAF796
:1062C00001F901230646A1F1F877109370E7012345
:1062D000B5E70E90B4E7C9F10003A8EB09080693EF
:1062E00000230D93C1E700230893099B002B00F3C3
:1062F00085804FF0010B5B46CDF804B0CDF824B09B
:106300000022666A7260042202F1140071689842E9
:106310007AD920464AF0C1FB636A30601B6800935B
:10632000019B0E2B00F2F580002D00F0F280B9F1F8
:10633000000F7DDD09F00F032E4A19F4807F4FEA2C
:10634000291702EBC30393ED007BB0EE478AF0EE12
:10635000678A5DD0284B07F00F070325D3E9082390
:10636000DDE90A01FAF752FACDE90201224E002FC7
:1063700050D1DDE9020153EC182BFAF747FACDE9C9
:1063800002016FE00123AFE700230893099B09EBAB
:10639000030B0BF10103012B0193B8BF0123AFE7FE
:1063A0000123F2E701250023089505934FF0FF3BF9
:1063B00000221223CDF804B00992A1E7012308932B
:1063C000F4E700BFAFF3008061436F63A787D23F5C
:1063D000B3C8608B288AC63FFB799F501344D33FD4
:1063E0000000F07FD9300800D03008009326080064
:1063F0000000F83F381D0600101D0600DDF824B02F
:106400005B46CDF804B07BE70131520071607BE759
:106410000225ABE7F90708D5013551EC180BD6E991
:106420000023FAF7C9F841EC180B7F1008369EE7F5
:1064300000F0AB80C9F10006AA4BAB4F022506F075
:106440000F02361103EBC203DDE90A01D3E9002391
:10645000FAF7B2F80023CDE90201002E40F08A805D
:10646000002B8CD10E9B002B00F0918000229F4BC3
:10647000DDE9026730463946FAF710FB002800F0E4
:106480008680019B002B00F08280BBF1000F3CDD79
:1064900009F1FF3301350022304607933946944B0A
:1064A000FAF78AF8CDF830B0CDE90201DDE90267EC
:1064B0002846FAF717F832463B46FAF77DF88D4B37
:1064C0000022F9F7C3FEA1F15073CDE90201039355
:1064D0000C9B002B60D10022874B30463946F9F7E0
:1064E000B3FE06460F46DDE90223FAF7F5FA002867
:1064F00040F097823046DDE9022101F10043394640
:10650000FAF7CCFA002840F08982DDE90A23CDE9C8
:106510000223139B002BC0F25B81B9F10E0F00F335
:106520005781704B03EBC90393ED007B099B002B54
:10653000B0EE478AF0EE678A80F2E280019B002B82
:1065400000F3DE8040F06A8200226B4B51EC170BA7
:10655000FAF732F8DDE90223FAF7B4FA019E37467A
:10656000002840F04082009D312309F1010905F81F
:10657000013B3CE2F20705D50135D7E90023FAF7E4
:106580001BF801237610083767E702256AE7019BAD
:10659000CDF81C900C9389E700990C980C9A014453
:1065A000504B9DED027B03EBC20302910899B0EEC4
:1065B000478AF0EE678A53E90223002945D000207C
:1065C0004E49FAF723F953EC182BF9F73DFE009DDD
:1065D00041EC180B39463046FAF79EFA0C90F9F761
:1065E00081FF02460B4630463946F9F72DFE0C9BDB
:1065F00006460F46303305F8013B53EC182BFAF7EB
:106600004DFA002864D132463B4600203749F9F75D
:106610001BFE53EC182BFAF741FA002840F0B88023
:10662000029B9D423FF471AF0022314B51EC180B9D
:10663000F9F7C2FF00222E4B41EC180B30463946C9
:10664000F9F7BAFF06460F46C4E751EC170BF9F706
:10665000B3FF029B009D0C9341EC180B394630466A
:10666000FAF75AFA1190F9F73DFF02460B46304609
:106670003946F9F7E9FD119B06460F4630330022F3
:1066800005F8013B029B9D4225D11C4B51EC180B98
:10669000F9F7DCFD02460B4630463946FAF71CFA9C
:1066A000002875D10020154953EC182BF9F7CCFDC3
:1066B00002460B4630463946FAF7F0F900283FF417
:1066C00024AF0C9D6B1E0C9315F8013C302BF8D0B9
:1066D000DDF81C904AE0064BF9F76EFF06460F46C0
:1066E000BCE700BF381D0600101D06000000F03F8B
:1066F0000000244000001C40000014400000E03F67
:10670000DDE90267009D3046394653EC182BFAF755
:106710007DF8FAF701FA8046F9F7E4FE53EC182BFE
:10672000F9F74AFF0246304608F130060B46394673
:10673000F9F78AFD05F8016B009E0246019F0B46A2
:10674000AE1BB74237D1F9F781FD06460F4653EC31
:10675000182BFAF7C1F9C8B93046394653EC182B53
:10676000FAF792F910B118F0010F0FD120465146F7
:106770004AF0C7F9002309F101002B700F9B186044
:10678000219B002B3FF4D8AC1D60D5E4CDF81C90C4
:106790002B461D4613F8012D392A08D1009A9A423A
:1067A000F7D1079A00990132079230220A701A78BD
:1067B00001321A708CE700229C4BF9F7FDFE002293
:1067C000002306460F46FAF75FF900289BD0CDE775
:1067D000089A002A00F0C480059A012A00F3A980D3
:1067E000109A002A00F0A18003F23343069E45462A
:1067F000049A0121204698441A4404924AF065FA0A
:106800000746002D0BDD049B002B08DDAB42049AEC
:10681000A8BF2B46A8EB0308ED1AD31A0493069BD6
:10682000FBB1089B002B00F09F80002E11DD394644
:10683000324620463FF0EAFE5246014607462046D1
:106840004AF04CFA5146079020464AF05AF9079B05
:106850009A46069B9A1B04D0514620463FF0D6FE2E
:106860008246012120464AF030FA0D9B0646002B55
:106870007CDD1A46014620463FF0C8FE059B0646D1
:10688000012B76DD00230693336906EB8303186939
:106890004AF0CBF9C0F12000049B184410F01F000F
:1068A00000F08680C0F12003042B7FDDC0F11C00C6
:1068B000049B8044054403440493B8F1000F05DDB4
:1068C0005146424620464AF0A4FA8246049B002BD9
:1068D00005DD31461A4620464AF09BFA06460E9BD5
:1068E000002B67D0314650464AF0F2FA002861DAB0
:1068F000002351460A2220464AF01AF9089B09F162
:10690000FF398246002B00F08781394600230A2296
:1069100020464AF00DF9BBF1000F074600F38E80C8
:10692000059B022B40F38A804CE0129BC3F1360397
:106930005CE7019B5E1E069BB342B7BF069B9E1B96
:106940000696F21ABFBF0D9B00269B180D93019B64
:10695000002BB5BFA8EB030545460023019B47E785
:10696000069E4546089F4CE7069A75E7059B012B56
:1069700018DC029BB3B9039BC3F31303A3B9039BB6
:1069800023F000431B0D1B052BB1049B08F10108EC
:1069900001330493012306930D9B002B7FF474AF06
:1069A000012079E70023F6E7029BF4E785D018463B
:1069B0001C307DE7019B002B3ADC059B022B37DD69
:1069C000DDF804B0BBF1000F0DD131465B46052266
:1069D00020464AF0ADF80146064650464AF078FA9D
:1069E00000283FF7C0AD099B009D6FEA03094FF0F7
:1069F0000008314620464AF084F8002F3FF4B6AE36
:106A0000B8F1000F05D0B84503D0414620464AF002
:106A100078F8394620464AF074F8A7E6002637464B
:106A2000E1E70C9EDDF81C9037469CE50000244011
:106A3000089BDDF804B0002B00F0F580002D05DD8B
:106A400039462A4620464AF0E4F90746069B002BC1
:106A500055D0796820464AF020F83A69054607F192
:106A60000C0102320C30920049F02EF90122294625
:106A700020464AF0CEF9009BB84607460133019301
:106A8000009B5B440793029B03F001030693019B69
:106A90003146504603F1FF3B49F032FE0346414682
:106AA00002905046303308934AF012FA3A46049066
:106AB000314620464AF028FAC2680546089B02BBC8
:106AC000014650464AF004FA089B024629462046F1
:106AD000CDE908324AF015F8059B099A019D43EA71
:106AE0000201069B0B43089B0DD1392B27D0049A3A
:106AF000002A01DD029B31338BF8003079E73846FC
:106B0000B9E70122E2E70499002904DB0598014373
:106B10000698014320D1002AEEDD5146012220468D
:106B200001934AF076F9314682464AF0D1F90028BD
:106B3000019B02DCE0D1DA07DED5392BDAD139232B
:106B40008BF800302B461D46013B15F8012C392AE5
:106B500050D001321A704CE7002A03DD392BEED0F9
:106B60000133C9E7019A079902F8013C8A422AD009
:106B7000514600230A22204649F0DAFFB8458246F2
:106B80004FF000034FF00A024146204607D149F07A
:106B9000CFFF80460746019B0133019377E749F019
:106BA000C7FF3946804600230A22204649F0C0FF2D
:106BB0000746F0E7BBF1000F009A4FF00008CCBF8A
:106BC0005D460125154451460122204601934AF0B5
:106BD00020F9314682464AF07BF90028B2DC02D126
:106BE000019BDB07AED42B461D4613F8012D302A3E
:106BF000FAD0FEE6009A9A42A5D1312309F10109A3
:106C00001370F6E6124BFFF7B8BA219B002B7FF406
:106C10008EAA104BFFF7B1BABBF1000F03DC059B46
:106C2000022B3FF7CFAE009D3146504649F068FD3C
:106C3000009A00F1300305F8013BAA1A9345B9DD2B
:106C4000514600230A22204649F072FF8246EBE7B4
:106C500092260800D03008009FED010B704700BF5E
:106C6000000000000000F87F08B50BF075FB2E4B0C
:106C70002E4918602E4840F093FB2E4840F090FBC0
:106C80002D4840F08DFB2D4840F08AFB00202BF072
:106C90003BFD2B4B98422DDC023B984232DC431CDF
:106CA00035D0A0F188600138012808D8254840F087
:106CB00077FB254840F074FB002008F077F9234863
:106CC00040F06EFB2CF02EFF2CF0D0FF47F01FF9A8
:106CD00006F074FA014610B11D4840F061FB04F063
:106CE0007BFC2FF05BFE0146C8B1BDE808401948A7
:106CF00040F056BB184B9842E1D1184840F050FB89
:106D00001748D7E70F4840F04BFB1648D2E7164824
:106D100040F046FBBDE808400B4840F041BB13483B
:106D2000BDE808402FF044BE88A20120C0580600EC
:106D3000C7580600DF580600FB5806001659060023
:106D400004004004305906004F590600FE59060061
:106D5000145A0600335A0600010050055D5906001A
:106D600080590600AE590600DE59060068770120FA
:106D700010B504460846114626F0EAFF20460021D9
:106D8000024A41F03EFA002010BD00BF5C5A0600E6
:106D900070B50546506848F0F4FE041E08DA02217A
:106DA00028462B4A41F02DFA6FF01504204670BD9D
:106DB00048D0234600212846264A41F022FA0021E5
:106DC0004FF480403AF0DCF9234837F031F920B134
:106DD000002302211A4642F0FBFA204837F028F936
:106DE00020B1002302211A4642F0F2FA002CDDD035
:106DF0004FF47A704FF400464443002140F2E730EC
:106E00004FF47A720023E6FB0401FAF75BF83AF0DC
:106E1000B7F9114837F00CF920B1002301211A46C7
:106E200042F0D6FA0D4837F003F920B100230121D2
:106E30001A4642F0CDFA00212846094A41F0E1F90C
:106E40000024B3E721462846064A41F0DAF9B6E7BE
:106E5000635A0600805A0600D05A0600D75A060028
:106E6000DE5A0600A95A0600034603480221034AD7
:106E7000006841F0C6B900BF88A20120F65A06009A
:106E800003480B46034A0021006841F0BAB900BF2D
:106E900088A20120FC5C0600F0B50024324DADF65E
:106EA000A42D012906468DF80F4028600BD82F4BE2
:106EB0002146CDE900332E4A2E4B41F0A2F920465F
:106EC0000DF6A42DF0BD57682B493846FAF7CAF9DC
:106ED000044688B9304629492CF0F2FE034628B909
:106EE00021463046264A41F08CF9E8E7254A2146FA
:106EF000304641F086F9E2E738462349FAF7B2F91D
:106F0000044620B930461D492CF028FFD7E70DF183
:106F10000F0340F68D22384604A92CF03FFD9DF862
:106F20000F400346E4B1013C062C0AD8DFE804F028
:106F3000040C0E1012141600144A0221286841F0A5
:106F400060F96FF01504BAE7114AF6E7114AF4E761
:106F5000114AF2E7114AF0E7114AEEE7114AECE76D
:106F6000114A04ABC3E700BF88A20120179E0700A7
:106F7000A67D0600235E0600125D0600816E0100FC
:106F8000205D0600525D0600895D0600F95D060081
:106F9000985D0600A75D0600B65D0600C75D0600A9
:106FA000E65D0600045E06001D5E0600F0B58FB0CB
:106FB00002AA06460C461746214B03F1300C154633
:106FC00018685968083303C563452A46F7D14CB998
:106FD0001C491D4818231D4A40F0E2F918211B489E
:106FE00040F0DEFC2046FAF747F92F28054609D97C
:106FF000174B0221174A186841F003F96FF015008A
:107000000FB0F0BD024630232146384648F069FEF5
:10701000192200953B460121304641F0C3FF051E71
:107020000CDA0B4B1E683DF07FFE2346CDE9005085
:1070300002213046084A41F0E4F8DFE70020DFE7AC
:10704000D01B060057CD0600235F06000A5F06002E
:1070500088A20120405F06005F5F0600F0B58FB098
:1070600002AA06460C461746174B03F1300C15468C
:1070700018685968083303C563452A46F7D1234683
:107080003021124A38463DF0CDFB3846FAF7F4F885
:10709000192200903B460121304641F083FF051E36
:1070A0000FDA0B4B1E683DF03FFE2346CDE9005042
:1070B00002213046074A41F0A4F86FF015000FB0E6
:1070C000F0BD0020FBE700BFD01B06008F5F06006D
:1070D00088A20120955F06000146008810B50228AD
:1070E00006D1BDE810402823054A04310EF0B8BC93
:1070F0000128F6D00349024849F090F9004810BD34
:10710000C4020220CA5F060003480021034B044A60
:10711000006841F076B800BF88A20120D263060063
:10712000A67D06002DE9F04F01272DED028BBD4D08
:10713000ADF5057DB9420646CDE91A1254682F60B7
:1071400008D8FFF7E1FF00200DF5057DBDEC028BAF
:10715000BDE8F08F2046B449FAF784F840B32046E2
:10716000B249FAF77FF800286CD02046B049FAF708
:1071700079F8002868D02046AE49FAF773F800285D
:1071800065D02046AC49FAF76DF8002862D0204659
:10719000AA49FAF767F800285FD023460221304653
:1071A000A74A41F02EF8FFF7AFFF6FF01500CBE7CD
:1071B00082462B686522013300211DA82B6048F010
:1071C000BDFD6522002137A848F0B8FDC922002185
:1071D00051A848F0B3FD01230893022300254FF086
:1071E000FF380B93012308EE105AA9469B464746E9
:1071F000CDE91855CDE91655CDE91355914C0F95AC
:107200001595CDF83880CDF848801195CDF83480AB
:1072100010950C950A9509930023DDE91A018A4A15
:1072200000938A4B42F0B5FD421C19D10AF1FF30A0
:10723000042800F2D481DFE810F0E701F501FF0136
:1072400003021302BA46B4E74FF0020AB1E74FF067
:10725000030AAEE74FF0040AABE74FF0050AA8E7D0
:1072600078287BDC4128D7DD42383628D4D801A3E2
:1072700053F820F0597501001972010019720100CC
:10728000197201001972010019720100DD74010008
:10729000977301001972010019720100197201003F
:1072A0001972010019720100197201007375010051
:1072B000197201001972010057730100B7740100BF
:1072C00019720100C97401001972010019720100DC
:1072D000197201001972010019720100197201007E
:1072E000197201001972010019720100197201006E
:1072F000B17301009D740100AF750100FD740100C0
:1073000037750100F573010019720100197201004F
:107310008D73010019720100197201002B750100B3
:10732000197201001972010019720100DB7301006A
:107330001972010053750100417501006D7401005F
:1073400019720100197201001972010025750100FE
:107350004FF0010860E7012310935DE7C838062865
:107360003FF65AAF06283FF657AF01A353F820F077
:1073700051730100A97501008D750100937501001D
:10738000997501009F750100A5750100206848F0FE
:10739000F8FB074640E7206848F0F3FB031E0C9318
:1073A0003FF73AAF2A4A0221304640F02AFFFCE676
:1073B0002068F9F761FF6428024608DD6423009322
:1073C0000346244A0221304640F01BFFEDE66523C8
:1073D00021681DA848F085FC1EE7206848F0D1FB15
:1073E0004FF6FE73421E9A4281467FF615AF034662
:1073F000194AD8E719492068F9F734FF002800F046
:10740000D98017492068F9F72DFF002800F0D580B2
:1074100014492068F9F726FF002800F0D18023687E
:10742000114AC0E7446D01204B140800D55F0600E7
:10743000D388070025140800DA5F0600CE8806000E
:10744000DE5F060034CF01201D6306005865012071
:10745000F75F06001F6006004B60060084600600B0
:10746000896006008F600600966006007E492068ED
:10747000F9F7F8FE002800F0A6807C492068F9F7AB
:10748000F1FE002800F0A28079492068F9F7EAFEB1
:10749000002800F09D802368764A84E7206848F041
:1074A00070FB4FF6FE73421E9A420A907FF6B4AE0E
:1074B0000346714A77E7206848F063FB031E0D938B
:1074C000BFF6AAAE6D4A6EE7206848F05AFB022864
:1074D00003460B907FF6A0AE694A64E72068F9F78F
:1074E000CBFE642804DD6423664A0093034669E703
:1074F0006522216837A848F099FF8DE62068F9F7E2
:10750000BBFEC8280ADD236802210193C8235E4A16
:1075100000930346304640F074FE46E6C9222168D7
:1075200051A8E8E70123139376E6206848F029FB89
:1075300008EE100A70E6206848F023FB12906BE614
:10754000206848F01EFB031E0E933FF765AE4F4ABE
:1075500029E7012314935FE6206848F012FB012815
:1075600002D923684A4A1EE700F0010308931593E5
:1075700052E648492068F9F775FE58B34649206835
:10758000F9F770FE48B32368444A0CE701231693C9
:1075900042E6012317933FE6012318933CE60123BB
:1075A000199339E6012537E64FF0000834E6012348
:1075B000119331E64FF0010B2EE64FF0020B2BE654
:1075C0004FF0030B28E60123099325E60223FBE78E
:1075D0000323F9E701230F931EE60223FBE737ABF2
:1075E00006930B9B58460593119B099904930D9B99
:1075F0001DAA0393109B02930C9B01930A9B00937B
:107600004B4600F0DBFB9FE5139B18EE102A02931C
:107610000E9B38460193089B51A90093129B00F0E2
:1076200051FE91E50F9B18EE102A00933846159BEA
:10763000149900F033FF87E5384600F08BFF83E5AF
:107640007B1C03D1404600F0A1FF7DE5199B384625
:10765000009316990195DDE9172300F0DDFF73E52E
:1076600001F034F870E500BF292C0800FF60060027
:10767000F9C707000561060069610600A7610600F9
:10768000DF61060012620600446206007C620600AA
:10769000A6620600DE620600E2620600E6620600FE
:1076A0002DE97F4315461C460646F8F70BFF80463A
:1076B000894628462146F8F751FF02460B464046C8
:1076C0004946F9F7A3F800220F4BF8F775FFCDE90B
:1076D000020121462846F9F767FBDFED0C7A07EE39
:1076E000100AC7EE277A17EE900AF8F70DFFCDE9DA
:1076F0000001074833460021064A006840F081FD3A
:1077000004B0BDE8708300BF0040BF4000007A4471
:1077100088A20120507C060038B50025064C237F46
:107720001BB1002160683FF003FD0135092D04F114
:10773000A004F4D138BD00BF488101202DE9F04FED
:1077400080460E460024DFF85090DFF850B097B026
:10775000B44202D317B0BDE8F08F371B082FA8BF83
:107760000827002508EB040ABD4208DB09485A46F1
:107770000021006801AB40F044FD3C44E8E705EB24
:10778000850001AB49461AF8012B18443DF07EF8FC
:107790000135E9E788A201209F7C0600A57D06004F
:1077A000421C034613B508D1114B0221114A186837
:1077B00040F027FD002002B010BD092808D9092299
:1077C0000B48009202210C4A006840F01AFDF1E7D4
:1077D000A0220A4802FB0300047F002CEBD10448DE
:1077E00002210068064A40F00CFD2046E3E700BF96
:1077F00088A20120A77C0600D47C060048810120D5
:10780000087D060038B50546006A0C4630B16B6A43
:107810008B4214D10A46002148F090FA01216C6293
:1078200060183AF013FF0446286258B9064802214E
:1078300000686B6A054A40F0E4FC204638BD3BF026
:1078400045FEEBE70120F9E788A20120247D060030
:1078500038B504464FF0FF324FF0FF33194804F1BA
:10786000600537F077FC284638F046FA002808DD36
:10787000284638F009FB144B0021144A186840F0E0
:10788000C0FC206A08B13BF021FE237F13B1606881
:1078900005F040FEE06D41F041FA9822002104F12C
:1078A000080048F04BFA4FF0FF330122C4E90033DF
:1078B00084F83820636584F859200248BDE83840D0
:1078C00037F042BD3876012088A20120607D060095
:1078D00073B50D46044616469DF8181053B11A4B61
:1078E000186831B30021194A40F08BFC3146284614
:1078F000FFF724FFE3686068022B21D1A368012B06
:107900001CD0022B14BF00231823E26D9269CDE92D
:10791000002300233246294641F0AFFA002806DA58
:1079200000220321606805F02BFE4FF0FF3002B00B
:1079300070BD2B46064A40F064FCDBE70823E4E711
:107940000023CDE90033E5E788A20120807D060011
:10795000937D0600F7B5446B217F04F1600559B9AA
:1079600017482368174A006840F04BFC284603B0CC
:10797000BDE8F04038F088BA90F8383020460093DF
:10798000D4E908120123FFF7A3FF4FF47A714FF4F3
:10799000004040F2E7360027D4F890304FF47A7276
:1079A0005943E0FB0167002330463946F9F78AFA6C
:1079B00002460B46284603B0BDE8F04038F05EBAF8
:1079C00088A20120AA7D06002DE9F04F2DED028B43
:1079D00004464FF0000ADFF838B187B00027236B68
:1079E000002B1CDC002584F828503FF0B4FBD4E9C0
:1079F0001023C4E91001821A206A61EB030330B13D
:107A0000CDE904233BF062FDDDE904236562E06A11
:107A100007B0BDEC028BBDE8F04FFFF741BE626AD4
:107A2000934208D20021206A48F088F96C21226B29
:107A3000206A48F083F9216A08460491F9F71CFC92
:107A400000230246049920460097FFF741FF0028D3
:107A500007DA012384F8283007B0BDEC028BBDE8BB
:107A6000F08FE36A0344E362236B181A20633FF04C
:107A700072FBD4E91032C51A61EB02062846314682
:107A8000F8F76CFD02460B4643EC182B52465B465A
:107A9000F8F7BCFE8046606B8946F8F723FD024686
:107AA0000B4640464946F9F717F8002897D0E76A91
:107AB0003846F8F707FD53EC182BF8F7A7FE00221D
:107AC0000F4BF8F779FDCDE9020131462846F9F769
:107AD0006BF9DFED0C7A07EE100AC7EE277A17EE86
:107AE000900AF8F711FDCDE9000107483B46002157
:107AF000064A006840F085FB636B0A3363636DE7F9
:107B00000040BF4000007A4488A20120E87D0600C2
:107B100000408F402DE9F04F0025DFF8248299B016
:107B2000002301261F469C464FF0050E844A117F14
:107B300099B1546818A800EBC70040F8484C92F877
:107B40002840F900002C0CBF3446744620F8444C01
:107B500018A8014421F842CC01370133092B02F166
:107B6000A002E4D17FB9774837F084FD15B12846EB
:107B700047F0E1FF4FF0FF324FF0FF33714837F02D
:107B8000EFFC0025CCE74FF47A72394606A80BF0DB
:107B900083FB0028C4DD0023DFF8CC9106AC0393FF
:107BA000039B9F42BCDD43460026226859688A42F7
:107BB0000ED1A023734308EB030A58F80330B342F5
:107BC00000F0A5807621604B604A61483AF020FDC4
:107BD0000136092E03F1A003E8D1039B08340133D9
:107BE0000393DDE74FF0A00B0BFB068B9BF858309F
:107BF00033B13FF0B0FA0023CBE910018BF85830D5
:107C0000206800234FF4C062CDE90033294641F0DB
:107C100064F9031E0493E0DD4FF0A00B3FF09BFAE4
:107C20000BFB068B049B0246CBE91201DBF85000EC
:107C30001844DBF85430CBF8500098420ED3DBF8F0
:107C400044300593DBF84030D21A059B61EB030307
:107C5000FFF726FD4FF0FF33CBF854304FF0A00B69
:107C60000BFB068B9BF8383083B1049B00210093FB
:107C7000384A3346D9F8000040F0C3FA9BF859302F
:107C8000022B3CD128460499FFF758FD4FF4C062FF
:107C90000021284648F052F8E3885B0702D5504699
:107CA000FFF792FEE38818070BD52368D9F8000088
:107CB000009300213346284A40F0A3FA5046FFF7CC
:107CC000C7FDE388D9060BD52368D9F800000093D7
:107CD00000213346214A40F094FA5046FFF7B8FDA0
:107CE000E3889A067FF579AFD9F800003346002182
:107CF0001B4A40F086FA5046FFF7AAFD6DE72B4677
:107D00000021184AD9F8000040F07BFABEE7E3886A
:107D1000DB07C1D5002D7FF465AF012140F2016082
:107D200047F014FF054600287FF45CAF0E484FF47F
